:020000040000FA
:040000006FD00400B9
:101000006F00907E00000000000000009020002093
:10101000AA220020A9BDF9F56C23002000000000E1
:10102000000000006C230020902000200000000041
:101030000000000090200020000000009020002010
:101040000000000090200020902000209020002030
:101050009020002090200020582F00209424002071
:101060000000000090200020902000201E2400207E
:1010700090200020D22300209020002090200020EB
:101080009020002090200020902000209020002020
:101090009020002001A04111B7170040985F3AC688
:1010A000945F3247E39CE6FE3245410182800111A4
:1010B00013078008F337078093F787083EC20100C3
:1010C0000100B7170040930570052380B70413068D
:1010D00080FA2380C7040100010083C6B70493F699
:1010E000F60DA385D704238007049246F3A6068055
:1010F0000100010093760502D5CEF336078093F602
:10110000860836C4010001002380B7042380C70489
:1011100001000100B70614007D89558D88C70100C4
:1011200001000100010023800704A246F3A6068007
:101130000100010073370780137787083AC6010062
:1011400001002380B7042380C704010001000100CF
:1011500001003727004093061005A303D7802380A2
:101160000704B247F3A70780010001009307800836
:10117000F3B7078093F787083ECE01000100B71749
:101180000040130770052380E704130780FA2380CB
:10119000E7040100010003C7B70413670708A3852C
:1011A000E70423800704F247F3A70780010001004A
:1011B0000561828093760504BDC6F336078093F6F9
:1011C000860836C8010001002380B7042380C704C5
:1011D00001000100B7061400938606047D89558D31
:1011E00088C7010001000100010023800704C246F6
:1011F000F3A6068001000100733707801377870884
:101200003ACA010001002380B7042380C70401000B
:1012100001003727004093062005A303D7802380D1
:101220000704D24781B773370780137787083ACC12
:10123000010001002380B7042380C70401000100DE
:1012400098471367070C98C723800704E24719BF24
:101250000111814601468145114506CE97000000E7
:10126000E780605893078008F3B7078093F78708F3
:101270003EC601000100B717004013077005238028
:10128000E704130780FA2380E7040100010003C785
:101290006704136717002383E70423800704B2471A
:1012A000F3A7078001000100F2400561828041112F
:1012B000814601468145114597000000E780A05214
:1012C00013078008F337078093F787083EC40100AF
:1012D0000100B7170040130670052380C70493066A
:1012E00080FA2380D70401000100FD552396B70240
:1012F00023800704A245F3A5058001000100733790
:101300000780137787083AC6010001002380C704CD
:101310002380D7040100010003C767041367170087
:101320002383E70423800704B247F3A70780010063
:10133000010001A0BD473305F50201007D1575FDD3
:101340008280411122C426C206C6AA8401446317C2
:101350009400B24022449244410182800504130566
:10136000803E420497000000E78000FD4180C5B741
:101370009305000273A04580824573901534924016
:101380002242B2424243D2436244F2440255925551
:101390002256B2564257D2576258F25806499649D9
:1013A000264AB64A464BD64B664CF64C065D965DD1
:1013B000265EB65E465FD65F09617300203041113C
:1013C000B7170040985F3AC6945F3247E39CE6FE49
:1013D000324541018280B71700401307000323887C
:1013E000E702854717170000232EF74673002030C9
:1013F000411122C42D6426C24AC006C637190040D6
:101400001304A4AAB704002023208900977000E0E9
:10141000E780A0169C408297977000E0E780E01577
:10142000E5B737370040834747009146BD8B639E41
:10143000D702B73600401306F00F973500009385AA
:10144000651E9737000083D7E72D03C7A6001377E3
:10145000F70F1DE3B7E70400BC4F09468945171590
:1014600000000345A5F7829731A099466394D70001
:10147000834757007300203003C786001377F70FA8
:10148000E365F6FC13851700AE9717380000231BA1
:10149000A8282380E70075B7B787004003C7670017
:1014A000098B6309071003C77700930600031377BE
:1014B0000703630DD708173800000348F87C173678
:1014C0000000130666790547B30606012380E6008F
:1014D00083C57700173700001307077A429793F503
:1014E000F50F2300B70003C58700973500009385EB
:1014F000A577C2951375F50F2380A5000347070054
:1015000089451377F703630CB70C63E7E50A6306B5
:10151000071A8545630CB7129737000083C7D77643
:101520003307F600034707001377F70F19CB85073A
:1015300093F7F70F3D476363F71A17370000A305CA
:10154000F774B787004009472383E700B787004057
:1015500083C77700E207E18763DE0704973700005F
:1015600083C79772173700001307076F3E978546AA
:101570002300D70017370000130707703E97930624
:1015800000032300D700173700001307E76D3E97CD
:10159000A14685072300D70093F7F70F3D47636403
:1015A000F71417370000A301F76EB787004009470B
:1015B0002383E70073002030930610026300D70EE8
:1015C000930620026305D70693060002E316D7F4BC
:1015D00003C727021377C70F13672700D5A803C7D0
:1015E00067001377070465CB03C7A702173800000D
:1015F00013080848173500001305453F134707082F
:101600002385E70203C7A7021377370F1367870005
:101610002385E702814713070004B305F5008C41D9
:10162000B306F80091078CC2E399E7FEF5B503C74E
:10163000A702134707042385E70203C7A70213770E
:10164000C70F136727002385E702F9B503C76700B3
:101650001377070449C303C767021738000013084C
:10166000E834173500001305252C1347070823839A
:10167000E70203C767021377370F136787002383D7
:10168000E702814713070004B305F5008C41B30658
:10169000F80091078CC2E399E7FEBDBD03C767025E
:1016A000134707042383E70203C767021377C70FB3
:1016B000136727002383E70285B503C76700137705
:1016C000070411CB03C727021377370F136787006F
:1016D0002381E70291B5238006003DBD97370000C6
:1016E000A384075AB9BD97370000A38F075875BD6B
:1016F0002303048015472303E48001002302A48010
:10170000828083076480E3CE07FE23030480828007
:1017100083076480E3CE07FE03454480828083070D
:101720006480E3CE07FE2302A4808280411126C498
:101730004AC24EC006C61377F50BAD47AA892E895B
:101740009544630CF700194597000000E78080FA84
:1017500097000000E78020FB8D444E859700000035
:10176000E78040F9FD59FD1463983401B240A2446A
:101770001249824941018280135509011375F50F01
:1017800097000000E780E0F92209F1BF011126CCA3
:1017900006CEB704080097000000E780C0F61545A4
:1017A00097000000E78000F597000000E78080F6D2
:1017B00097000000E78000F62AC697000000E78047
:1017C00080F432459377150089EB13651500137586
:1017D000F50FF240E24405618280FD14E9F0014515
:1017E000CDBF397126DC4ADA4ED852D656D45AD2F9
:1017F0005ED006DE62CE66CCB7E700E07D5783AAF6
:10180000070022C603AA470023A0E71823A2E7186F
:10181000B7170040130770052380E704130780FA09
:101820002380E70483C74704930B75FFB684E20760
:1018300093FBFB0F8546AA892E8B32893724004003
:10184000E187015763FA76016308D50089461307DB
:1018500000026313D5000157D98F93F7F70FB71C18
:1018600000402382FC0411472303E4801305F00F9A
:1018700097000000E78000E8094C97000000E7802F
:1018800080E863657C15B7050700DA9537870700A0
:10189000795563FEE504B3879500636AF704370B57
:1018A0000800A94733EB65016395F90881E8814495
:1018B00097000000E78020E5268515A8DA85094510
:1018C00097000000E780C0E605090345F9FFFD1415
:1018D000050B97000000E780C0E481C49377FB0FFD
:1018E000E5F797000000E780A0EA69F17D55B7179A
:1018F0000040130770052380E704130780FA238054
:10190000E70403C74704418B2382E704F250B7E79B
:1019100000E023A0571123A24711E2543244525948
:10192000C259325AA25A125B825B724CE24C21615C
:101930008280A547639BF90685691309F00FB306FA
:101940009900B3742B01B6941349F9FFB37499004D
:10195000856B33796901416B9387F9FFB3F72701F1
:1019600099E363FC340193D94900C147E3E637FFAB
:101970003DBF0569C1697D19D9B71305800D63881D
:101980006901130500026384790113051008CA85F3
:1019900097000000E780C0D997000000E78040DF93
:1019A00031D54E99B38434416DBFDA852D4597000A
:1019B0000000E780E0D7CA94E30B99EE0509970091
:1019C0000000E78020D5A30FA9FEFDB79387F9FF9C
:1019D00093F7F70F636DFC0C83C71C0413073008E3
:1019E0006315F706370708006361EB06B3079B0032
:1019F000B706100063FBD704334BEB0089476399AC
:101A0000F9068980D549E38404EADA850945970017
:101A10000000E780E0D111090327C9FF9147232087
:101A2000E48003076480E34E07FE23033481FD173F
:101A3000EDFBFD14110B81C49377FB0FE9FF9700B9
:101A40000000E780E0D461F155B5B717004003C747
:101A50005704B70708001377070219E3B787070091
:101A60007955E376FBE833079B00E3F9E7F841B5E6
:101A70008547E380F9F0DA852D4597000000E7807F
:101A800020CB9389F4FFE38404E297000000E78011
:101A900060C893F7390091EB83260480032709007F
:101AA00093074900E396E6E03E89CE84D9BFB54767
:101AB0006399F9001305900B97000000E78080C33D
:101AC000FDB3B1471305B00AE388F9FE9947639760
:101AD000F904B7050800B365BB002D459700000069
:101AE000E78000C581448D4BA14997000000E78045
:101AF00060C263967401832704802320F900850463
:101B0000E39534FF8327048013172B0163550700E7
:101B10002312F90069BB2322F90051BB9D47639F43
:101B2000F90281451305B00497000000E78040C02A
:101B3000BD442320090023220900FD59970000001D
:101B4000E78040BD93F77400CA9703C70700FD14F0
:101B5000398D2380A700E39334FF91BBA14763979E
:101B6000F90697000000E780A0C28144630D0B00D6
:101B70008D479304C0036308FB00930400056304CE
:101B80008B01930440041375C507E30295D21945F0
:101B900097000000E78000B697000000E780A0B63D
:101BA000054597000000E780E0B426859700000017
:101BB000E78020B7094597000000E78080B69700CE
:101BC0000000E780E0BCE31405CE0DB39147639FAE
:101BD000F9001305600697000000E780A0B19700A8
:101BE0000000E78040B213059009F9B5E38109CC04
:101BF000F1547DB9BD66014717360000130606355E
:101C0000938606A685458347060093F7F70F91C391
:101C100082800507E3F9E6FE973700002388B73294
:101C2000DDB77D166206618693178601E18763D46E
:101C3000070001458280931726003307F500AE9711
:101C400018439C4363E7E7007D16E37FF7FC7D556F
:101C5000828005458280FD15E205E18513978501A7
:101C6000618793F7F50F63480700FD15139725006B
:101C70002A97584365D713851700620561858280CE
:101C80003308B5021C4283A80600B335B502C297DB
:101C900033B50701AE98469585486367B5006394F0
:101CA000A50063E3070181480C43C6950CC388C2B5
:101CB0001CC2828081471397870161876343B70005
:101CC0008280139727002A97232007008507E5B70E
:101CD0008147014793968701E18663C5B6001335B6
:101CE0001700828093962700AA9694428507558F05
:101CF000D5B793D755408A07AA979C430545331516
:101D0000B5007D8D828017F3FFDFE702833D2A84D3
:101D100097000000E78060F405C5931725003E9406
:101D20000327C4FF814711EB7D1516053E9542053B
:101D3000418517F3FFDF6700033D05838507E5B79E
:101D40000145C5BF81471397870161876343C7007A
:101D5000828013972700B386E50094422A9785076F
:101D600014C3D5B77D1662066186014793178601B5
:101D7000E18763D50700133517008280931726008B
:101D8000B306F500AE9794429C437D16B58F5D8FE8
:101D9000F1BF8A05AA9501476363B500828083A6D7
:101DA000C5FFF11593D71600D98F9CC11397F60183
:101DB000E5B72A830148014701456343D700828084
:101DC000B387050183A80700B30706019C43C697A4
:101DD000AA976384F80033B517010507B308030118
:101DE000620723A0F80061871108C1BF2A83014759
:101DF0008147014563C3D70082803388E50083288B
:101E00000800330EE600032E0E003388A840330886
:101E1000C8416384080133B508018507B308E300AE
:101E2000E20723A00801E1871107E9B717F3FFDFF5
:101E3000E702232B0111B286B2842E86AA850A8579
:101E400097000000E780C0FA2A84A6850A859700DB
:101E50000000E78020E833348000060413351500C5
:101E6000018D056117F3FFDF6700E32917F3FFDF3B
:101E7000E702A3244111AA89AE8A328BB68402C23A
:101E800002C402C60144131C8401135C8C416349E3
:101E90009C02939B1400FD1B0549138CF4FFF15C1D
:101EA00033048901620461846340740792478E049D
:101EB000CE9423AEF4FE410117F3FFDF67006323E6
:101EC00013192400B30B2B01014A93172A00D6974C
:101ED00083A50B0088437800340050009700000071
:101EE000E78040DA050A93178A01E187F11BE35E78
:101EF000FCFC92474E9905042320F900A2473EC2FC
:101F0000B24702C63EC441B7131A8901135A8A4127
:101F1000131D240093178A01E18763CF970092472E
:101F20000A044E941CC0A24705091379F90F3EC25A
:101F3000B24702C63EC4ADB7B3079A0313152A00D1
:101F400056950841780034005000050AEA97DA9760
:101F50008C4397000000E780E0D26DBF197106C284
:101F600012C416C61AC81ECA22CC26CE2AD02ED219
:101F700032D436D63AD83EDA42DC46DECAC0CEC2C9
:101F8000D2C4D6C6DAC8DECAE2CCE6CEEAD0EED2F9
:101F9000F2D4F6D6FAD8FEDA971500009385058CB0
:101FA0008841E700050092402242B2424243D243B8
:101FB0006244F244025592552256B2564257D257C5
:101FC0006258F25806499649264AB64A464BD64BBD
:101FD000664CF64C065D965D265EB65E465FD65F45
:101FE0000961730020300000972100209381810156
:101FF000175100201301018117F5FFFF1305C500DC
:102000009705002093850500171600201306C6FDCE
:1020100063FAC5008322050023A055001105910530
:10202000E3EAC5FE17150200130545F597150020D4
:102030009385C5FB171600201306C66563FAC50015
:102040008322050023A0550011059105E3EAC5FE92
:102050001715002013050564974500209385053B5F
:102060006377B500232005001105E36DB5FEFD4241
:10207000739002BC8D4273904280B722000093821D
:10208000828873900230970200209382A2F793E235
:1020900032007390523097520000938222C27390A4
:1020A00012346FB0F47573002030397101436EC67D
:1020B00019A0397141536AC866CA62CC5ECE19A0B4
:1020C000397101535AD056D252D44ED64AD826DA54
:1020D00022DC06DE33016140828241114AC026C201
:1020E00022C406C68282B24D4101024D924C224C5E
:1020F000B24B4101024B924A224AB2494101024984
:1021000092442244B240410182803D432A87637356
:10211000C3029377F700BDEFADE5937606FF3D8AE6
:10212000BA960CC34CC30CC74CC74107E36BD7FE30
:1021300011E28280B306C3408A0697020000969699
:102140006780A6002307B700A306B7002306B700E1
:10215000A305B7002305B700A304B7002304B70005
:10216000A303B7002303B700A302B7002302B700FD
:10217000A301B7002301B700A300B7002300B700F5
:10218000828093F5F50F93968500D58D9396050182
:10219000D58D61B7939627009702000096968682A8
:1021A000E78086FA9680C1171D8F3E96E374C3F8C8
:1021B000A5B73367B500FD530D8B79E7B7877F7FF0
:1021C0009387F7F710419441B372F6003363F6003A
:1021D000BE92B3E262006397720C6318D606504158
:1021E000D441B372F6003363F600BE92B3E26200EC
:1021F0006398720A631BD60410459445B372F600C7
:102200003363F600BE92B3E262006391720A631E0A
:10221000D6025045D445B372F6003363F600BE9241
:10222000B3E26200639A72086311D60210499449BE
:10223000B372F6003363F600BE92B3E262006393BA
:1022400072085105D105E30FD6F6131706019397CF
:102250000601631CF7001357060193D706013305E7
:10226000F7409375F50F91E982804183C18333056F
:10227000F7409375F50F91E182801377F70F93F78D
:10228000F70F3305F74082800346050083C605003B
:10229000050585056313D60065FA3305D6408280AF
:1022A00011059105E312D6FE014582802105A105A5
:1022B000E31CD6FC014582803105B105E316D6FC4E
:1022C000014582804105C105E310D6FC01458280AD
:1022D000B717004003C777051377E70FA38BE70411
:1022E000130700F8A38DE7043D47238CE704130789
:1022F0005003A38CE70403C7A7051377D70F238DDB
:10230000E7048280B717004003C7E7020D89411137
:102310001377C70F498F93068008F3B6068093F6AC
:10232000860836C601000100930670052380D70495
:10233000930680FA2380D704010001002387E70277
:1023400023800704B247F3A7078001000100410181
:10235000828041112A83014E930E407E130F001993
:10236000930F400663E56E129308001913034006AD
:10237000B3781503854E0D4FA14F337365020D8958
:102380001335150063EFBE121308F6FF79467298F5
:102390004208135808013307C70213D61700BE07B7
:1023A00032976146B3F6C60213068070B386C60242
:1023B0003697A166F58F42075D8FB716004083C739
:1023C000F60293F70708A303F1000346710083C7E1
:1023D000F60293F70708E394C7FE83477100B71628
:1023E000004093F7F70F6388071293078008F3B74D
:1023F000078093F787083EC401000100B71700402B
:10240000930670052380D704930680FA2380D704AF
:102410000100010023AA070383C6170393E60608F9
:10242000A388D70223800704A247F3A707800100EF
:1024300001001166B71700407D16D45BC85F938515
:102440004703A98EF18EF5FA93068008F3B606804D
:1024500093F6860836C601000100930670052380B6
:10246000D704930680FA2380D7040100010098C1A5
:1024700003C7170313670704A388E7022380070431
:10248000B247F3A7078001000100410182807D135C
:102490003368E3039308E016630E08003368F30320
:1024A0009308D016630808009378330093B8180097
:1024B0009388D81633081E01131E0801135E0E01FF
:1024C00055B56393E5030548638608000148630337
:1024D00003002A8871087298FD15131E0801C205B1
:1024E000135E0E01C18179BD13F8150063F4BF00BE
:1024F0007908D5B713381800E5BF83C7F60293F7FC
:102500000708A303F1000346710083C7F60293F79F
:102510000708E394C7FE8347710093F7F70FF1DFD5
:10252000E9B531714AD966CB06DF22DD26DB4ED70D
:1025300052D556D35AD15ECF62CD6AC96EC7AA8C26
:1025400002D897100000E78020B12A8993078008FD
:10255000F3B7078093F787083EDA01000100B71749
:102560000040130770052380E704130780FA2380D7
:10257000E7040100010003C7F7021377770FA38771
:10258000E70203C7F70213678700A387E7022380E8
:102590000704D257F3A70780010001000545970003
:1025A0000000E78060D6130780C13347E902116A53
:1025B00093070AE893065002BD69930BA004814A71
:1025C000014B13048008930470057D1AB347F90288
:1025D0003307D7023EC0FD873ECC938709A69309F7
:1025E000803E3347F7023AC27D873AC43347390306
:1025F0008549B399990193D93940B306D702B30BF2
:102600007703B3C6F602B3CBFB0236C6FD8636C8E7
:1026100093D6FB4136CEB7460F0093860624334946
:10262000D9028566938606FAB3969601B389E902C4
:10263000130760553309D90293060010B389E902E4
:102640003349D902B3C9F9029316390036CA37198A
:102650000040FD8636D0930D090493D7F9413ED250
:10266000F336048093F6860836DC010001009307F8
:1026700070052380FD00930680FA2380DD000100B1
:1026800001008346390593F6860FA309D9048346D2
:10269000390593E61600A309D90423800D00E256FC
:1026A000F3A6068001000100130C80FA116DF336C9
:1026B000048093F6860836DE01000100930770055A
:1026C0002380FD0023808D01010001008346390530
:1026D000216693E60602A309D90483560905B3E6E9
:1026E000A6012318D90483560905D18E2318D904CD
:1026F00023800D00F256F3A60680010001008346F8
:10270000390593F606026381061A03463905218AC4
:102710006DDE081897100000E7800098733604807B
:1027200013768608B2C20100010023809D00238039
:102730008D0101000100B717004003C6370513766D
:10274000F60DA389C70403C6370513660602A389DD
:10275000C704835609052166B3E6A6012318D904E8
:1027600083560905D18E2318D90423800D0096467F
:10277000F3A60680010001008346390593F60602A0
:10278000638B061483463905A18AEDFE970000206D
:10279000E7806090AA8636D497000020E780A08F5B
:1027A000A256E30AD5FE835609054255B3E6A601B3
:1027B0002318D90497100000E780C08F834639059D
:1027C000A18AEDDE03560905834629058247337643
:1027D000CA00B306DA0293D5F641B296B388F64042
:1027E000E24733B8C6002E983308F840A247B3B684
:1027F00016013308D84063C70701631DF8009247EC
:1028000063FA1701C247634FF80E63950701B24799
:1028100063EAF80E894663E9660FF24693151800DD
:1028200013D3F8015E8613951800B365B30042D642
:1028300046D497D00100E780A0BA3258050B137B2D
:10284000FB0F63470001631A0838A25863870838F2
:1028500013081500B336A800B69513D6F5013298C3
:10286000B336C800AE9613581800FE06B3E606014C
:102870007336048013768608B2C6010001002380F7
:102880009D0023808D01010001000356C902B2960C
:10289000C206C1822316D90223800D00B646F3A6D4
:1028A00006800100010021B5F336048093F6860806
:1028B000B6C00100010023809D0023808D0101002E
:1028C00001008346390593E60602A309D904238053
:1028D0000D0086460DB5F336048093F68608B6C41F
:1028E0000100010023809D0023808D010100010073
:1028F0008346390593E60602A309D90423800D0017
:10290000A646BDB5E30B0BF0F336048093F68608BC
:10291000B6C801000100930680FA23809D00238041
:10292000DD00010001008346390593F5FC0F93F6A5
:10293000860FA309D90483463905CD8EA309D9048E
:1029400023800D00C646F3A6068001000100130592
:1029500080FA03463905930639051D8A631C9629BA
:102960007336048013768608B2CC0100010013068A
:1029700080FA23809D002380CD000100010003C662
:1029800006001376F60D2380C60003C60600136604
:1029900006022380C600835609051166D18E2318CE
:1029A000D904835609052166D18E2318D9042380C2
:1029B0000D00E646F3A6068001000100130680FA2A
:1029C0008346390593F60602638006268346390559
:1029D000130C3905A18AFDDA081897000000E7807A
:1029E000A06BF336048093F68608B6D00100010090
:1029F000930680FA23809D002380DD000100010002
:102A000083460C00116693F6F60D2300DC00834626
:102A10000C0093E606022300DC0083560905D18EE4
:102A20002318D904835609052166D18E2318D904A9
:102A300023800D008656F3A60680010001001306D0
:102A400080FA8346390593F60602638A0620834698
:102A50003905A18AEDFE97F0FF1FE780C0632A8C3D
:102A600097F0FF1FE7802063E30C85FF835609057D
:102A700011664255D18E2318D90497000000E780D3
:102A800060638346390513063905A18AFDDAF336FA
:102A9000048093F68608B6D401000100930680FAFC
:102AA00023809D002380DD00010001008346060095
:102AB00093F6F60D2300D60023800D00A656F3A64C
:102AC0000680010001008356090503462905D24707
:102AD000B376DA003306CA021305800C9355F6412B
:102AE0003696330DF6408257333CD6002E9C333653
:102AF000A601330CFC40330CCC40330885039256BE
:102B00004E86B335A5033305A503C29597D00100C2
:102B1000E780008D63468001631E0C16630C0D1662
:102B2000130615003335A6002E959356F5013696FB
:102B3000B335D600AA959396F50105828585D18E89
:102B40006346B000639D051A638B061A0356C902DB
:102B500015823305D6003336C500B2956348B00000
:102B6000639105241306F00F637DA622894663F363
:102B7000561593078008F3B7078093F78708BED6EA
:102B80000100010037170040930770052300F70488
:102B9000930780FA2300F704010001008356C7025F
:102BA00089678117D58FC207C1832316F7022300D7
:102BB0000704B657F3A7078001000100FA506A54D2
:102BC000DA544A59BA592A5A9A5A0A5BFA4B6A4C49
:102BD000DA4C4A4DBA4D296182801308F5FF33352E
:102BE000A800FD152E951356F5013298B336C8008E
:102BF000AA9695B9F336048093F68608B6CA010002
:102C0000010023809D002380AD0001000100834668
:102C10003905CD8EA309D90423800D00D646F3A62D
:102C200006800100010035B3F336048093F6860870
:102C3000B6CE0100010023809D002380CD0001005D
:102C400001008346390593E60602A309D9042380CF
:102C50000D00F646F3A606800100010095B3F33699
:102C6000048093F68608B6D20100010023809D00FF
:102C70002380CD00010001008346390593E606025A
:102C8000A309D90423800D009656F3A606800100FF
:102C9000010045BB9306F5FF33B5A600FD152E9543
:102CA0009355F501AE96B3B5B600AA951396F50106
:102CB000858269B5F336048093F68608B6D801009C
:102CC0000100930680FA23809D002380DD0001002F
:102CD00001008356C9020566011693F6F60FD18EE0
:102CE000C206C1822316D90223800D00C656F3A660
:102CF000068001000100850A93FAFA0F95B233E6C7
:102D0000B60045C20356C9023305D0403338A0008F
:102D1000B305B040B385054115826345B000D1E1EC
:102D20006371A608894663F0560593078008F3B7D8
:102D3000078093F78708BEDA01000100B71700404B
:102D4000130770052380E704130780FA2380E70444
:102D50000100010003D7C7027D8B2396E702238081
:102D60000704D65781BDF336048093F68608B6DC97
:102D700001000100930680FA23809D002380DD007E
:102D8000010001008356C9020566011693F6F60F8D
:102D9000D18EC206C1822316D90223800D00E656C9
:102DA000B9B793078008F3B7078093F78708BEDEAB
:102DB0000100010037170040930770052300F70456
:102DC000930780FA2300F704010001000356C702AD
:102DD00093975600B297C207C1832316F7022300C8
:102DE0000704F657C1BB914763EEB70217E701002E
:102DF000130747FD8A05BA959C41BA978287B71792
:102E0000004003A7470B1345F5FF698F23AAE70A84
:102E100003A7070B698F23A8E70A03A7070A798D81
:102E200023A0A70A8280B717004083A6470B134749
:102E3000F5FFF98E23AAD70A83A6070B558D23A881
:102E4000A70A83A6070A758F23A0E70A8280B7170F
:102E5000004003A7470B498F23AAE70A03A7070BE4
:102E60001345F5FF45BFB717004083A6470B13472F
:102E7000F5FF758F23AAE70A03A7070A598D4DB7F7
:102E8000B717004003A7470B498FEDB7914763EE93
:102E9000B70217E70100130727F48A05BA959C418A
:102EA000BA978287B717004003A7470D1345F5FF70
:102EB000698F23AAE70C03A7070D698F23A8E70CE6
:102EC00003A7070C798D23A0A70C8280B7170040B9
:102ED00083A6470D1347F5FFF98E23AAD70C83A6C7
:102EE000070D558D23A8A70C83A6070C758F23A06B
:102EF000E70C8280B717004003A7470D498F23AA2C
:102F0000E70C03A7070D1345F5FF45BFB7170040B2
:102F100083A6470D1347F5FF758F23AAE70C03A778
:102F2000070C598D4DB7B717004003A7470D498FC0
:102F3000EDB7797122D43714004026D24AD0035914
:102F400024028354040206D64209C2044ECE52CC57
:102F500056CA13590901C1802DE11379F9F793F489
:102F6000F49F4209C20413590901C18093078008E4
:102F7000F3B7078093F787083EC401000100930769
:102F800070052300F404930780FA2300F404010081
:102F90000100231124032310940223000404A247F8
:102FA000F3A7078001000100B25022549254025945
:102FB000F249624AD24A45618280B7F507008146EC
:102FC0003000B105194597000020E7808081A247B5
:102FD00013972701E34A07FC1369090893E40440A7
:102FE00093098008F3B7098093F787083EC0010072
:102FF0000100930A700523005405130A80FA230088
:10300000440501000100231124032310940223002E
:1030100004048247F3A7078001000100294597F0C7
:10302000FF1FE7802031F3B9098093F989084EC268
:1030300001000100230054052300440501000100A4
:103040008357040293E707202310F40223000404AB
:103050009247B9B7B7170040884742054181937737
:10306000050491EB9377F5013755E80113050580C9
:103070003345F50282809377050C130700046397AC
:10308000E7009377F50137459C1CCDB72165130503
:1030900005D0828037E700E01C435443A183E20659
:1030A000D58F1CC1FD572320F7182322F7188280E3
:1030B00013178500B7E700E023A0E710618123A282
:1030C000A7108280B7F700E08847CC47828081470D
:1030D00037370040A14663C4C7003285828003456C
:1030E000B740E38EA6FE3385F5000345050085074E
:1030F0002304A740CDB797070020938727EF9C4371
:1031000017370020130787303E95636EE5001737A9
:1031100000201307273F6368A70017070020232715
:10312000A7EC3E858280FD57EDBF8280411122C40D
:1031300006C62A8497000000E78000F22947B307FB
:10314000E502B2408D83B3D7870222449507B3D7F7
:10315000E70237370040C207C1832316F700410159
:103160008280411137150E0006C697000000E780E7
:1031700020FCB7370040130770F82381E7000D47A4
:10318000A381E70013070004A380E7000547238716
:10319000E700B24041018280373700408347270073
:1031A0001A0593F7F703C98F93F7F70F2301F70079
:1031B0008280B737004003C7170019C9D98DA38093
:1031C000B70003C70700136787002380E7008280EA
:1031D00093C5F5FFF98DA380B7008280AE872A875B
:1031E000B736004021463738004089E71703000012
:1031F0006700E3F383C8B600E30916FF05078348B9
:10320000F7FFFD17C20723041801C183F9BF41115D
:1032100022C406C62A8497000000E780E0E329471D
:10322000B307E502B2408D83B3D7870222449507E6
:10323000B3D7E70237370040C207C1832316F740F0
:1032400041018280716541111305052006C6970072
:103250000000E78000FCB7370040130770F82381B7
:10326000E7400D47A381E74013070004A380E74030
:1032700005472387E740B24041018280CC4141119C
:1032800006C6328503C6150083C5050022064D8E8D
:1032900042068D654186138875A2630C0611634B47
:1032A000C804138845A26300060D634AC8009385CD
:1032B00035A26301B6082390060029464DA0138865
:1032C00055A26305060D938565A2E316B6FE8D45EE
:1032D0001D4663E6E5081146198E63F3C7003E8676
:1032E000B7E704002390C600FC4797E501009385EB
:1032F000E5B09DA0138895A263030611634E060DE9
:103300001388A5A263000613938505A5E315B6FAF5
:1033100099451D4663E5E504198E63F3C7003E86B3
:10332000B7E704002390C600FC479705002093856B
:1033300025D61DA09D451D4663E3E5022146198E55
:1033400063F3C7003E86B7E70400FC472390C6003E
:103350009705002093858534BA9582970146B2403F
:10336000328541018280AD451D46E3EAE5FE3146E6
:10337000198E63F3C7003E86B7E704002390C600AA
:10338000FC4797E501009385E5A9F9B7B1451D46CE
:10339000E3E7E5FC3546198E63F3C7003E86B7E7E1
:1033A00004002390C600FC4797E50100938585A89B
:1033B00065B78D451D46E3E4E5FA1146198E63F3C2
:1033C000C7003E86B7E704002390C600FC4797E598
:1033D0000100938565A349B78D451D46E3E1E5F8F6
:1033E0001146198E63F3C7003E86B7E704002390A9
:1033F000C600FC4797E50100938585A5B1BFA545AB
:103400001D46E3EEE5F42946198E63F3C7003E86B8
:10341000B7E704002390C600FC4797E501009385B9
:10342000659F1DBFB5451D46E3EBE5F23946198E94
:1034300063F3C7003E86B7E704002390C600FC474D
:1034400097E501009385859A01BFB7E7040003A3C0
:103450000713970600209386A6C24146A545170587
:1034600000201305E5B802832D455DE703C505007F
:103470000947631FE50803A84500411106C6034735
:10348000180032850346080022074168518F9308CF
:1034900028FE6307170563E9E800051863030703BF
:1034A00023900600294591A8130648FE630AC70425
:1034B0001518E31707FF15463E87637BF60015478F
:1034C00001A8130600023E876374F600130700028A
:1034D000B7E704002390E600FC471316070111A884
:1034E0003E8691C30546B7E70400FC472390C6001B
:1034F0004206CC45418282970145B240410182801B
:10350000130600083E87E375F6FC13070008C9B7E9
:103510002390060005458280828041677917630405
:10352000E504411122C406C685472A84639FF5003D
:10353000B7E7040022852244B24003A3871397050E
:1035400000209385E52F4101028389476399F500A7
:10355000B7E7040083A7070B8545829771D9B2406E
:103560002244410182808280797126D252CCAE847D
:103570002A8A97E501009385A58F17E501001305B9
:10358000A59106D63AC622D44AD0368432894ECE88
:1035900097C00100E7800030A28517E50100130500
:1035A000A59097C00100E780E02E294597C0010053
:1035B000E780203383C7840093F70702F9E383C9C8
:1035C00004008947054532476396F908D44083C70C
:1035D000160083C60600A207D58FC166138616FEA5
:1035E000638CC7028D16638FD7068D6693862690EF
:1035F00029456391D706B7E70400A286225403A3A6
:103600004714B250F2494A86A6850259925452850F
:10361000624A8547456102832D450DEF93070002FD
:10362000354563E98702B7E70400FC47C844130641
:103630000002CA8582978149970700209387072156
:103640009C43014581CB9C4391C74E852286CA8508
:1036500082970145B250225492540259F249624A6B
:10366000456182802D457DF79307700F3545E3E373
:1036700087FEB7E70400FC47C8442286CA858297C4
:1036800065BF2145C1BF411122C437E4040083272F
:10369000841326C2AA84416506C697050020938537
:1036A000251A7D1582978327C40A17050000130584
:1036B00005E78588829795C0032304132244B2400E
:1036C000924497060020938626AE4146C5451705CD
:1036D00000201305659C41010283B24022449244BC
:1036E00001454101828019C59707002023A0A71634
:1036F00001458280454582801147636AA70A97D6B3
:1037000001009386A6750A0536951841411106C633
:103710003697AE87B2850287130700026145639D25
:10372000E700B7E70400FC47130600021705002076
:10373000130545F782970145B24041018280054754
:103740006145E39BE7FEB7E70400FC470546170524
:103750000020130525F7F9BF1307700F6145E39D9E
:10376000E7FCB7E70400FC471306700F17050020BD
:10377000130585F5C1B7130700086145E39EE7FA15
:10378000B7E70400FC4713060008170500201305DF
:1037900025034DB715476145E390E7FAB7E7040005
:1037A000FC471546170500201305C50961B70945F3
:1037B0008280411126C2B7E4040083A7C41322C447
:1037C0004AC006C62E8497050020938565072A897E
:1037D0008297058905C5970700209387E78B83D7D4
:1037E000A70BA28503A3440D2310F4002244B2408A
:1037F00092444A850249014641010283B240224473
:103800009244024949454101828097070020238163
:1038100007049707002023AF0702B717004003A74C
:10382000070CB706C0FFFD16758F23A0E70C03A792
:10383000070DB7064000558F23A8E70C03A7070C18
:103840003D9B23A0E70C03A7070D1367070123A8DF
:10385000E70C8280B717004003A5470C83A7470CED
:10386000598113451500C18B058999E3136525001E
:103870009707002083C7C7FD6380A7029707002032
:103880002388A7FC11C9970700209387A7FC03A3EF
:1038900007006303030002838280114517F3FFFFD3
:1038A000670063C8011122CC06CE3714004026CA37
:1038B0004AC84EC652C483447405034AB4058349BA
:1038C00084050349940597F0FFFFE780A0A0834794
:1038D000A40593F4F40F137AFA0F93E71700230D5E
:1038E000F40493F9F90F1379F90FB717004003C7E0
:1038F000A705058B6DFF03D5C705A38D4705238C51
:103900003705A38C2705A38B9704F2406244D24469
:103910004249B249224A05618280411193970501CB
:1039200022C406C626C2C1872E8463DC0700B7E422
:103930000400FC54829719C1BC5482972165218DE3
:1039400015A893F7150013C515008DE793F725000B
:103950009DC797000000E78020F0B7E70400BC4F48
:103960001306000A894517050020034525EF8297B5
:1039700013452400B240224492444101828093972F
:10398000250163D80702B7E4040083A7C41E829709
:1039900097000000E780A0F0BC4C375607001306E4
:1039A0000630896517050020034545EB82970965B8
:1039B00079B7939715010145E3DE07FA17D50100A2
:1039C0001305855697C00100E780A004B7E70400FF
:1039D000BC4F13060064916517050020034505E8F8
:1039E00082971165A9BF1D71A2CC37E404005C5C0D
:1039F000485886CE494697D501009385654E8297F3
:103A000011E917D501001305E54E97C00100E780C5
:103A1000400001A0B7F600E0795798CAFD57DCCA0C
:103A20000567B7E700E023A0E7101306F00290C295
:103A300023A0E718010001003707002018471306EC
:103A4000000481459706002023A8E6E04157A38A99
:103A5000E7403C4408088297970700209387077C3B
:103A60003EC8856713870740938757D1231AE10023
:103A70002312F1021307B00F97F7FFFF9387C76474
:103A80002310E1023ED81547970700009387C7E14E
:103A9000B7F50700A30FE1003EDC054797070000DC
:103AA0009387E7DF81463000E10519452301E102F4
:103AB0003EDE97F0FF1FE780C0D218088147994685
:103AC00030003E960346060085070507A30BC70096
:103AD000E398D7FEC24791C70357410185676373D7
:103AE000F70001A0B7E7040083A7470A08088297F8
:103AF000AA8511C917D501001305054197C001001A
:103B0000E78040D901A0F6406644256182804111DA
:103B100026C2B7E4040083A7040806C622C417051A
:103B200000001305C5DF829717040020130404D397
:103B30002300A40097000000E780800297000000A7
:103B4000E780E0CC03450400224403A38405B2408F
:103B5000924413060032896541010283797106D6C9
:103B600022D413078008F337078093F787083EC2F3
:103B700001000100B7170040930570052380B704CA
:103B8000130680FA2380C7040100010083C6F702F0
:103B900093F6A60FA387D702238007049246F3A6C5
:103BA00006800100010073370780137787083AC445
:103BB000010001002380B7042380C7040100010035
:103BC00003C7F70213672700A387E70223800704D0
:103BD000A247F3A7078001000100054597E0FFFF1A
:103BE000E780807297000000E78060CB0147814644
:103BF0008147054685451305407E97E0FFFFE78036
:103C0000807537E404003C44680051468145829742
:103C1000B707C0A83EC8B787E803938707D03ECA56
:103C200097E7FF1F9387A7793EC67C586800829765
:103C3000B250225445618280411197E5010093857D
:103C4000A59317D501001305252506C697C00100C9
:103C5000E78040C417E50100130505AB97C00100DC
:103C6000E78040C3B2402945410117C30100670006
:103C700043C7411197E501009385459117D5010090
:103C80001305852106C697C00100E780A0C017E58F
:103C90000100130525A697C00100E780A0BFB24030
:103CA0002945410117C301006700A3C3411122C484
:103CB00006C6834705002A849DC797E501009385C2
:103CC000A59217D501001305251D97C00100E780B7
:103CD00060BC4C4017E50100130545BB97C00100CF
:103CE000E78040BB3DA058410DEF97E5010093856B
:103CF000A58F17D501001305251A97C00100E7808D
:103D000060B917E501001305E5B997C00100E78028
:103D100060B82244B2402945410117C30100670041
:103D200043BCA1679386D7036313D70297E50100CD
:103D30009385858B17D501001305051697C00100E3
:103D4000E78040B517E501001305C5B67DBFED0757
:103D500097E501009385458917D501001305C51323
:103D6000631BF70097C00100E780C0B217E50100B0
:103D7000130585B559BF97C00100E780A0B14C403D
:103D800017E50100130545B691BF411197E5010004
:103D90009385058117D501001305051006C697C048
:103DA0000100E78020AFB2402945410117C301005F
:103DB000670023B3397122DC26DA4AD82E842A8997
:103DC0008145B2844808714636C606DE97E0FFFF9B
:103DD000E780E03397F7FF1F9387075EDC4783D7C1
:103DE0000700231C2101231BF10097600000E780DE
:103DF000E0C1B246230DA10091E285469307001968
:103E00003ECE2686FD57A2854808A30DD100230289
:103E1000F10297600000E78040C2F2506254D25431
:103E20004259216182808546170300006700C3F86C
:103E30004111972700202396078E97170020238F84
:103E4000077C06C6170700200347C72D9307F00A13
:103E50006315F7029307F0F889451705002013054D
:103E6000652C17070020230FF72A97070020A38B44
:103E7000072A97600000E780A07A97700000E7802B
:103E800060A797700000E780A0A88145370504006F
:103E90009707002023AE07269707002023890726CF
:103EA000970700202398071E970700202396071CDA
:103EB00097070020239B072497070020239C0724B3
:103EC00097400000E780600C014597600000E780A4
:103ED000207ED14717070020231AF722B7E70400F6
:103EE000BC4F13060014894517050020034585972C
:103EF000829797D501009385256D17D5010013058D
:103F0000A5F997C00100E780E0989705002083D5C8
:103F1000E51F17E50100130565A397C00100E780C1
:103F20006097B2402945410117C301006700639BB8
:103F30004111814617F6FF1F1306464585451705B3
:103F400000200355251306C697D00000E7804006E1
:103F500015C997D501009385E56717D501001305AD
:103F6000A5F397C00100E780E09217E50100130573
:103F7000E58D97C00100E780E091294597C00100D9
:103F8000E780209697D501009385C56417D5010079
:103F9000130585F097C00100E780C08F17E5010089
:103FA0001305058C97C00100E780C08E294597C096
:103FB0000100E780009397F7FF1F9387E73FDC47F7
:103FC000054797D501009385E5602390E70017D555
:103FD0000100130565EC97C00100E780A08B17E591
:103FE00001001305258997C00100E780A08AB2402F
:103FF0002945410117C301006700A38E411122C466
:1040000097D501009385855F2A8417D50100130594
:10401000A5E806C697C00100E780C0874C4017E5B9
:1040200001001305258097C00100E780A08629457F
:1040300097C00100E780E08A034704009307F00F70
:10404000631FF70297D501009385455B17D50100E3
:10405000130585E497C00100E780C0834C4017D565
:1040600001001305257D97C00100E780A08222444E
:10407000B2402945410117C3010067008386B24061
:10408000224441018280411122C426C22A84AE8486
:1040900017D50100130545E097D501009385C5515B
:1040A00006C697B00100E780E07E17E50100130522
:1040B000658897B00100E780E07D294597C0010041
:1040C000E780208297D501009385054F9707002050
:1040D000239287FA17D50100130505DC05449707DD
:1040E0000020239797F897070020239487F89717C5
:1040F00000202398976297B00100E780A079971578
:10410000002083D5056217E501001305258397B0CC
:104110000100E7802078294597B00100E780607CA6
:1041200097170020238C874E97F7FF1F9387C72888
:10413000DC4717F5FF1F0345E57203D70700C1678A
:10414000FD17631EF700B7E7040003A387051306F6
:10415000000A85452244B240924441010283B7E7F8
:10416000040003A387051306001493050010DDB7B0
:10417000B1C1411122C417D501001305E5D12E8428
:1041800097D501009385854206C697B00100E78068
:104190006070A28517D501001305057997B001005D
:1041A000E780406F2244B2402945410117B3010026
:1041B000670023738280B7E70400FC471171A2DD1A
:1041C000CAD986DFA6DBCED72E8432892E86AA8571
:1041D00017050020130505F5829717070020130720
:1041E00067F483470700930680029387E70793F7F6
:1041F000F70FE3ECF610BA898A0717D70100130707
:10420000E7D2BA979C43BA9782878D4797D501002A
:104210009385454417D50100130505C8630FF400C5
:1042200097B00100E780006717D50100130545012D
:1042300097B00100E7800066BDA497B00100E78059
:10424000606517D501001305250197B00100E780CF
:104250006064294597B00100E780A068930720F8C3
:104260001146970500209385E5EB4A851707002046
:10427000230AF7EA97070020A38707EA97000000C0
:10428000E780A0BA2A841DC997D501009385853C93
:1042900017D50100130545C097B00100E780805F86
:1042A000A28517D501001305E5FE97B00100E78050
:1042B000605E294597B00100E780A06297D50100B4
:1042C0009385453917D50100130505BD97B0010049
:1042D000E780405C17D50100130505FD97B001008C
:1042E000E780405B294597B00100E780805F41652A
:1042F000930730FA0546970500209385A5E27D15C2
:10430000170700202300F7E297000000E780E0B1E4
:104310002A841DC997D501009385C53317D501009F
:10432000130585B797B00100E780C056A28517D561
:104330000100130525F697B00100E780A055294537
:1043400097B00100E780E059B7E70400BC4F05666D
:10435000130606C8A14517F5FF1F0345A550829710
:10436000FE506E54DE544E59BE5911618280914701
:104370006303F40297D501009385C52D17D501007D
:10438000130585B197B00100E780C05017D5010033
:104390001305C5F471BDB7E70400FC4F914517F54F
:1043A000FF1F0345254C829797D501009385852AE9
:1043B00017D50100130545AE97B00100E780804D89
:1043C00017D50100130545F397B00100E780804C35
:1043D000294597B00100E780C05097500000E78062
:1043E000E079914535A485476303F40297D5010030
:1043F0009385452617D50100130505AA97B001003E
:10440000E780404917D50100130585F015B59707DA
:104410000020239127C9B7E704000566BC4F1306A7
:1044200006C8C1450DBF8D476303F40297D501004F
:104430009385452217D50100130505A697B0010005
:10444000E780404517D50100130545EED5B3930726
:1044500040F81146970500209385C5CC4A8517077B
:1044600000202301F7CC97070020A38E07CA9700EE
:104470000000E780809B2A84E30405EE97D50100C5
:104480009385451D17D50100130505A197B00100BF
:10449000E7804040A28517D501001305A5DF97B03E
:1044A0000100E780203F294597B00100E780604385
:1044B00045BD9147E31CF4F6B7E70400FC4F9305B4
:1044C000000217F5FF1F0345E539829797D50100D4
:1044D0009385451817D501001305059C97B0010079
:1044E000E780403B17D501001305C5E5F1BD8947BD
:1044F00063E3870297D501009385C51517D50100A1
:104500001305859997B00100E780C03817D50100E1
:10451000130585E431BB9704002083C4C4C097070A
:10452000002083C737C097D501009385A512A20448
:1045300017D5010013054596DD8C97B00100E78083
:104540006035A28517D50100130545E297B001003B
:10455000E7804034C204294597B00100E780603805
:10456000C1849305D4FF93960401C1824A8693F5D2
:10457000F50F17050020130515BB97400000E780D5
:1045800080A4E35F90DC930750F817070020230B0B
:10459000F7B883C73900228697050020938585B830
:1045A00085074A8517070020A30FF7B6970000007C
:1045B000E780A0872A84E30505DA97D50100938573
:1045C000650917D501001305258D97B00100E78017
:1045D000602CA28517D5010013050534C9B589479C
:1045E00063E3870297D501009385C50617D50100BF
:1045F0001305858A97B00100E780C02917D501000F
:10460000130585D835B197500000E7802057A28563
:1046100017050020130505B197600000E7804000F2
:1046200081B38D476303F40297D50100938585021A
:1046300017D501001305458697B00100E780802556
:1046400017D50100130505D6E5B6B7660200014689
:10465000B7750200054597E0FF1FE78080189307B4
:1046600060F817070020230FF7AA97070020A38CF4
:1046700007AA93070006170700202307F7AA894710
:1046800017070020A302F7AA97070020238F07A887
:1046900097070020A38B07A8C1471707002023070F
:1046A000F7A8930720F917070020A301F7A83146C0
:1046B00097070020A38DA7A697050020938585A6C0
:1046C0004A8597070020238407A697F0FFFFE7801D
:1046D000C0752A84E30605C897D50100938585F740
:1046E00017C501001305457B97B00100E780801ACC
:1046F000A28517D50100130565CC55B3B1476303F7
:10470000F40297D501009385E5F417C50100130560
:10471000A57897B00100E780E01717D501001305D1
:10472000A5CB39B6B7E70400FC4F9305000417F595
:10473000FF1F03452513829797500000E780004430
:10474000B145F9B5914763E3870297D50100938599
:1047500065F017C501001305257497B00100E780C7
:10476000601317D501001305E5C8D9B497040020DC
:1047700083C4849B9707002083C7F79AA204DD8C2B
:104780008E04B77702006D14BE942286A68517D5D5
:104790000100130565C797B00100E780A00FB7E7D8
:1047A0000400FC472286970500209385F597280092
:1047B000829793160401C1823000A685094597E0CF
:1047C000FF1FE78000022A8409C917D501001305DD
:1047D00065C597B00100E780C023930770F81946BC
:1047E00097050020938505944A8517070020230B21
:1047F000F79297070020A389879297F0FFFFE78041
:10480000C0622A84E30E05B497D50100938585E440
:1048100017C501001305456897B00100E7808007C0
:10482000A28517D501001305E5C095B99947630B1B
:10483000F41297D501009385E5E117C50100130532
:10484000A56597B00100E780E00417D501001305C6
:10485000E5BFF9BA914763E3870297D501009385D5
:1048600065DF17C501001305256397B00100E780D8
:10487000600217D501001305E5BE5DBA970400205C
:1048800083C4848A9707002083C7F789A204DD8C3C
:104890008E04B77702006D14BE942286A68517D5C4
:1048A0000100130565BD97B00100E780A0FEB7E7E2
:1048B0000400FC472286970500209385F586280092
:1048C000829793160401C1823000A6850D4597E0BA
:1048D000FF1FE78000F12A8409C917D501001305DD
:1048E00065BB97B00100E780C012930780F81946B6
:1048F00097050020938505834A8517070020230329
:10490000F78297070020A381878297F0FFFFE78057
:10491000C0512A84E30605A497D50100938585D369
:1049200017C501001305455797B00100E78080F6D1
:10493000A28517D50100130525B795B699476303DE
:10494000F40297D501009385E5D017C50100130542
:10495000A55497B00100E780E0F317D501001305D7
:1049600025B6F9B0B7E70400FC4F9305000417F52E
:10497000FF1F034525EF829797500000E780002036
:10498000994579B18D476303F40297D5010093856A
:1049900065CC17C501001305255097B00100E780CD
:1049A00060EF17D50100130525B359B017D50100E5
:1049B000130585B397B00100E780A0051305C01269
:1049C00097E0FF1FE780E097014597E0FFFFE78052
:1049D000A06C0D4597100000E7800048294597E03E
:1049E000FF1FE780009697E0FF1FE78060868DBA83
:1049F00099476303F40297D501009385A5C517C5B0
:104A000001001305654997B00100E780A0E817D5BC
:104A10000100130525AE29B817F7FF1F0347D7700C
:104A200097F7FF1F83C7477022075D8F9166BA967D
:104A3000C2061166C1821306F6EF8D476365D60282
:104A400097F7FF1F938747979C4B17F6FF1F034667
:104A5000966D9386C7002DC203D6070069CA8907E1
:104A6000E39CD7FE89471307A0F8114697F5FF1F6F
:104A70009385456B4A8597F6FF1F2385E66A17F7EE
:104A8000FF1FA302F76A97F0FFFFE780003A2A842E
:104A9000E308058C97D501009385C5BB17C50100B8
:104AA0001305853F97B00100E780C0DEA28517D5CA
:104AB0000100130565A5E5B203D60700630EE60AFB
:104AC0008907E39BF6FE8D4779BF91476304F402A3
:104AD00097D50100938505B817C501001305C53B9F
:104AE00097B00100E78000DB17D50100130545A34F
:104AF0006FF00FF4B7E70400FC4F9305000817F5BB
:104B0000FF1F034525D68297C9B897D50100938525
:104B100065B417C501001305253897B00100E7807B
:104B200060D717D50100130525A16FF06FF0239012
:104B3000E70017F5FF1F1305258897400100E78060
:104B4000E00197D501009385E5B017C50100130575
:104B5000A53497B00100E780E0D317D50100130515
:104B6000A59E97B00100E780E0D2294597B00100EB
:104B7000E78020D78147C5BD2390070017F5FF1FA9
:104B80001305858397400100E78040FD97D501001C
:104B9000938545AC17C501001305053097B001009A
:104BA000E78040CF17D501001305859B5DBF01113C
:104BB00022CC06CE26CA4AC8834705002A849DC750
:104BC00097D501009385C5A417C501001305C52C11
:104BD00097B00100E78000CC4C4017D501001305C9
:104BE000A5DA97B00100E780E0CA21A25841B707D3
:104BF000CF009387777D631DF70A0359C50085476A
:104C000004450356E50063FA270903C7040083C57A
:104C10001400F17693178700CD8FC207C187938662
:104C2000C6556393D70297300000E780C0F5630450
:104C300005106244F240CA8526854249D244056186
:104C4000173300006700C3F4954763F827059307FF
:104C500030056314F704930750046390F50483C68A
:104C6000240093071004639AF60283C73400639606
:104C7000E70203C744009307B0046310F70203C7B9
:104C8000540093079005631AF700CA85268532C63B
:104C900097300000E780C0EF32466244F240CA8598
:104CA00026854249D244056117F3FFFF6700E350B0
:104CB000B707CC009387777D6317F70497D501007A
:104CC0009385059517C501001305051D97B00100D3
:104CD000E78040BC1C448356E4008355C40003C6EF
:104CE000070017D501001305A5CB97B00100E78099
:104CF00060BA6244F240D24442492945056117B383
:104D00000100670003BEB707CE009387777D630479
:104D1000F70297D501009385A58F17C501001305EC
:104D2000A51797B00100E780E0B64C4017D5010009
:104D3000130585BB7DB5F2406244D244424905610A
:104D40008280B7E70400FC4741112E8606C622C4C4
:104D500026C24AC02E842A89AA8517F5FF1F13058B
:104D6000653C829797D501009385859017C5010012
:104D70001305851297B00100E780C0B197F5FF1FBA
:104D800083C5453A17C501001305853697B0010064
:104D9000E78040B0294597B00100E78080B497F4E0
:104DA000FF1F9384243883C7040041479387070675
:104DB00093F7F70F6369F75A17C7010013074721E5
:104DC0008A07BA979C43BA9782879D476307F40284
:104DD00097D501009385C58917C501001305C50B3B
:104DE00097B00100E78000AB17C501001305C5307F
:104DF00097B00100E78000AAA1AC97F7FF1F83C717
:104E00007732DDCB17F7FF1F0347F73197F7FF1F07
:104E100083C7673122075D8F97F7FF1F83C7C730AE
:104E2000C2075D8F97F7FF1F83C71730E207D98F3F
:104E300017F7FF1F232EF72C83C7640097D50100B7
:104E40009385058317C501001305050517F7FF1F97
:104E5000230FF72A97B00100E780C0A397F7FF1F41
:104E60009387072B8C4317F6FF1F0346462A17C567
:104E700001001305252A97B00100E780A0A129456C
:104E800097B00100E780E0A597F7FF1FA38C0728E4
:104E90002244B24092440249930700F817F7FF1FDB
:104EA0002302F7289D4517F5FF1F1305A52741018C
:104EB000175300006700C37697700000E7808046B4
:104EC00097F7FF1F2381A7269357850017F7FF1F2A
:104ED000A30BF724935705012A8417F7FF1F230517
:104EE000F72493578501014517F7FF1FA30EF722FB
:104EF00097700000E780604797F7FF1F2387A7227E
:104F000097C501009385C57617C501001305C5F83F
:104F100097B00100E780009817F6FF1F0346E620D0
:104F2000A28517C5010013056520B1B7CD476303FE
:104F3000F40297C501009385A57317C501001305F9
:104F4000A5F597B00100E780E09417C501001305AF
:104F5000651F79BD97F7FF1F83C7E71DA20717F7E6
:104F6000FF1F0347371DD98FC207C1876357F00260
:104F700017F7FF1F231CF718B7E7040003A38705E3
:104F80001306000A89452244B2409244024917F5AB
:104F9000FF1F0345258D41010283D147D1BF8D47B6
:104FA0006303F40297C501009385856C17C5010062
:104FB000130585EE97B00100E780C08D17C501008D
:104FC0001305052835B517F4FF1F0344C41597F7DB
:104FD000FF1F83C7371597C50100938565692204B4
:104FE00017C50100130545EB5D8C97B00100E78004
:104FF000608AA28517C501001305451697B0010008
:10500000E7804089294597B00100E780808D0D46F3
:1050100097F5FF1F93850511228597F0FFFFE78025
:10502000C0E0AA8421C197C501009385656417C5B6
:105030000100130565E697B00100E780A085A6850D
:1050400017C501001305C51297B00100E7808084E1
:105050002244B240924402492945410117B301005C
:105060006700238897F7FF1F23968702B7E704009E
:10507000116603A38705130606E8914529B78D47F6
:105080006303F40297C501009385855E17C501008F
:10509000130585E097A00100E780C07F17C50100D8
:1050A0001305C528B1B317F4FF1F0344C40797F7CE
:1050B000FF1F83C7370797C501009385655B2204EF
:1050C00017C50100130545DD5D8C97A00100E78041
:1050D000607CA28517C501001305C50A97A00100D1
:1050E000E780407B294597A00100E780807F0D463F
:1050F00097F5FF1F93850503228597F0FFFFE78053
:10510000C0D2AA841DC197C501009385655617C5F5
:105110000100130565D897A00100E780A077A68558
:1051200017C501001305450705B797F7FF1F23951E
:1051300087F4B7E70400116603A38705130606E8A2
:105140009305000289B5894763E3870297C501008B
:105150009385055217C50100130505D497A00100DA
:10516000E780407317C501001305051F51B197F47F
:10517000FF1F83C444FB97F7FF1F83C7B7FA97C588
:1051800001009385E54EA20417C501001305C5D0A3
:10519000DD8C97A00100E780E06FA68517C50100B0
:1051A0001305050197A00100E780C06E294597A06F
:1051B0000100E7800073228697F5FF1F938585F62F
:1051C000268597F0FFFFE78040C62A84630E051A04
:1051D00097C501009385C54917C501001305C5CBC7
:1051E00097A00100E780006BA28517C50100130599
:1051F00065FD99BD854763F98718834519002244E9
:10520000B24092440249B335B00097F7FF1F238D97
:10521000B7E817C50100130525FC410117A30100DC
:1052200067004367A2852244B24092444A850249FE
:10523000410117130000670063C899476303F40234
:1052400097C501009385C54217C501001305C5C464
:1052500097A00100E780006417C5010013058529A8
:1052600041BE17F4FF1F034404EC97F7FF1F83C7E9
:1052700077EB97C501009385A53F220417C5010070
:10528000130585C15D8C97A00100E780A060A28511
:1052900017C501001305C5F597A00100E780805FE1
:1052A000294597A00100E780C063194697F5FF1FC5
:1052B000938545E7228597F0FFFFE78000B7AA8432
:1052C0001DC197C501009385A53A17C501001305B7
:1052D000A5BC97A00100E780E05BA68517C501008B
:1052E000130505F295B397F7FF1F239587E2B7E7FC
:1052F0000400116603A38705130606E8930500085A
:1053000059B1854797C501009385853617C50100BA
:10531000130585B8630BF40097A00100E780805760
:1053200017C50100130505EFE1B497A00100E78060
:10533000605617C50100130565EF97A00100E780CF
:105340006055294597A00100E780A0592244B2404A
:105350009244024997F7FF1F239A07DA4101177316
:1053600000006700A3EC97C501009385653017C561
:105370000100130565B297A00100E780A05117C591
:1053800001001305651BADB4B240224492440249AA
:1053900041018280411106C622C426C239C12A8435
:1053A00097F00000E7804075AA8411EDB7E704008C
:1053B000BC474146814522858297B24022442685DA
:1053C00092444101828041657D1597F00000E7809D
:1053D0008073B7E7040001E9BC4741468145228557
:1053E00082978144D9BF0347E501FC4793059008A4
:1053F00019E393050003AA954146228582978544C7
:105400006DBF411106C622C426C24AC097F00000F3
:10541000E780806E55CD97700000E78060F12A84A8
:1054200097100000E7800058AA84228563739400D7
:105430002685B7D7B0009387F75E63F3A702B7E777
:10544000B000130514009387F74F63E3A7082244C5
:10545000B24092440249410117730000670003EE15
:105460008567938707F13E956364A4003305F400D4
:1054700097700000E78080EC97700000E78040EBB9
:105480002A8963F6A40097100000E780605497C54E
:1054900001009385651F17C501001305E59F97A0BF
:1054A0000100E780203FA6864A86A28517C5010035
:1054B000130545B697A00100E780C03D2244B240E5
:1054C000924402492945410117A301006700634145
:1054D000B24022449244024941018280011122CC0F
:1054E00037E404005C5C06CE26CA354697C5010049
:1054F0009385C52217D501001305050E829711E982
:1055000017C501001305059F97A00100E7806050B3
:1055100001A097E7FF1F9387A7353EC4B7F50700A3
:10552000856793870780814617E6FF1F1306C633FA
:10553000E10519453EC697D0FF1FE780802A7C44CD
:10554000194697E5FF1F9385253217F5FF1F1305B1
:10555000A5B48297340017E6FF1F1306E63097C5FF
:1055600001009385656717C501001305656897708D
:105570000000E780C090AA8421C197C501009385EF
:10558000250B17C501001305259197A00100E780A1
:105590006030A68517C501001305451997A00100C5
:1055A000E780402F294597A00100E7808033F24033
:1055B0006244D2440561828097E00000E78080FA6F
:1055C00017C501001305850D97600000E780E08492
:1055D00097A00000E780C04E97600100E78040B3CD
:1055E00017E5FF1F1305C5D997600100E780E09B11
:1055F00017C501001305850B97600100E780C0B354
:10560000AA8497600000E78020EB97100100E780F4
:10561000208B97800100E780402497700000E7808E
:10562000E04A97600000E780206197300100E78042
:10563000804C97C501009385A5FF17C50100130590
:10564000A58599C897A00100E780C024A68517C545
:1056500001001305E50F99B797A00100E7808023AB
:1056600017C501001305051197A00100E7808022EE
:10567000294597A00100E780C02697300100E78008
:10568000602897F00000E7802047630A051297E73B
:10569000FF1F83D7E7C1170700202314F7085147DE
:1056A0006381E70897C50100938585F817B5010068
:1056B0001305857E97A00100E780C01D5146970520
:1056C000002083D5050617C501001305250C97A0FA
:1056D0000100E780201C294597A00100E780602099
:1056E00097070020238C07F297070020239B0702CF
:1056F00097700000E78080B397C50100938545F35C
:1057000017B501001305457997A00100E7808018BF
:1057100017C501001305C50F97A00100E78080178A
:1057200051B585453705040097300000E780E085D6
:1057300097C501009385C5EF17B501001305C57521
:1057400097A00100E780001517C501001305450764
:1057500097A00100E7800014294597A00100E78089
:105760004018854717070020230AF7EA97E7FF1F2D
:10577000938787C4DC4703D70700C167FD1763160B
:10578000F70097E0FFFFE780E07A97000000E780EE
:1057900080C797100000E78000F51705002003552B
:1057A00045F897500000E78020BD05459750000060
:1057B000E78000F097500000E780801535BFD147A3
:1057C00097C501009385C5E617B501001305C56CA3
:1057D00017F7FF1F231CF79297A00100E780800BAB
:1057E00017C601001306065B97F5FF1F83D50592C8
:1057F00017C50100130505FF97A00100E780800988
:10580000294597A00100E780C00D3C4C1306000A13
:10581000894517E5FF1F0345E50482970145975029
:105820000000E780E0E8C9BD411122C437E404006C
:105830008327041A06C6829797500000E78080B736
:10584000832704081705000013050503829797E7CF
:10585000FF1F2389A70017E5FF1F1305E5B5974034
:105860000000E78060682244B24041011703000055
:10587000670003C7011122CC06CE26CA4AC84EC60D
:1058800093F715002E84B5CB97E0FFFFE780806A81
:10589000930710F817F7FF1F2306F78897E7FF1FF6
:1058A00083D7077D17F7FF1FA30EF7869145A183C6
:1058B00017F5FF1F1305058717F7FF1F2305F78649
:1058C00097F7FF1FA381078697500000E78040D518
:1058D000B7E70400BC4F130600149305001017E54A
:1058E000FF1F034525F8829713451400F2406244D8
:1058F000D2444249B2490561828093F70510B1C78D
:10590000054597500000E780A0DA170500200355F1
:1059100045E197500000E78020A697000000E7804F
:1059200080AE97100000E78000DC97F7FF1F83C769
:10593000B78E89E797500000E780C0FB97500000C2
:10594000E78000FD1345041055B793F72500E9CF14
:1059500017E7FF1F0357877B69C7AD64B71900407E
:105960009384A4AA23A0990097E6FF1F9386467A02
:10597000944297C70100938727FF17E6FF1F03464E
:105980000679814517C50100130505FF97600000E2
:10599000E780E07923A0990097E7FF1F2392A79261
:1059A0002A8941C197C50100938585C917B50100B2
:1059B0001305854E97A00100E780C0EDCA8517B595
:1059C00001001305E56797A00100E780A0EC2945D9
:1059D00097A00100E780E0F097E7FF1F2398077288
:1059E000930710F817E7FF1F230EF77297E7FF1FC3
:1059F00083D7076817E7FF1FA306F772A18317E78E
:105A0000FF1F2302F77291458D4717E5FF1F13050E
:105A1000657117E7FF1FA308F77097500000E78034
:105A200020C013452400D9B593F74500D1C397C5CD
:105A300001009385E5C017B501001305E54597A062
:105A40000100E78020E517B501001305256197A047
:105A50000100E78020E4294597A00100E78060E885
:105A6000930720F817E7FF1F230EF76A97E7FF1F3A
:105A700083D7476217E7FF1FA306F76AA18317E7DB
:105A8000FF1F2302F76A854717E7FF1FA30DF7687B
:105A900097400000E780800E17E5FF1F130585681B
:105AA000914597500000E780A0B7134544003DBDE5
:105AB00093F78500A9C797C50100938565B817B509
:105AC00001001305653D97A00100E780A0DC17B534
:105AD00001001305E55997A00100E780A0DB2945E7
:105AE00097A00100E780E0DF97E7FF1F23900762A0
:105AF00097600000E780807313458400C5BB93F76F
:105B00000501D1C3854517E5FF1F0355A5589750DB
:105B10000100E780202D97C50100938565B217B578
:105B200001001305653797A00100E780A0D617B5DF
:105B300001001305255597A00100E780A0D5294550
:105B400097A00100E780E0D9930730F817E7FF1F1F
:105B5000230AF75C97E7FF1F83D7C75317E7FF1F99
:105B6000A302F75C17E5FF1F1305C55BA1838D45F5
:105B700017E7FF1F2309F75A97500000E78040AA54
:105B800013450401A5B393F70502D1C797C50100DA
:105B9000938505AB17B501001305053097A00100EB
:105BA000E78040CF17B501001305055097A001000D
:105BB000E78040CE294597A00100E78080D2930777
:105BC00040F817E7FF1F230FF75497E7FF1F83D70E
:105BD000A74A17E7FF1FA307F754A18317E7FF1F83
:105BE0002303F754854717E7FF1FA30EF75297E7E4
:105BF000FF1F2393074897400000E78020F817E530
:105C0000FF1F13052552914597500000E78040A1E2
:105C100013450402E1B993F70504FDC397C50100DC
:105C2000938505A217B501001305052797A001006C
:105C3000E78040C617B501001305854897A001000D
:105C4000E78040C5294597A00100E78080C997E714
:105C5000FF1F83C7274D1307700A6386E7061307E4
:105C6000800A638CE7081307600A6393E7049307CD
:105C700060F817E7FF1F2307F74A97E7FF1F83D74F
:105C8000C74817E7FF1FA30FF748A18317E7FF1FB8
:105C9000230BF748854717E7FF1FA30AF748B145CD
:105CA00017E5FF1F1305054897500000E780409750
:105CB00097400000E78080EC1345040497E7FF1F3E
:105CC0002395074425B1930770F817E7FF1F230BAF
:105CD000F74497E7FF1F83D7474317E7FF1FA30347
:105CE000F744A18317E7FF1F230FF742854717E704
:105CF000FF1FA30BF742994565B7930780F8F1B7EB
:105D000093F705080145E38307BE97C50100938516
:105D1000259317B501001305251897A00100E7800A
:105D200060B717B501001305253B97A00100E78078
:105D300060B6294597A00100E780A0BA9307A0F8B4
:105D400017E7FF1F2300F73E97E7FF1F83D7873C26
:105D500017E7FF1FA308F73CA18317E7FF1F2304E2
:105D6000F73C854717E7FF1FA30FF73A97E7FF1F99
:105D70002392073A97400000E78040E017E5FF1FB5
:105D80001305453A914597500000E7806089134517
:105D90000408A9BE1307F5FF75714207C16706C75E
:105DA00022C526C34AC14183F51763EFE700854545
:105DB00097500100E78000038544BA402A442685B5
:105DC0000A499A4449618280B7E70400BC47130638
:105DD000000881450A8582970A8597600000E78060
:105DE000C05A0A841309010881440355040009C9F3
:105DF0008545850497500100E780C0FE93F4F40FB9
:105E00002104E31489FE55BF411106C697E0FFFF48
:105E1000E78080FA0DC197E7FF1F83D70729850721
:105E200017E7FF1F2313F72897E7FF1F2390A728E3
:105E3000B2404101828097E7FF1F83D7472785073C
:105E400017E7FF1F2315F726E5B785461703000060
:105E50006700C3FB411122C491462A8417E6FF1F45
:105E60001306463A9D652D4506C697D0FF1FE7806D
:105E70004097B7F7070003C70701A5476313F7006B
:105E800001A09306001001469D65254597D0FF1F90
:105E9000E780209597E7FF1F238687362244B2408C
:105EA000914617E6FF1F1306E6359D65294541011A
:105EB00017D3FF1F6700E3921171CED7B7E9040033
:105EC00083A7C904CAD917E9FF1F1309A925A2DDB1
:105ED0002E8686DFA6DB2E84AA854A85829797E7E1
:105EE000FF1F83C727241307700A6385E710636DBC
:105EF000F7001307600A6385E704FE506E54DE5412
:105F00004E59BE59116182801307800A6385E716D6
:105F10001307900AE393E7FE8D476306F41C97C5C9
:105F20000100938565B317B501001305E5F697A049
:105F30000100E780209617C50100130525AF25A0B5
:105F40008D47630CF40297C501009385E5B017B542
:105F50000100130565F497A00100E780A09317C521
:105F600001001305E5A597A00100E780A09229454F
:105F700097A00100E780E09649B7854717C5010063
:105F80001305C5A517E7FF1F2300F71297A001000F
:105F9000E78020A8B7750200B766020001460545F4
:105FA00097D0FF1FE780E083930760F817E7FF1F94
:105FB000230AF71697E7FF1FA38707169307002604
:105FC00017E7FF1F2322F716E5779387072117E7C7
:105FD000FF1F231DF714B14597E7FF1F23890714FF
:105FE00097E7FF1FA385A7144A8597000000E78065
:105FF000E01621B7914763E3870297C501009385B7
:10600000A5A517B50100130525E997A00100E780B4
:10601000608817C501001305659EB1B797E4FF1F9F
:1060200083C4841097E7FF1F83C7F70FA204DD8C9A
:1060300083A7C9046D14228697E5FF1F9385D50EAB
:10604000280082978E0493160401B7750200C1825E
:106050003000A695094597C0FF1FE7808078930719
:1060600070F817E7FF1F230FF70A994597E7FF1FFF
:10607000A38CA70A95BF914763E3870297C50100E8
:106080009385859D17B50100130505E197A00100D3
:10609000E780408017C501001305C597E9B597E46F
:1060A000FF1F83C4640897E7FF1F83C7D707A204B5
:1060B000DD8C83A7C9046D14228697E5FF1F9385A5
:1060C000B506280082978E0493160401B775020066
:1060D000C1823000A6950D4597C0FF1FE780607014
:1060E000930780F8BDBF17C501001305659597A0FC
:1060F0000100E7800092930790F82304F1008347A2
:1061000019008D452800A304F100834729002305C9
:10611000F10097000000E78060041305C01297C0EB
:10612000FF1FE7800022014597D0FFFFE780C0F600
:106130000D4597000000E78020D2294597C0FF1F3A
:10614000E780202097C0FF1FE78080107DB397E78E
:10615000FF1F23A1A70C828097E7FF1F9387870B60
:1061600003A30700630303000283174300006700D3
:10617000234B41114AC097F6FF1F83D6865A3289B6
:1061800017D6FF1F0356662522C426C206C62A84D8
:10619000AE8497000000E780406C29C921C8994768
:1061A00063F697048347140003470400A207D98FBE
:1061B00013978700A183D98FC2073167C183130763
:1061C000C7556395E70297D7FF1F83D70721A30120
:1061D000F400A1832302F40097F7FF1F83D76754CD
:1061E00091C7A302F400A1832303F400630D090205
:1061F00097F7FF1F83C787429DE797E7FF1F83C776
:10620000A70195C38DC097E7FF1F83C7E7E981EF1B
:1062100022852244B2400249A68592444101174397
:1062200000006700E33FB24022449244024941012A
:1062300082801DCD95472A87014563FDB70297F7F8
:10624000FF1F83C7A73D9DC783475700834647006D
:10625000A207D58F85C341112E863E85BA8506C615
:1062600097000000E780A0BEB24005454101828052
:1062700001458280828097B70100938767B29C4373
:1062800001116800914506CE3EC697000000E780E8
:10629000E0ECF240056182808D4763F6B70801119A
:1062A00026CA06CE22CC0344350097E4FF1F83C4E0
:1062B000B4F697B501009385E57BB337800017E707
:1062C000FF1FA30BF7F409C497B501009385457B25
:1062D00017B501001305457B97900100E780805BAF
:1062E00097E7FF1F83C757F3638697009700000067
:1062F000E780C04697400000E780806199679387F8
:1063000057EE2316F100680085479145A3078100E9
:106310002307F10097000000E78040E4F240624468
:10632000D244056182808280894763F7B7080111F2
:1063300022CC06CE26CA8344250085472A84639D45
:10634000F404914763F5B7040345450083473400DF
:1063500022055D8D97D7FF1F2391A70897000000A6
:10636000E78080589967938767EE2314F10083478D
:10637000340023059100A305F100834744009545AF
:1063800028002306F10097000000E78020DDF2409E
:106390006244D24405618280FDF89967938767EE75
:1063A0002314F10097D7FF1F83D72703A305F1001C
:1063B00023050100A183E1B782800111996722CCF6
:1063C000D51717F4FF1F130464252314F100834726
:1063D000040026CA97F4FF1F9384A4342305F10018
:1063E00083D7040028009545A305F100A18306CEBC
:1063F0002306F10097000000E78040D603D6040092
:106400008345040017B50100130505699790010045
:10641000E7804048F2406244D244056182809D6733
:106420007971D9172316F10097F7FF1F9387071F7C
:1064300083C707001305F10006D62307F10097F084
:10644000FFFFE78060F509E9B7E70400BC47414674
:1064500081451305F10082976800CD459700000043
:10646000E780C0CF97F5FF1F83C5451B17B5010017
:106470001305856597900100E780C041B2504561E2
:106480008280630C0516011126CA06CE22CC4AC8AA
:106490004EC697E7FF1F83C737D897F4FF1F83C403
:1064A000E41799C393E424002A8497100000E7803E
:1064B000806D93E9C40119E193E9C40037E9040050
:1064C0008327890422851306200381458297930739
:1064D00050FA2300F4009307A005A300F4008D47B1
:1064E0002301F4009147A301F40093077005A30270
:1064F000F40097F7FF1F83D7C7222304F400A1837A
:10650000A304F40097D7FF1F83D727ED2305F400DA
:106510009304C400A1832302040023033401A305D0
:10652000F400268597F0FFFFE78000E719E5832751
:106530008904414681452685829797D7FF1F83D7D7
:1065400067E7230EF400A183A30EF4009307000273
:10655000230FF400930710FAA30FF4009D472300C4
:10656000F402A3000402B7E70400FC471305240269
:10657000194697D5FF1F9385252F829797E7FF1F11
:1065800083D7E7B22304F402A183A304F40297E7BC
:10659000FF1F83D787B12305F402A183A305F4026B
:1065A00097E7FF1F938787B083970700228593059E
:1065B00000032306F402C207C183A183A306F402E9
:1065C00097D7FF1F9387C7CF839707002307F4024E
:1065D000C207C183A183A307F40297000000E780EC
:1065E000C0232308A4022181A308A402F24062442C
:1065F000D2444249B2490561828082805D71E1776F
:1066000093C777FF1305E10086C62316F1009700B4
:106610000000E78040E76800930540039700000012
:10662000E780C0B3B640616182805DC9411122C478
:1066300026C206C6930750FA2300F5009307A0056B
:10664000A300F50089472301F5009147A301F50058
:1066500093077005A302F50097F7FF1F938707FCC8
:1066600083C707009304C5002A842303F50097E736
:10667000FF1F938777BA83C7070023020500A30390
:10668000F50097F7FF1F83D7C7092304F500A183FF
:10669000A304F50097D7FF1F83D727D42305F50060
:1066A000A183A305F500268597F0FFFFE780C0CE04
:1066B00001E9B7E70400BC4741468145268582973A
:1066C0002285F14597000000E7802015230EA400E5
:1066D0002181A30EA400B240224492444101828051
:1066E00082805D710A8586C6A2C497000000E7809B
:1066F00000F437E404007C448A85081079468297C8
:106700003C441305E1030946814582971010930527
:106710000002014597D0FFFFE78040FEB6402644C7
:1067200061618280411122C426C22A84AE848566BA
:10673000AA850146254506C697C0FF1FE780600A67
:10674000A2852244B24026869244A14629454101B1
:1067500017C3FF1F6700E3080111B7C7A55A22CC72
:106760009387C73317E4FF1F130414AB3EC483475A
:1067700004002C00196506CE3EC697000000E78095
:10678000A0FA8345040017B501001305653E9790F4
:106790000100E7802010F24062440561828001110F
:1067A000A146300099652D4522CC06CE97C0FF1F2B
:1067B000E7802003A24737C4A55A1304C433639566
:1067C0008702B24517B5010013054532B335B00055
:1067D00097E7FF1FA382B7A497900100E780800B83
:1067E000F2406244056182809165A1463000938544
:1067F00005F02D4597C0FF1FE780A0FEA247E3826A
:1068000087FC97E7FF1FA38907A0814517B5010003
:1068100013050530D1B7C16769768146FD170506B6
:106820001397060141836364B7003E858280330776
:10683000D50003470700B98F214713F81700858358
:1068400063050800B18FC207C1837D171377F70F67
:106850006DF78506F1B741C5A547054763F2B7084F
:1068600083471500034705003168A207D98F1397A6
:106870008700A183D98FC207C1831308C855054774
:1068800063900707411106C622C426C203442500AF
:10689000914763F087049307540063ECF502A3016A
:1068A000C50021822302C5009304340091C6A302CF
:1068B000D500A1822303D5002A84A6859700000075
:1068C000E780A0F526942300A4002181A300A40062
:1068D0000147B240224492443A85410182800547F3
:1068E0003A8582800111B7C7A55A22CC9387E73435
:1068F0002A842AC62C00156506CE3EC497000000E7
:10690000E78080E2A28517B50100130565289790FE
:106910000100E78020F897000000E780C0DCF2402B
:106920006244056182800111A146300095652D45C4
:1069300022CC06CE97C0FF1FE780A0EAA24737C44B
:10694000A55A1304E43463958702B24517B50100D4
:106950001305051E97D7FF1F2391B7A8C205C18154
:1069600097900100E78000F3F24062440561828065
:106970009165A1463000938505EE2D4597C0FF1F18
:10698000E78020E6A247E38287FCD14717D7FF1FA5
:106990002315F7A4D14517B501001305651BC9B729
:1069A0000111A146300091652D4506CE97C0FF1F0D
:1069B000E78020E32247B7C7A55A938707350145EB
:1069C0006313F7003245F240056182800111B7C7B9
:1069D000A55A2AC6938707352C00116506CE3EC4FA
:1069E00097000000E78040D4F2400561828021C119
:1069F000411126C206C622C4AE848DC52A849710D2
:106A00000000E780E01897E7FF1F83C7E78099CB76
:106A100022852244B240A6859244410117430000DA
:106A2000670003C0B24022449244410182808280C8
:106A300001114EC606CE22CC26CA4AC893F71500CD
:106A4000AE899DCBAD67371700409387A7AA1CC3BB
:106A5000B7E70400BC4F13060019854517D5FF1F83
:106A600003458597829713C51900F2406244D244CA
:106A70004249B2490561828093F725000145F5D767
:106A800017F7FF1F0357C7C9954763F9E70C014480
:106A900017F6FF1F1306C6B89306300513055004FA
:106AA000130810049308B0041303900593076400BF
:106AB0006374F7043A847D5997F4FF1F83C444B686
:106AC00097F7FF1F83C7D7B5A204DD8CAD67938707
:106AD000B755638BF41463E3970AA9679387A755A7
:106AE000638EF414A28517F5FF1F130565B3970095
:106AF0000000E78000F0E9A0B307860083C5070027
:106B0000639AD50483C517006396A50483C527003F
:106B10006392050583C53700639ED50283C5470090
:106B2000639A150383C757006396670222890DE8AD
:106B300097F5FF1F83D5C5BEB3852541C20517F55F
:106B4000FF1F1305E5ADC1814A9597000000E7805E
:106B500040EAE1A005044204418089BF3A847D599E
:106B60008547E3EB87F45DC4854517F5FF1F1305E3
:106B700025AB97000000E780C0E769A8B16793875D
:106B8000C7556389F404B5679387D755E39CF4F43C
:106B9000A28517F5FF1F1305A5A897400000E78001
:106BA00020A88947630EF4009305E4FFC205C18164
:106BB00017F5FF1F1305E5A697100000E78040FDBD
:106BC000A68517B50100130565FE97900100E780C3
:106BD00060CC89A097300000E780E0999710000012
:106BE000E78060FA11C9A28517F5FF1F130545A3B9
:106BF00097100000E780C0F90546A28517F5FF1F32
:106C0000130505A297F0FFFFE780E05697300000DC
:106C1000E7806096FD57E31DF9F097F7FF1F23917A
:106C200007B013C5290091B5A28517F5FF1F1305FD
:106C3000259F97F0FFFFE780006059B7A28517F501
:106C4000FF1F1305E59D97F0FFFFE78000638DBFF1
:106C5000411122C437E404005C5C06C6354697B592
:106C600001009385A5AB17C501001305E596829732
:106C700011E917B501001305A5F497900100E7800D
:106C800040D901A08327041C82972A84054597D008
:106C90000000E780808C97700100E780A01197705A
:106CA0000100E780A0E697C00000E780009E2285F3
:106CB000B2402244410182804111054506C622C4EA
:106CC00026C297C0FFFFE78000271305A00497B0F6
:106CD000FF1FE780C03D757585457D1597C0FFFF97
:106CE000E780A0107D7585451305F53697C0FFFF39
:106CF000E780001A371400408327840A8D45130566
:106D0000002093E707202324F40A97C0FFFFE780C1
:106D1000C00DB7E4040097C0FFFFE780E052C858F9
:106D200097900100E780E0CE17C501001305C58AE2
:106D300097900100E780E0CD8327840C854541458D
:106D400093E707082324F40C97C0FFFFE780401463
:106D50008D451305000897C0FFFFE780601397C0BB
:106D6000FFFFE780404037A507001305051297C0D5
:106D7000FFFFE780E03B014597C0FFFFE78000424F
:106D800095450545894717F7FF1F230DF79897C0CD
:106D9000FFFFE7804042B7E700E013070006238DBE
:106DA000E7403707000423A0E71097D0FFFFE780F4
:106DB000C0C397D0FFFFE780C0D597000000E780F1
:106DC00060E997000000E780C09D97000000E78021
:106DD000C0B597F0FFFFE78060A597100000E7803F
:106DE00060DC97000000E780801083A70408170587
:106DF0000000130525C4829797C7FF1F238EA75C49
:106E0000BC4C130600648545829797B0FF1FE7804E
:106E1000205E01458280AD67371700409387A7AA9F
:106E20001CC3B7E700E03707400023A0E7180100C4
:106E30000100B7F7070003C70701A5476316F7006E
:106E40009397450191C301A04111AE860146AA85E1
:106E5000254506C697C0FF1FE780A098B240B7E758
:106E600000E03707400023A0E71041018280411174
:106E7000B2862E86AA852D4506C697C0FF1FE780DD
:106E80004096B2400145410182809307000463ECC3
:106E9000C7041D71A2CC2A840808A6CACAC886CE17
:106EA00032C697900100E7808093AD6737170040A6
:106EB0009387A7AA1CC3B7E400E03709400023A0CA
:106EC000241901000100B2461008A285294597C087
:106ED000FF1FE7800091F640664423A02411D644AA
:106EE0004649256182803955828041110D658D4565
:106EF00006C697C0FFFFE78040EFB71700408D66DA
:106F000023A6D70A17F5FF1F130505821387C70AA3
:106F10009387870A1CC15CC5856689675CC958C1AF
:106F200014C518C9B7E70400B24003A3871E410186
:106F300002830387060009E763E0C5022E8582808D
:106F400093871500C207C183E3F8C7FEAA95238083
:106F5000E5008506BE85F1BF2E9523000500F9BF2B
:106F600001111C08BA9706CE238A07FE5C003E97E3
:106F700097B801009388080213F8F6004698034872
:106F800008007D17918223000701E397E7FEBE8684
:106F900097000000E78020FAF24005618280814678
:106FA000E548B307D50003C70700B387D50083C7FB
:106FB0000700A1C31308F7F91378F80F63E5080178
:106FC00001171377F70F1388F7F91378F80F63E5B4
:106FD0000801811793F7F70F631FF7008506939752
:106FE0000601C183E3EFC7FAB2958387050093B723
:106FF00017003E8582808147EDBF8547814663F15A
:10700000B7020347050093070003631BF70083479C
:1070100015001307800593F7F70D6393E700894682
:1070200001470148254E1543914E89A0B307D5006D
:1070300083C70700938807FD93F8F80F637C1E0150
:107040009388F7FB93F8F80F63681303938797FC13
:1070500093F8F70F120833681801050742081377F1
:10706000F70F135808018506630FD70193970601A0
:10707000C183E3EDB7FA39A09388F7F993F8F80FD5
:107080006378130101C72310060105473A85828002
:10709000938797FA75BF8145B307B50083870700CB
:1070A00089E7172300006700A3538505C205C18146
:1070B000E5B7411106C6B94763EEB70017B5010041
:1070C000130505BA97000000E78020FDB240054592
:1070D000410182808347E500130710036394E702B0
:1070E000854717E7FF1F230BF77817B50100130536
:1070F00065B997E7FF1F2392077897E7FF1F23994A
:107100000768C9B713070003E39AE7FA97E7FF1F79
:107110002386077697E7FF1F2391077697E7FF1FE0
:107120002398076617B50100130545B761BF4111E4
:1071300026C2E97797E4FF1F9384847422C493875F
:10714000A7552E842381B4002E86AA8517E5FF1F3C
:107150001305457306C62390F400A38104009780AD
:107160000100E780C06793052400C205C18117E5CF
:10717000FF1F1305057197F0FFFFE780006AB387D3
:1071800084002382A7002181A382A70093056400C5
:107190002244B24026859244C205C1814101172391
:1071A00000006700E34309C99307000463E6B700E2
:1071B000170300006700E3F78280011106CE230762
:1071C000010081EE97B60100938686DC97000000EF
:1071D000E78060D6F2400561828058002A88AE8838
:1071E0003283A9473A85A945254E33F6B602FD17E5
:1071F00093F7F70F13060603A304C70033D6B602AE
:107200006375DE007D17B286EDF3B306F5001A86CE
:10721000C685428565BF397197B60100938606D051
:107220001306001006DE22DC26DA2A844AD84ED65F
:1072300097000000E78020D0AA8597E6FF1F83D63D
:10724000464E114713060010228597000000E78084
:1072500060D197E7FF1F83C7673CAA8597B60100F7
:10726000938646C989C797B60100938626C8130638
:107270000010228597000000E780E0CBAA8597B632
:1072800001009386E6C913060010228597000000CE
:10729000E78060CAAA8597B601009386E6C8130600
:1072A0000010228597000000E780E0C8AA8591467B
:1072B00013060010228597000000E78040F0AA85A1
:1072C00097B6010093864625130600102285970085
:1072D0000000E78040C6AA8597B60100938646CB9A
:1072E00013060010228597000000E780C0C4AA851D
:1072F00097B6010093864622130600102285970058
:107300000000E78040C3AA859306700513060010AD
:10731000228597000000E78080EA97D7FF1F83C788
:10732000B7EFAA8597B60100938646BD89E797B661
:107330000100938626BD13060010228597000000E9
:10734000E78060BFAA8597B60100938666BE1306E4
:107350000010228597000000E780E0BDB7A6070077
:10736000AA85938606121306001022859700000056
:10737000E780E0E4AA8597B601009386E6BB130692
:107380000010228597000000E780E0BA97C7FF1F32
:1073900083C7C704AA8597B60100938626B789E7F5
:1073A00097B60100938606B7130600102285970052
:1073B0000000E78040B8AA8597B60100938686B89A
:1073C00013060010228597000000E780C0B6AA854A
:1073D00097B60100938686B71306001022859700A2
:1073E0000000E78040B5AA8597B60100938686B66F
:1073F00013060010228597000000E780C0B31147F4
:10740000AA8597C6FF1F83D6E6FA130600102285C9
:1074100097000000E78000B52AC697500000E7807B
:1074200020F1B245AA8497B601009386E6B213060E
:107430000010228597000000E780E0AF93D604019A
:10744000AA85094793F6F60F1306001022859700C8
:107450000000E78020B1939604011147AA85C182FC
:1074600013060010228597000000E780A0AFAA85D0
:1074700097B601009386C6AE1306001022859700CA
:107480000000E78040AB1147AA8597C6FF1F83D64F
:10749000C6F413060010228597000000E78080AC38
:1074A000AA8597B60100938626AC130600102285A4
:1074B00097000000E78020A81147AA8597D6FF1FF4
:1074C00083D6E6BE13060010228597000000E780F1
:1074D00060A9AA8597B60100938686A913060010B5
:1074E000228597000000E78000A51147AA8597D65E
:1074F000FF1F83D686BB130600102285970000006D
:10750000E78040A6AA8597B601009386E6A61306F3
:107510000010228597000000E780E0A11147AA85AE
:1075200097D6FF1F83D686B81306001022859700D2
:107530000000E78020A3AA8597B60100938606A4E1
:1075400013060010228597000000E780C09EAA85E0
:10755000114797C6FF1F83D6A6D6130600102285B3
:1075600097000000E78000A0AA8597B601009386E7
:1075700066A113060010228597000000E780A09BFB
:10758000AA85814497C9FF1F9389092E1949B3879A
:10759000340183C6070009471306001022859700AF
:1075A0000000E780209C8504AA85E39224FF97B61B
:1075B00001009386A69D1306001022859700000007
:1075C000E78060972AC6080897E0FFFFE780C0DCE5
:1075D000B24504081309010283C7040083C61400DE
:1075E0001147A207DD8E13060010228597000000C8
:1075F000E78040978904AA85E31099FEF25062540F
:10760000D2544259B2592161828029713707400012
:10761000232C811223282113232E1112232A9112A5
:1076200023263113232441132322511317E9FF1F6B
:10763000130909110144594625076302A4548347DD
:107640000900D91793F7F70F6369F600B357F700EE
:10765000858B930619006390071633048540420416
:107660004180BD4763EE87140147630AF416B706ED
:1076700040005946A506B307E90083C70700131564
:1076800007014181D91793F7F70F636FF600B3D75E
:10769000F600858B91CB0507050593170701420579
:1076A000C1834181E3E987FCB309A440C20993D9AE
:1076B0000901A14763FF3727B304A900254697A511
:1076C00001009385A56A268597800100E780C00E9A
:1076D00063110526A547638EF90083C794003547DB
:1076E0006389E70029476386E70093F7F70D639204
:1076F000072497A601009386266813060004814597
:10770000081097000000E7800083AA8597A6010073
:107710009386C66713060004081097000000E780F0
:107720008081AA8597A60100938606671306000448
:10773000081097000000E7800080AA859146130694
:107740000004081097000000E78060A7AA8597B69C
:107750000100938666DC13060004081097F0FFFF13
:10776000E780607DAA8597B601009386668213063E
:107770000004081097F0FFFFE780E07BAA8597B62A
:107780000100938666D913060004081097F0FFFFE6
:10779000E780607A9306700513060004AA85081036
:1077A00097000000E780A0A197A60100938646CE2F
:1077B0001306000485A80504420441803689B5BD3E
:1077C000414697A501009385E54F4A8597800100C2
:1077D000E78080FE97A601009386065005C13D46CE
:1077E00097A50100938585504A8597800100E78021
:1077F000A0FC3DE597A601009386465013060010B5
:107800008145081097F0FFFFE780E072AA85081015
:1078100097000000E78060A097A60100938646C706
:1078200013060010AA85081097F0FFFFE780A070EC
:10783000AA85081097200000E78080DA854483201D
:10784000C1130324811326850329011383244113C3
:107850008329C112032A8112832A41123161828055
:10786000C14763F6870C454697A501009385454AB5
:107870004A8597800100E78020F40147E31905DE7F
:10788000FD572314F100C54497AA0100938A8A4941
:107890009389540093970901139A0401C183135AE1
:1078A0000A0163FA8702338524011546D68597F0CD
:1078B000FFFFE780006F850461DD9305B4FFB385AA
:1078C0004541C2053000C1813305390197F0FFFF02
:1078D000E780E07221C50355810097E0FFFFE78054
:1078E000A04B2A8497A60100938646441306800283
:1078F0008145081097F0FFFFE780E063AA85A28624
:1079000013068002081097000000E780408B97A6BE
:1079100001009386E6B71306800229B717A5010078
:107920001305454297F0FFFFE780207701BF01472D
:107930003DBBB5478144E3F487F0394697A5010084
:10794000938505464A8597800100E780E0E609E9CE
:10795000A2854A8597F0FFFFE780E075AA84C5B548
:10796000394697A501009385A5444A859780010073
:10797000E78080E46315051A930724FFC2072313E9
:107980000100C1830D476373F70A9304E9001146B0
:1079900097A5010093850532268597F0FFFFE780C4
:1079A00040602DC1391442044909418097A9010062
:1079B00093894930814497AA0100938AAA36138A91
:1079C0005400637C8A021546D6853305990097F0EA
:1079D000FFFFE780005D2DC56D14B3059440C2051F
:1079E00013066100C1813305490197F0FFFFE7806D
:1079F000006131C183576100B1EB17A50100130588
:107A0000653E0DB7114697A501009385252B268568
:107A100097F0FFFFE780E05811C939144204490983
:107A2000418097A901009389692969B717A50100C9
:107A300013050539C5BD17A501001305A53CDDB526
:107A40009385140093940501C18095BF2167B98F78
:107A50007917E374F7FA97E7FF1F83C727BC17A5C9
:107A600001001305653CE38F07EA97A601009386A2
:107A7000263461468145280097F0FFFFE780A04B40
:107A8000AA85CE866146280097F0FFFFE780A04ACE
:107A9000AA8597A601009386A69F6146280097F0C5
:107AA000FFFFE78040492A860355610095462C0078
:107AB00097E0FFFFE780803511C517A5010013058A
:107AC000A5388DB597A601009386063A1306800265
:107AD0008145081097F0FFFFE780E045CE86AA8534
:107AE00013068002081097F0FFFFE780C044AA85C4
:107AF00097A601009386863813068002081097F037
:107B0000FFFFE780404383566100AA8511471306B3
:107B10008002081097F0FFFFE780C044CDBBC1474B
:107B2000E3FF87D0414697A501009385A5354A8597
:107B300097800100E78040C8E31305D0834709011F
:107B400013071003639CE700854717C7FF1F230730
:107B5000F78817A5010013052534E9B313070003BF
:107B600017A5010013054536E39EE7DA97C7FF1F07
:107B70002386078617A501001305853365B3814465
:107B80007DB917C5FF1F03456585828097E7FF1FF5
:107B900083C7C7CE89E717230000670063A48280EC
:107BA00097E7FF1F83C727D299EF411106C6972099
:107BB0000000E780C09AB240854717E7FF1F230403
:107BC000F7D0410182808280630E053A638C053ACA
:107BD0001D71B706400086CEA2CCA6CACAC8CEC6C2
:107BE000D2C4D6C2DAC05EDE62DC66DA6AD86ED68D
:107BF00001475948A5061319070113590901637173
:107C0000B902B307E50083C70700D91793F7F70F49
:107C10006368F800B3D7F600858B13061700B9EF39
:107C200033892541420913590901B947AE89AA840C
:107C300063F827053304E500394697A501009385CD
:107C40002516228597800100E78000B715E9CA85CF
:107C5000228597F0FFFFE7800046630E0530F6406F
:107C60006644D6444649B649264A964A064BF25BD4
:107C7000625CD25C425DB25D256182803287A5BFC5
:107C800097E7FF1F83C787BF63840722BD6A396CEC
:107C9000014A17EBFF1F130BEBAF938BFA55938C35
:107CA000FA66130DEC5505A8B387440183C6070097
:107CB00097E7FF1F83D767BC8DE79307A005639BFA
:107CC000F600854717E7FF1F2319F7BA97E7FF1F4D
:107CD0002382D7AC050A93170A01C183E3E637FD77
:107CE000BDBF854D639BB7039307500A639EF600A3
:107CF000894717E7FF1F2312F7B8930750FA17E7D2
:107D0000FF1FA309F7A8F9B79307A005E384F6FCC2
:107D100097E7FF1F239307B675BF13871700420726
:107D2000DA9741832380D70017E6FF1F2317E6B4B5
:107D30008D47E3F1E7FA17E4FF1F0344D4A597E763
:107D4000FF1F83C747A522045D8C9307F4FFC2077A
:107D5000C1839306F00DE3EDF6FA93076400C207C2
:107D6000C183E319F7F693052400C205C18117E525
:107D7000FF1F130545A297F0FFFFE78000AA330716
:107D80008B008347570003474700A207D98F17E7A7
:107D9000FF1F231407AE6312F5100149630DB401F0
:107DA00017E9FF1F0349499F220997E7FF1F83C770
:107DB000B79E3369F90017F5FFFF1305053F97E0FC
:107DC000FFFFE78000396305790963EF2B03630840
:107DD000A9059307EC656303F90697E7FF1F83C7BF
:107DE000A79B05476380E70881CB1387A705137717
:107DF000F70F8D4663F9E6081307F0072300E1004B
:107E0000A300F100894595A8630999059387FA773E
:107E1000E315F9FC97E0FFFFE780807E11A8A285BB
:107E200017E5FF1F1305459797E0FFFFE780004721
:107E3000014597E0FFFFE780C03169BDA28517E5E6
:107E4000FF1F1305659597E0FFFFE780204ECDB734
:107E500097E0FFFFE780A056E1BF97E0FFFFE780D4
:107E6000405CF9B7930710F8130511002300F100E7
:107E700097E0FFFFE780A07BFD450A8597F0FFFFB5
:107E8000E780202B75B7A28517E5FF1F1305C59066
:107E900097E0FFFFE780800261BF9307F007894505
:107EA0000A852310F10097F0FFFFE78080281DB5B9
:107EB000954763F8370B03C704009307500B631211
:107EC000F70A03C714009307B0050144631CF708C1
:107ED000CE85268597E0FFFFE780E03511C917A51D
:107EE00001001305A5D497F0FFFFE780001B85BBB9
:107EF00017A501001305C5D4FDB7B387840083C758
:107F0000070063842701639C47010DC597F0FFFFBD
:107F1000E780E06F97E7FF1F239C078621A8E3EB2C
:107F2000AAFE130715005A9597E6FF1F2392E686CF
:107F30002300F500050493170401C18317E5FF1F13
:107F400003550585E3EB37FBE30B05D097F0FFFF07
:107F5000E780E06BE30505D097E7FF1F239A0782D0
:107F6000FDB901443549294A930AE00417DBFF1F94
:107F7000130B0B7DC9B7CE85268597B0FFFFE78031
:107F80002026F1B98280411126C2AE848D4522C4DB
:107F900006C62A8497B0FFFFE78080EFB71700403E
:107FA00099C803A5C70C418D23A6A70CB240224453
:107FB00092444101828003A5870C418D23A4A70C24
:107FC000F5B78347050003471500A207D98FC207FD
:107FD0006177C18713072720639AE700834525004F
:107FE0003705040017030000670023FA828017E6B4
:107FF000FF1F1306A68D8147B2861303F00FA94811
:108000003308F6000348080013F7F70F6307A80CBE
:10801000630668008507E39517FF2947B387E600E5
:108020002380A70097E7FF1F9387078B5DA8411167
:1080300013D765001347170006C693F63500058B66
:10804000954791CA054699476387C60009469D47EB
:108050006383C600A14713F645003336C00093F68C
:108060008503050685C2A145638BB604E145638A95
:10807000B604930580026388B60493058003639376
:10808000B600914697E5FF1F238DF5AA97E5FF1FE0
:108090002388C5AA97E5FF1FA384D5AABE8517A587
:1080A0000100130525F397700100E780A07EB24020
:1080B000854717E7FF1FA306F7A841018280854681
:1080C000D1B78946C1B78D4675BF17A50100130505
:1080D000E5F2177301006700E37B17D7FF1F130753
:1080E000A77FBA972380B700E147E302F5F493072F
:1080F0007002E30CF5FC82802A872380050081470B
:1081000017D5FF1F1305857C1308F00F2946B3060A
:10811000F50083C606006396E60297D6FF1F938696
:10812000A67BB69783C7070005452380F5009947CE
:10813000636EF7029D4763FDE700E147630DF700BB
:108140008280638506018507E393C7FC0145C5B7B7
:10815000238005008280B737004003C7370083C7FC
:10816000050093F70704D98F2380F50082805D71A5
:1081700052DC56DA5ED6716A97EBFF1F938B8BAD9C
:108180008D6AA6C24EDE62D486C6A2C4CAC05AD8C0
:1081900066D26AD06ECEC1495E8C97D4FF1F93849D
:1081A0006474130A0A20938A7ADC17E9FF1F0349D3
:1081B00069ADB3872B0183C7070093F7F70FC9EFAA
:1081C000B787004003C76700058BE310077C03C730
:1081D0006700118BE30D077E83C75700918B99E3EE
:1081E0006F10200317E7FF1F0347E7A985476304C4
:1081F000F7006F10400197E7FF1FA384E79497D71C
:10820000FF1F2381077A97E7FF1F238F078497E7D4
:10821000FF1F238D079097E7FF1F238A079097D7AB
:10822000FF1FA381077897E7FF1FA38F078297E7B8
:10823000FF1FA38D078E97E7FF1FA38A078E97E77F
:10824000FF1FA381079097E7FF1FA38E07A2B787A1
:10825000004011476F0070779307190093F7F70FED
:108260003D476364F70617E7FF1F230DF7A097E765
:10827000FF1F938727A0CA9783C707001307100221
:1082800093F7F703638EE71E6366F704054463857F
:10829000871CE38C07620947638EE710130700020F
:1082A000E384E74EB7E700E03707400023A0E71874
:1082B00001000100629923000900FD1923A0E710C5
:1082C00093F9F90FE39309EEE5BD97E7FF1F238BC1
:1082D000079A71BF130730026388E70C63E8E7165B
:1082E00013074002638CE70A13070003E39CE7FAD5
:1082F00097E7FF1F93870797CA9703C70700A14710
:108300001377F70FE31BF71483C7640097E6FF1F8B
:108310002380F68297D7FF1F83C7375D91C7FD572C
:1083200097E6FF1F2386F68097D5FF1F83C5955BD1
:1083300097D7FF1FA38EB77E97D7FF1F83C7875A94
:1083400013FB07089306000493F70706639FD74CB7
:108350009307A009638DF51663EAB7129307F0053A
:108360006386F54A930750096384F52A014497D739
:10837000FF1F83C7F77B1547E392E736B7E700E0B7
:108380003707400023A0E71801000100B78600402E
:1083900023808602130680FC6F00500EFD5717D70E
:1083A000FF1F2306F778FDBDFD5717D7FF1F230FCB
:1083B000F776CDBD17A501001305C5D5977001004F
:1083C000E780206597E7FF1F9387C789CA9703C493
:1083D0000700014B97DCFF1F938C4C691374F40F5B
:1083E00017AD0100130D8DD363478B04294597709A
:1083F0000100E780004F854717D7FF1FA306F766E8
:1084000017D7FF1F2303876617D7FF1F230CF772A9
:1084100037E700E0B70640002320D718010001002D
:10842000378600408347A60293F7370F2305F602ED
:108430002320D71085BDB3876C0183C507006A85EB
:10844000050B97700100E780E04479BF854717D797
:10845000FF1F230BF760B9B517E7FF1F13078780CE
:108460004A970347070097D6FF1FA38DF65297D66A
:10847000FF1F238AE65217D7FF1F2305F76C1DB590
:10848000854717D7FF1F230FF75029BD9307400AD1
:108490006389F5349307200B6384F5369307100A3C
:1084A000E396F5EC838724000144E3D207EC97D7E9
:1084B000FF1F83C7574393F63700638A061A0546A2
:1084C000638AC62209466395C61A1D4755A217D569
:1084D000FF1F03454541C94797DCFF1F83CCBC40C4
:1084E00097D5FF1F83C5454017D4FF1F0344D43FD2
:1084F0006315F510CD476392FC1093077008639CD9
:10850000F5021307300FB7170E006308E4001307D6
:10851000900DB7B704006314E40817D7FF1F232F8B
:10852000F760BE8517A501001305C5BF9770010050
:10853000E780403625BD93078008639DF500B307AB
:10854000804013F4F70FB7774600938787CDB3D7F2
:108550008702E1B793079008639AF500B30780405C
:1085600013F4F70F91679387C766D5B79307A008F1
:10857000639BF500B307804013F4F70FB7173D0076
:1085800093870790E9B79307B008639AF500B3079C
:10859000804013F4F70F9167938797D04DBF93F501
:1085A000F5078D47639BF500B307804013F4F70F81
:1085B000B7975B00938707D859BF8947639BF5003E
:1085C000B307804013F4F70FB7770B009387071BAF
:1085D000BDBF8547639AF500B307804013F4F70FDA
:1085E000DD67938767E3A5B7D28785F9B307804036
:1085F00093F7F70FB3D7FA020DB797000000E780A3
:10860000409FA285668597000000E780809EB9BBE9
:108610009305610017D5FF1F0345E52C17D4FF1FF5
:108620000344742C97000000E78040AD930571006F
:10863000228597000000E78060AC3C0017D7FF1F41
:108640002328F760834761002304F100834771000A
:10865000A304F100894717D7FF1F230BF74C83575B
:10866000810017D7FF1F231FF726094409B31547B9
:1086700093F64700B336D00093F78703850685C38A
:108680002146638BC7066146638AC70613068002CC
:108690006388C706130680036393C700914717D604
:1086A000FF1F230FD64897D6FF1FA38BF64897D7F7
:1086B000FF1F2388E74817D7FF1F0347E72293765A
:1086C000070497D7FF1F83C737228DEE1377770CE8
:1086D00093067008630CD7021377F7078D46631271
:1086E000D70CB307F040B7955B0093F7F70F93856E
:1086F00005D849A81947ADBF854755B7894745B73C
:108700008D4771BF930670086311D7021307300FAE
:10871000B7150E006389E7021307900DB7B5040083
:108720006383E7021307700845BF9306800C63114B
:10873000D702B307F040B775460013F7F70F9387DA
:1087400085CDB3D5E70297D7FF1F23A9B73ED9BB85
:108750009306900C631CD700B307F04093F5F70F16
:1087600091679387C766B3D5B702F1BF9306A00C94
:10877000631DD700B307F040B7153D0093F7F70F1F
:1087800093850590B3D5F5027DBF9306B00CE31534
:10879000D7F4B307F04093F5F70F9167938797D01D
:1087A000D9B78946631BD700B307F040B7750B00F4
:1087B00093F7F70F9385051BF1B78546631AD7002A
:1087C000B307F040DD6593F7F70F938565E35DBF71
:1087D000D28535FBB305F04093F5F50FB3D5BA025A
:1087E0009DB783C72400C18B99C7854717D7FF1F43
:1087F0002303F734A5BE97D7FF1F238E0732BDB6DC
:10880000854717D7FF1FA30EF7328DB63C0017D749
:10881000FF1F232FF7420947930700032314F1009A
:1088200097D6FF1F2386E6302DBD63940756A947D0
:1088300063E5B74217970100130707778A05BA95D2
:108840009C41BA97828717D4FF1F0344D409894CEF
:108850006306940D63E68C0685476303F40893076B
:10886000F00F17D7FF1F0347A72C63F6E70017D7B2
:10887000FF1F230FF72A97DCFF1F83CC6C2B930776
:10888000000413F4FC0F63F497011304000497D75A
:10889000FF1F9387E73B03AD070022862685EA8505
:1088A000B38C8C40229D97700100E78040F397D7EE
:1088B000FF1F238F972797D7FF1F23ABA73945BCEF
:1088C0008D47630CF40A9947E31BF4F8979701006E
:1088D0009387077417D7FF1F232CF736A94751B783
:1088E00017D7FF1F0347273A97D7FF1F93874726BE
:1088F0004946979501009385A57A63068700979569
:1089000001009385E5753E8597700100E78020EDB5
:1089100017D7FF1F232EA732C947A1B797D6FF1F2E
:1089200083C66636054797D7FF1F938767226394F0
:10893000E6023E8513067002979501009385C57384
:1089400097700100E780A0E917D7FF1F2322A73007
:108950009307700239B73E851306300497950100DE
:108960009385C56B97700100E78060E717D7FF1FFD
:108970002320A72E93073004EDB597D5FF1F83C59D
:1089800085F6179501001305257B97700100E78098
:1089900060F0054D97DDFF1F83CDED2E97D5FF1FAE
:1089A00083C565F417950100130505796398AD0B30
:1089B00097700100E78000EE97D7FF1F83C7A7F2EB
:1089C000B5CBE36EF4E8179401001304A471638C33
:1089D000B70117940100130464716386970117941B
:1089E000010013042472228597700100E780A00320
:1089F0001375F50F93071500860717D7FF1F230977
:108A0000F7148D4717D7FF1FA304F71497D7FF1F3D
:108A1000938707140147BE861376F70F89076365AE
:108A2000A60297D7FF1F23A5D72297D7FF1F83C77B
:108A3000271205BD979701009387C76317D7FF1FBC
:108A40002328F720914731BD3306E4000346060092
:108A5000A380070005072380C7007DBF9770010032
:108A6000E78040E397D7FF1F83C7E7E7E1D7E368D5
:108A7000F4DE179401001304E463638CA7011794D8
:108A800001001304A4636386970117940100130483
:108A90006464228597700100E780E0F81375F50F94
:108AA00093071500860717D7FF1F2303F70A8D4783
:108AB00017D7FF1FA30EF70897D7FF1F9387470904
:108AC0000147BE861376F70F8907E37CA6F43306C9
:108AD000E40003460600A380070005072380C700C3
:108AE000D5B797D5FF1F83C505E01795010013057E
:108AF000656597700100E780E0D997D7FF1F83C7AE
:108B0000F70493E7470017D7FF1FA301F70483C7B4
:108B1000240017D7FF1FA309F70289B81795010092
:108B20001305856397700100E780A0EE97D7FF1FBC
:108B30009387870183C7070017D7FF1F2304F7DA3E
:108B400017D4FF1F0344C4FE333480000DB01795C3
:108B500001001305A56197700100E78080EB97D7AE
:108B6000FF1F83C7B7FE93E7070117D7FF1FA30FA8
:108B7000F7FC83C7240017D7FF1F2307F7FC6FF00C
:108B8000EFFE179501001305A55F97700100E780C0
:108B900040E803C704007D8B51EFB787004003C74F
:108BA00067021377C70B136727002383E70203C706
:108BB000A7021377C70B136727002385E70203C7B4
:108BC000E7021377C70B136727002387E70203C762
:108BD00027031377C70B136727002389E70285470D
:108BE00017D7FF1F2300F7DC17D7FF1F230EF7E669
:108BF00017D7FF1F230CF7F217D7FF1F2309F7F230
:108C000097D7FF1FA38007DA97D7FF1FA38E07E42C
:108C100097D7FF1FA38C07F097D7FF1FA38907F0F3
:108C200097D7FF1FA38007F297D7FF1FA38D0704D5
:108C30006FF0CFF389476312F70297D7FF1F83C7FF
:108C4000A7CA9146638CD70863E0F604638EE70CED
:108C50006369F70A05476380E70EFD5717D7FF1FC3
:108C6000A308F7EC37074000B7E700E023A0E718B8
:108C700001000100B78600401306F0FC2381C60204
:108C800023A0E7106FF00FE2130720086382E708C4
:108C90006362F70213071008E391E7FC378700408F
:108CA0008347670293F7C70B93E727002303F70275
:108CB0006FF0CFEB130730086389E7021307400812
:108CC000E39DE7F8378700408347270393F7C70BF7
:108CD00093E727002309F7026FF04FE93787004039
:108CE0008347270393F73707F5B737870040834754
:108CF000E70293F7C70B93E727002307F7026FF00C
:108D0000EFE6378700408347E70293F73707F5B769
:108D1000378700408347A70293F7C70B93E72700E5
:108D20002305F7026FF08FE4378700408347A702DF
:108D300093F73707F5B7378700408347670293F704
:108D40003707ADB7179501001305854497700100EB
:108D5000E78020CC97D7FF1F238607B8D5B3179598
:108D600001001305E54397700100E78080CA97D79B
:108D7000FF1F239907B697D7FF1F938767DB03C4AD
:108D80000700894763F3870009441374F40F6FF0F9
:108D90000FDE13070002E392E7EC631B0B0A638FFD
:108DA000F500930720026383F5081795010013056A
:108DB000A54297700100E780E0AD45B51795010029
:108DC0001305C53E97700100E780A0C40144179DBC
:108DD0000100130DED3EA14CB387840083C507004D
:108DE0006A85050497700100E780C0AAE31694FF26
:108DF000178501001305C56F97700100E78060C1FA
:108E000017D4FF1F034444AE01E897D7FF1F238DFB
:108E100007AA014B6FF0AFD58947E310F4E485470B
:108E200017D7FF1F2302F7AA6FF04FD417D6FF1FE3
:108E3000034676AB97D5FF1F83C5E5AA17950100BA
:108E40001305853897700100E780C0A46FF00FD23A
:108E50006380F50693071002E399F5F497D5FF1F99
:108E600083C585A817950100130505389770010083
:108E7000E78040A297D7FF1F23AC97DC97D7FF1F4F
:108E80009387C7CB944383D7470017D7FF1F034768
:108E900047CB17D6FF1F2327D6A41D4497D6FF1F05
:108EA0002394F6A497D7FF1F2381E7A46FF02FCC5C
:108EB00097D5FF1F83C545A31795010013054534BA
:108EC00097700100E780009D97D7FF1F238E079EB4
:108ED00097D7FF1F239807A06FF02FF92547638FBF
:108EE000E7C89946378700406394D702230087027A
:108EF000B7E700E0B706400023A0D7180100010043
:108F0000130600FC2301C70223A0D7106FF08FB90E
:108F10009306100A639FD70023008702B7E700E09B
:108F2000B706400023A0D71801000100130680FCFB
:108F3000D1BF9306A009E381D7FE9306400AE38DD3
:108F4000D7FC93062002639DD700B7E700E0B70681
:108F5000400023A0D7180100010023008702F9B7C1
:108F60008546E384D7FE93070008E300FBFEB7E7DE
:108F700000E0B706400023A0D71801000100130647
:108F800020FC23008702BDBF17D7FF1F034757BA36
:108F90006302F71E63E7E70295476300F7109947FE
:108FA000630AF704B786004023800602B7E700E0B3
:108FB0003707400023A0E718010001001306A0FCBA
:108FC00075B99307F005630AF70093075009630624
:108FD000F70093071002E317F7FCB7E700E0370745
:108FE000400023A0E71801000100B78600401306E7
:108FF00020FC69B117DBFF1F034B8BB39307000401
:109000005A8D63F46701130D000497D7FF1F9387F0
:1090100027C483AC07001374FD0F2286E6852685DE
:1090200097600100E780A07BB3078B40669417D759
:10903000FF1F230FF7AE97D7FF1F23AB87C0B7875C
:109040000040630C0B022380A703B7E600E037065D
:10905000400023A0C6180100010003C727021347E0
:1090600007042381E70203C727021377C70F238171
:10907000E70223A0C6106FF0EFA22380070237E7B4
:1090800000E0B70640002320D718010001001306B6
:1090900020FC2381C7026FF0AFB9378700408347B8
:1090A000370097D6FF1F83C636AA93F70708D58FD8
:1090B000A301F700B7064000B7E700E023A0D718E8
:1090C000010001001306A0FC35BD97D7FF1F938751
:1090D00067B9CA9783C7070093F7F70FC1CF97D730
:1090E000FF1F83C747BAD9E717D7FF1F034757A406
:1090F000930700026310F70883AD040017CDFF1F2C
:10910000034D8D7E97CCFF1F83CC1C7E17CBFF1F9A
:10911000034BAB7DE6876A87DA866E8697C5FF1FAD
:1091200083C5857A179501001305050F9760010027
:10913000E780407697D7FF1F23A2B7A197D7FF1FDD
:109140002380A7A197D7FF1FA38C979F97D7FF1FB7
:109150002389679F97C7FF1FA3878776B7E700E03C
:109160003707400023A0E71801000100B786004040
:109170006FF04FA2B7E700E03707400023A0E718E1
:1091800001000100B786004015BD97D6FF1F83C6BA
:1091900086AF0547639CE60429472381E702094718
:1091A0002383E7022385E70297D7FF1FA38C079845
:1091B00097D7FF1FA38907ACB7870040A38107009B
:1091C00017D7FF1FA302079805472383E700B64080
:1091D000264496440649F259625AD25A425BB25B1F
:1091E000225C925C025DF24D61618280294723819D
:1091F000E70209472383E7022385E7022387E70283
:109200002389E70255B717C7FF1FA30EF76A6FE060
:109210001FFF854717C7FF1F2306F77817D7FF1FC4
:109220002304F78417D7FF1F2302F79017D7FF1FD8
:10923000230FF78E6FE0BFFE854717C7FF1F23037D
:10924000F77617D7FF1F2301F78217D7FF1F230FCA
:10925000F78C17D7FF1F230CF78C17C7FF1FA3032B
:10926000077417D7FF1FA301078017D7FF1FA30F8E
:10927000078A97D7FF1FA38C078A8280411106C6F1
:1092800097000000E78080FBB7870040238007003D
:10929000130740FC2386E7001307C004A386E700FA
:1092A00017C7FF1F130707642398E70017C7FF1F9F
:1092B00013074767239AE70017C7FF1F1307C772F3
:1092C000239CE70017C7FF1F1307477E239EE70075
:1092D00029472381E70209472383E7022385E70221
:1092E0002387E7022389E702A3810700930600F89A
:1092F000A380D700930690022380D700FD562383D6
:10930000D7002381E7009306000537E700E0230B31
:10931000D740B70640002320D71003C717001367B4
:109320001700A380E700B24097D7FF1F239E078056
:1093300041018280411106C697000000E78000F0DD
:10934000B787004023800700130700FC2386E7004F
:109350003147A386E70017C7FF1F1307A7582398B5
:10936000E70017C7FF1F1307E75B239AE70017C73C
:10937000FF1F13076767239CE70029472381E70244
:1093800009472383E7022385E702A38107009306A9
:1093900000F8A380D700930690022380D700FD56E3
:1093A0002383D7002381E7009306000537E700E019
:1093B000230BD740B70640002320D71003C7170060
:1093C00013671700A380E700B24097C7FF1F239DD4
:1093D000077641018280F1679387072017C7FF1F37
:1093E000232EF774854717C7FF1F231BF774A14768
:1093F00017C7FF1F2307F77497C7FF1FA3830774BF
:1094000097C7FF1F2380077497C7FF1F238E074A44
:1094100097C7FF1FA389074A814717C5FF1F130579
:10942000E54AFD5517C6FF1F1306064B2947B3062D
:10943000F5002380B600B306F600238006008507FA
:10944000E397E7FE97C7FF1FA385076E97C7FF1F28
:10945000A383076E97C7FF1F238E076C97C7FF1F55
:109460002389076C97C7FF1F2388076C97C7FF1FC7
:10947000A382076C97C7FF1F238F076A814717C610
:10948000FF1F1306267D4147B306F6002380060022
:109490008507E39BE7FE828017C7FF1F0347A77E70
:1094A00085476316F700170300006700E3E817031A
:1094B00000006700E3DC411122C406C617C7FF1F86
:1094C0000347677C85472E8613F4F50FAA8563173B
:1094D000F70417C5FF1F1305255597600100E780A6
:1094E000003097C7FF1F23810758B78700402384A8
:1094F0008702B7E600E03706400023A0C618010047
:10950000010003C7A7021377C70F2385E702B24004
:10951000224423A0C61001454101828017C5FF1FC8
:109520001305454497600100E780602B97C7FF1F34
:10953000238A0746B787004023828702B7E600E008
:109540003706400023A0C6180100010003C76702C8
:109550001377C70F2383E7025DBF411106C697004B
:109560000000E78080E7B240410117030000670078
:10957000E3F2411106C697F0FFFFE78080BF97C76F
:10958000FF1F83C73742A1CB97C5FF1F83C5A541E6
:1095900089C917C5FF1F1305254197E0FFFFE78025
:1095A000E06297C7FF1FA38F073E97C7FF1F238B5C
:1095B000075837E700E0B70640002320D71801001E
:1095C0000100378600408347660293F7370F230375
:1095D000F6022320D710B2404101828041C9D9C58B
:1095E00097C7FF1F83C74756D1C3011122CC4AC872
:1095F0004EC656C25AC006CE26CA52C42E89AA8961
:109600000144930A0004371B030063772403B30764
:109610008940C207C183BE8463F4FA009304000446
:10962000C204C180130A1BD497C7FF1F83C78737A3
:109630009DE37D1A631C0A00F2406244D244424911
:10964000B249224A924A024B0561828097F0FFFF9D
:10965000E78020B2D1BF338589002694A6854204D5
:1096600097000000E78060E5418045B7828097C79A
:10967000FF1F9387A77318429C4383D64500034579
:10968000070083C5C700035646006396A50083D52F
:10969000E700638DD502011106CE2386A70023972C
:1096A000D700B705CF00DC4B9385757D05077D1688
:1096B0002EC2230001003AC42316C1002317D10093
:1096C00099C30A858297F2400561828082804111A8
:1096D00022C417A4FF1F1304E4D25C4C06C691CB2E
:1096E000C84B01C9B7E70400BC5782975C4C23AA5A
:1096F0000700B240224441018280DC4DDC4B81CF27
:10970000B7E70400904503A38705914517C5FF1FE0
:109710000345056A02838280B7E7040003A30705B7
:10972000A14517C5FF1F0345A56802836D713C085D
:109730003EC6B707E500232291103EC8AA843C0824
:109740003285232611103ECA2324811023202111A3
:109750002E8997300000E780405E2A8497950100AB
:10976000938505AF17750100130505739760010018
:10977000E7804012A28517950100130525BA97606E
:109780000100E7802011294597600100E7806015FE
:10979000B705CB009385757D680097100000E780C2
:1097A000E05FA285680097300000E780604B0147CA
:1097B00081467000CA85268597200000E780608377
:1097C00005CD2A8497950100938585A8177501001A
:1097D0001305856C97600100E780C00BA285179583
:1097E0000100130565B497600100E780A00A2945D0
:1097F00097600100E780E00E8320C11003248110F0
:1098000083244110032901105161828097C7FF1FF3
:109810009387C75918429C43797122D406D60348CE
:10982000070083C807012A8483D6450003554600F4
:109830006396080183D82701638DD8022388070126
:1098400005072399D7003708CC00DC4B1308787D37
:109850003ACC1307F5FF42CA23080100231EE1009A
:10986000231FD10099C7080832C62EC482973246FA
:10987000A245228597000000E78080EBB250225479
:1098800045618280797131469775010093858551D4
:10989000280006D697600100E78060F497A7FF1FB5
:1098A00083D747B6231B0100231C0100231D0100A1
:1098B000231E0100231F010099E3C167FD17231A2E
:1098C000F10097A7FF1F83D707B491EB97C7FF1F3E
:1098D0009387C74D9C439C43DC4783D7070097A6DB
:1098E000FF1F938626B2231BF100D84E83D7460074
:1098F000231CF1005C4B91CB97A7FF1F83C7F7B0E8
:1099000081EB97000000E780C0DCB25045618280A7
:10991000FD1717A6FF1FA30AF6AE0356070183C75C
:1099200006014C472800230FF10097300000E78024
:10993000403097C7FF1F938767479C43014797961F
:1099400001009386669A884330004C089710000007
:10995000E780206A5DD975B799C9B7E7040003A30A
:109960000705A14517C5FF1F034585440283828073
:109970005C4EDC4BB9CFB1CD411122C4177501004B
:10998000130585512E84979501009385A59106C6F0
:1099900097600100E78000F0A2851795010013058C
:1099A000A59297600100E780E0EE294597600100ED
:1099B000E78020F3B7E704002244B24003A3870501
:1099C00017C5FF1F0345C53E1306400691454101DB
:1099D00002838280411122C417A4FF1F130444A0F4
:1099E0001C4C06C689C7DC4399C34C488297584C27
:1099F000B7E70400BC57484B82975C4CB240224406
:109A000023AA07004101828017A7FF1F1307479F62
:109A1000834707009306F00B850793F7F70F63E979
:109A2000F60097A6FF1F238DF69C03450700828052
:109A3000930700F8FDB78357450099E37D55828071
:109A4000011122CC17A4FF1F1304C49B5C4C4AC80D
:109A50004EC6DC4B52C406CE26CA56C2B2892E8AE6
:109A60002A898DC7B7E70400FC5F829797C7FF1F5D
:109A70009387C7319C431307301FB307F5407155D7
:109A80006375F70697000000E780A0C49307D00D28
:109A90007D5563EC3705B7E4040093878900B85817
:109AA000832AC401139507014181029723AAAA00C2
:109AB000484C584921E7978501009385A57C177587
:109AC00001001305653D97600100E780A0DC179554
:109AD00001001305258897600100E780A0DB294578
:109AE00097600100E780E0DF5D55F2406244D244B8
:109AF0004249B249224A924A05618280138749004D
:109B0000B705CF002319E5009385757D31059710C2
:109B10000000E780A028484C834569003105973054
:109B20000000E780E013484C4E86D285310597301F
:109B30000000E78000107146CA8517A5FF1F1305B6
:109B4000658C97600100E78080C9FC5C82970326E2
:109B5000C90097C7FF1F23ABA72211CABC4C85457C
:109B600017C5FF1F0345C52482970145BDBF970058
:109B70000000E78060D1D5BF411106C622C426C2CD
:109B800017C4FF1F1304C42297000000E78060B4CD
:109B9000B7E40400FC4C0345040085458297034567
:109BA0000400224403A3C405B2409244A1454101EC
:109BB0000283411126C297C4FF1F9384241F9C4037
:109BC00006C622C44AC0D5C3DC43C5C35CC123005A
:109BD000B5002A84978501009385056617750100F5
:109BE0001305852B97600100E780C0CA294597605F
:109BF0000100E78000CF9C4023A4070023A20700B8
:109C00009797FF1F9387C77DDC4FDC4B91C7295582
:109C100097000000E78040DC9797FF1F9387877EBF
:109C2000DC4FDC4B89C797000000E78020F537E95F
:109C300004008327C905894517C5FF1F034545173C
:109C400082978327C905914517C5FF1F0345451610
:109C500082979C4003A347016309030022852244A5
:109C6000B2409244024941010283B24022449244EC
:109C70000249410182800111328506CE22CC26CADA
:109C80002E8497300000E780400BAA84978501005E
:109C90009385C55D177501001305052097600100C8
:109CA000E78040BF030784000356640083554400E7
:109CB000A686178501001305A56397600100E7805C
:109CC00060BD294597600100E780A0C19797FF1FFD
:109CD00083C76771639D9700014597000000E78087
:109CE000A0CF81450A8597000000E780C0ECF240D4
:109CF0006244D244056182806D7123248110232641
:109D000011102322911093F745002E8463870714C6
:109D10003C083EC0B707E5003EC23C083EC42317DE
:109D200001002318010023190100231A0100231B3D
:109D300001009797FF1F83D7A76A99E3C167FD17B3
:109D40002316F1009797FF1F83D7A76991EB97C759
:109D5000FF1F9387A7059C439C43DC4783D70700DD
:109D60001797FF1F1307C7672317F100544F835737
:109D700047002318F100DC4AA1E79785010093858D
:109D80002553177501001305251197600100E78021
:109D900060B0178501001305656297600100E780D8
:109DA00060AF294597600100E780A0B313454400E8
:109DB0008320C110032481108324411051618280CB
:109DC0009797FF1F83C737622555D9C3FD1717968D
:109DD000FF1FA30AF66003D6060183470701CC469E
:109DE0000A85230BF10097300000E78080E497C7D5
:109DF000FF1F9387A7FB9C431797FF1F1307475E1F
:109E0000978601009386C64B88430A866C0097109C
:109E10000000E780001EAA8451D997850100938530
:109E20002549177501001305250797600100E78094
:109E300060A6A685178501001305055997600100E6
:109E4000E78040A5294597600100E78080A9268525
:109E500097000000E78040B891BF93F725009DC7A9
:109E6000B7E70400BC47414681452808829725553D
:109E700097000000E78040B628089305F00F970090
:109E80000000E78040D3134524001DB793F7150069
:109E900081CB97000000E780209F1345140009BF85
:109EA00093F78500014589D71797FF1F0347F7559B
:109EB0009797FF1F938707550DC3D84F584B11CF66
:109EC00037E70400384F9047854517C5FF1F034506
:109ED00025EE029713458400E1BD97F0FFFFE78070
:109EE000407FCDBF5C4D411106C688C317C7FF1F19
:109EF000232EF7EAB7E7040083A707081705000039
:109F00001305C5DF8297B24097C7FF1F2382A7EAD8
:109F100001454101828001113335A000A307A10052
:109F2000B7E7040083A7471706CE1306F10085455F
:109F3000130550308297F240056182808280411182
:109F400022C406C697A7FF1F83C7172D054489EFB4
:109F500097B7FF1F83C7876C014499E717A4FF1FBA
:109F60000344842B13441400228597000000E780EB
:109F7000C0FA178501001305E54B09E417850100B8
:109F80001305454C2244B2404101176301006700AC
:109F90006390797122D4A30F010037E40400832772
:109FA000841726D24AD006D6AA842E8913055030AB
:109FB0009305F10132C6829732468347F10193152A
:109FC0000601C18185CB01452EC697000000E780C0
:109FD000C0F483274417B2454A86268582970545F3
:109FE00097000000E78060F3B25022549254025967
:109FF00045618280832744174A8626858297EDB77C
:10A0000041119397050122C406C626C2C1872E843A
:10A0100063D40702B7E40400FC541795FF1F0345FF
:10A020006541829719C1BC5482972165218DB24048
:10A03000224492444101828093F715008DC7B7E70F
:10A04000040083A7471A1796FF1F1306A63D97C55E
:10A05000FF1F9385A5D61795FF1F0345A53D829742
:10A0600013451400E9B793F725000145E9D397C7D5
:10A07000FF1F83C727D685E7B7E7040003A8871A21
:10A080001307401F9797FF1F83C7C73A81461306E0
:10A090004006994517C5FF1F035545D30298134540
:10A0A000240071B797C7FF1F83D747D26398A702D1
:10A0B00017C7FF1F231DB7D017C7FF1F231AC7D00D
:10A0C00017C7FF1F2317D7D02E861785010013054A
:10A0D000E53DBE85175301006700C37B178501006E
:10A0E0001305453E176301006700A392035745001F
:10A0F00097C7FF1F83D787CD6318F702C167F9178A
:10A1000017C7FF1F2324F7CC97C7FF1F23A207CC35
:10A1100097C7FF1F238A07CA97C7FF1F238C07CA49
:10A12000170300006700E3E1178501001305853977
:10A13000176301006700E38D7D15954763E2A71C57
:10A14000178701001307872D0A053A951C41011155
:10A1500022CC06CEBA972E8482871785010013057C
:10A16000E53697600100E780C08AA1A203C72500F9
:10A1700099476311F7022E8597000000E78040F7AA
:10A18000834564001785010013054535975001008C
:10A19000E780407097A7FF1F2380070817850100FD
:10A1A000130585357DBF03C7250095476319F70261
:10A1B000C16717C7FF1F035767C1F91703D5A5006C
:10A1C0006309F702B7E7040083A7C71782971785CB
:10A1D00001001305653397600100E78080838547A0
:10A1E00017A7FF1F230AF70217850100130545343F
:10A1F0008DBF97C7FF1F239BA7BC83D7E50097C6DA
:10A20000FF1F2396F6BC83D7050197C6FF1F239136
:10A21000F6BC83D7250197C6FF1F239CF6BA97C7C4
:10A22000FF1F238307BA631BE502B7E70400BC4F97
:10A2300009661306069089451795FF1F0345851F7C
:10A2400082970356E4008355A40017850100130587
:10A25000E52C97500100E780E06351B79307700F3A
:10A260002316F100B7E7040083A7870D1796FF1F99
:10A270000346461C6C0082974DF9854717C7FF1FA0
:10A280002304F7B45DB7178501001305252BD1BD55
:10A2900083C5250091476392F502178501001305D8
:10A2A000652B97500100E780C07697000000E7809B
:10A2B00040C9F24062440561828099476392F50289
:10A2C000228597000000E780A0E28345640017859F
:10A2D00001001305A52097500100E780A05BD1BFC6
:10A2E0009547639AF50083471400E1F31785010051
:10A2F00013058528BDB51785010013056528E1BF45
:10A3000082803757315F9797FF1F9387E7131307B3
:10A3100077D598C39356C500178701001307C71553
:10A32000BA9683C5060093568500BD8ABA9603C6C1
:10A33000060093564500BD8A3D89BA962A9783C682
:10A34000060003470700238407002383D700A38365
:10A35000E7002382B700A382C7009797FF1F938768
:10A36000A70F2383B700A383C7002384D700A38448
:10A37000E7008280411106C697000000E780A0F840
:10A38000B7E7040083A787141796FF1F1306C60BB1
:10A39000D54501458297B2404D469795FF1F93855D
:10A3A000A50B130570304101170300006700A3BE21
:10A3B00061712324811A37E40400832704082326CB
:10A3C000111A2322911A2320211B232E311917053C
:10A3D0000000130525C382971799FF1F13098905EC
:10A3E000994785442300A900231CF10097850100AB
:10A3F0009385850793074006177501001305C5A9C6
:10A40000231CF1082308910097B9FF1F9389693134
:10A4100097500100E780004883D5090017850100A7
:10A420001305850397500100E780C04629459750E2
:10A430000100E780004B03D5090097000000E7808A
:10A4400080EC832744171008854513055030829708
:10A45000832744171796FF1F13060600CD451305E3
:10A4600070308297832744171796FF1F1306C6FC88
:10A47000B545130560308297832744173008894516
:10A480001305103182978327441730098945130536
:10A4900020318297832744159305000A0D45829742
:10A4A000832744159305000A11458297A30591005F
:10A4B0002306910002CD23080100230C010083270D
:10A4C00084163009914513057040829783278416BE
:10A4D0001306B10085451305004082978327841633
:10A4E0007000854513051040829783278416300835
:10A4F00085451305204082978327841610088545DB
:10A50000130550408297832704157D558297832732
:10A5100044137D5582977D559790FFFFE780E016A5
:10A520008327440C82979790FFFFE78040F28327B0
:10A5300084141796FF1F130626F1D545014582970F
:10A5400089471306700F814528092306F10097807B
:10A55000FFFFE780C0BB8D47130600088145280830
:10A56000230CF1089780FFFFE78060BA9147230C26
:10A57000F100977701009387A783984383C747002B
:10A580003AC8230AF10097C0FFFFE780C0157000AA
:10A59000854505459790FFFFE780401630099305F4
:10A5A000700F09459790FFFFE7804015300893052D
:10A5B00000080D459790FFFFE7804014100895456F
:10A5C00011459790FFFFE7806013C16717B7FF1F22
:10A5D0001307C77FF9171CC3232207001795FF1F16
:10A5E000130505E59790FFFFE78020108327C41D22
:10A5F00017B5FF1F1305057C82973C4803450900EA
:10A60000854582978320C11A0324811A8324411A25
:10A610000329011A8329C1195D618280C16717B8B6
:10A62000FF1F0358A87AF9176301F8083DCDB5CD8F
:10A63000011126CAB7E4040083A7841222CC2E8617
:10A640002315B10006CE2A8401478146ED45428597
:10A6500082972AC611ED17850100130525E397504F
:10A660000100E780003BF2406244D24405618280F1
:10A67000FC440356A100A28582972C0017B5FF1F4A
:10A680000355C5749790FFFFE780E01269DD1785D9
:10A6900001001305E5E097500100E780803783A7AC
:10A6A000C412ED45280082977DBF82800DC5854785
:10A6B0001797FF1FA307F7D89797FF1F238407D883
:10A6C00035469795FF1F938525D7130560301703EF
:10A6D00000006700438C9797FF1FA38407D6E9BF4C
:10A6E00097B7FF1F83C7076FA9EFC16717B7FF1F92
:10A6F0000357C76DF9176306F7044111854722C454
:10A7000017B7FF1F2308F76C37E404007C4C06C61C
:10A7100089451795FF1F0345E5D182970323841AC6
:10A720002244B2409797FF1F83C7C7D017B5FF1FBA
:10A730000355C5691307401F8146314699454101BC
:10A74000028382806D71232481102326111023221D
:10A750009110328401CD8947630AF5028320C1102C
:10A7600003248110832441105161828017850100E8
:10A770001305C5E1AE8497500100E7808029A285CA
:10A78000268597A0FFFFE780005CC9BFB7E70400FC
:10A79000FC4728008297178501001305E5DF9750D5
:10A7A0000100E78000278347810039C41307000BAD
:10A7B0006380E7021387A7051377F70F8D4663EDD4
:10A7C000E602A285280097B0FFFFE780206F79B7E7
:10A7D0008547E3F587F88345910017750100130558
:10A7E000A59FB335B00097A7FF1F238FB78A975057
:10A7F0000100E780200A9DB703479100A207B966D0
:10A80000D98F1387E6556384E70C636DF7042D67D2
:10A810001307B755638FE708636AF70029671307C3
:10A82000A755638FE708A2852800A1BF31671307EA
:10A83000C7556388E70635671307D755E395E7FEE5
:10A840008947E3FD87F097000000E780A0E99305C2
:10A85000E4FFC205C1811305A1009790FFFFE780C7
:10A860002098EDBD3D671306F7556389C706636DF4
:10A87000F6009386E665E398D7FAA285280097C08C
:10A88000FFFFE780A0AAD9BD9306F766638DD704C2
:10A890001307F777E399E7F897C0FFFFE78040D603
:10A8A00075BD0146A285280097C0FFFFE780A08CF8
:10A8B00075B5A285280097C0FFFFE780C09779BDD6
:10A8C000A285280097C0FFFFE780209B41BDA2859D
:10A8D000280097C0FFFFE780609C49B597C0FFFF45
:10A8E000E780E0ADA5BD97C0FFFFE78080B3BDB5B1
:10A8F000C16717B5FF1F0355654DF9176307F500CD
:10A90000B7E7040003A3C7170283828017F3FFFF92
:10A91000670023631773FFFFE702C37A2A840845A1
:10A920002E89B28919C900C1971500009385A586A3
:10A93000610597300100E780000981447D5A971036
:10A940000000E780E03963C7A40481449710000049
:10A95000E780003A63C8A40497B7FF1F9387C747EF
:10A960009C43DC47B307F94091872302F4006383DB
:10A9700009048327C900B307F4409587A302F400B4
:10A980001C4C89C79C4799C3228582971773FFFF88
:10A99000670083765C44139714008504BA9723906C
:10A9A000470171BF1C48139714008504BA97239080
:10A9B000070069BF832789000547B307F4409587DF
:10A9C000A302F40083570400638EE7028DC3094796
:10A9D0006384E7040D47E395E7FA978701009387BF
:10A9E000670E1CCC978701009387C70E11A8978725
:10A9F00001009387A7D41CCC97870100938707D5C4
:10AA00005CC8BDBF97870100938747C01CCC978760
:10AA100001009387A7C0EDB7978701009387470F81
:10AA20001CCC978701009387A70FD9BF95E51773B3
:10AA3000FFFFE702C36A004618448347940075830A
:10AA40009D8B6317F70097100000E78060B448C43F
:10AA50001773FFFF6700E36A82801773FFFFE70247
:10AA6000636613893500C16442094111AA89014412
:10AA7000F11413590901054A2EC697100000E7800A
:10AA80002026B2456348A400014541011773FFFF2A
:10AA90006700836683A7090013171400BA9783D74A
:10AAA00007006388B7006394970063742A01050464
:10AAB000E1B70545D9BF1773FFFFE702C35FAA8956
:10AAC0002E89328BB6843A8ABE8A97A00000E7802E
:10AAD000A00271C9268597200000E780A0108D474D
:10AAE00063E7A7007D551773FFFF6700436083DBB3
:10AAF000440097100000E780A0242A8497100000EB
:10AB0000E78040259307740031443305850263CD07
:10AB1000A70297100000E780A02297100000E780AE
:10AB200020222A8497100000E780C0229307740037
:10AB300031443305850263C3A70497100000E78002
:10AB400020209307450029A897100000E780802067
:10AB5000330585021307F0179307C017E35FA7FAC1
:10AB60002D55E3C277F963040B02D6865286A6857B
:10AB70004A8597200100E780A0C1B5B79710000073
:10AB8000E780401D330585029307C5FFD1BF8327AA
:10AB900049001385C90083D5270097000000E7808E
:10ABA00000EC61F581B769553DBF97B7FF1F23974B
:10ABB000A72297B7FF1F93872722904381470C4610
:10ABC0003307F500420741836393B7008280544600
:10ABD000139847008507C2962390E600D5B797B72C
:10ABE000FF1F9387671F9C4303C58700828017B5AB
:10ABF000FF1F0355A51E82801773FFFFE702234E38
:10AC0000C1671387D7FF630BE502636AA700F117DB
:10AC10006300F50201451773FFFF6700834E13873A
:10AC2000E7FF6302E502FD171D8D13351500E5B73B
:10AC300097500000E780402E7D15C5BF975000005B
:10AC4000E780C002D5BF97500000E780E000EDB775
:10AC50001773FFFFE702A3484111AA8401442EC6DF
:10AC600097100000E780C008B2456348A400014582
:10AC700041011773FFFF6700C3489C481315140078
:10AC80003E9583570500E385B7FE0504C9BF034819
:10AC90005500814693F7F60F63E5070181473E852E
:10ACA0008280584593975600BA9703D727006316BA
:10ACB000B70003D70700E304C7FE8506E1BF83465C
:10ACC000450001479377F70F63E4D700814711A848
:10ACD0001C45131657000507B29703D60700E31368
:10ACE000B6FE3E8582801773FFFFE702A33D9317F0
:10ACF0000501C18797BAFF1F938A0A0E635BF008AC
:10AD000083A70A00C0479C4703570400198D4205DA
:10AD100041816368F500014422851773FFFF6700D6
:10AD2000A33D12052A94CDBFDC4713944900014A84
:10AD30003E94834744006341FA02014A834754002A
:10AD40006349FA028509C20993D9090183A70A0058
:10AD50009847E3EBE9FCC1B71C4413195A00A685D8
:10AD60003E994A8597000000E780C0EE05E1050A9C
:10AD7000C9B75C4413195A00A6853E994A859700C5
:10AD80000000E78020ED19E1050A4DBFE30C09FA48
:10AD900061B7AA8481495DBF1773FFFFE7022334BF
:10ADA0001C452A8481E79307C5001CC51C44231257
:10ADB00004001CC09307F00F63EDB70093F5F50F87
:10ADC000228597200000E780A0E91773FFFF670046
:10ADD000433393940501C167C18063F9F500A685EB
:10ADE000228597200000E780C0ECC5B7C18193F5AC
:10ADF000F50F228597200000E78080E6A685228552
:10AE000097200000E780C0E7C9B797B7FF1F938777
:10AE1000A7FC884382801C4599C797B7FF1F23ADC5
:10AE2000A7FA014582807D55828097B7FF1F9387DF
:10AE3000A7FA984383474500484792073E9582808A
:10AE40001773FFFFE702A329617100451C183EC676
:10AE5000B70780013EC81C183ECA8357440002CE83
:10AE600002D002CC231EF100834784002A8902D23B
:10AE70002301F1023C083ED402D697000000E7808F
:10AE800000FB835705002316F10297500000E7806E
:10AE9000E0CB2307A1025C4003556400F18313F764
:10AEA00017008347F10252055181F99BD98FA307FF
:10AEB000F10297100100E780007D39CDAA84035587
:10AEC000050097A00000E78000C483D704002AD2C1
:10AED0006800231CF10083D72400231DF1001C48C7
:10AEE00003D647008C4397200000E78080D4834737
:10AEF000B400CA86177601001306C66A8117A30537
:10AF0000F4006C00481097200100E78060885D61C4
:10AF10001773FFFF6700E31E2155D5BF1C45B1CF56
:10AF200003C5A700894613576500630BD7028D46FA
:10AF3000630ED70285466300D70213074006330528
:10AF4000E50203C7B700418B15CB83C7B700BD8BA4
:10AF50003355F54082801375F5031307803EC5B75E
:10AF600009671375F50313070771D1BF3727090068
:10AF70001375F5031307077CD9B701458280177352
:10AF8000FFFFE702C31503A98500630C090483478B
:10AF9000B900AE8493F7070E85C303459900930566
:10AFA00020030D810505B305B5028844610597307E
:10AFB0000100E78060B135A02E8597000000E78092
:10AFC00020F62A8419CD97000000E780605C832575
:10AFD000C900B307B54063FA87002E94B305A440B7
:10AFE000E9F51773FFFF6700C31185457DBF177330
:10AFF000FFFFE702C30E2A8403D50500011132C604
:10B0000036C43AC22EC002CA02CC02CE97A00000BB
:10B01000E78060AF82452ACA22852ECC97000000C7
:10B02000E780E0E003570500231EE1009750000091
:10B03000E780C0B1A24632469247230FA10036876F
:10B040004C08B2862285014697000000E780E0A602
:10B0500005611773FFFF6700C30A1773FFFFE7025D
:10B06000030861711C183EC6B70780013EC81C1852
:10B070003ECA3C0800453ED4AA8402CC02CE02D08F
:10B0800002D202D697000000E78060DA83570500FD
:10B0900035592316F10297500000E78020AB2307B3
:10B0A000A10209C48357440081EB21594A855D619F
:10B0B0001773FFFF6700E3040355640052055181D5
:10B0C00097100100E780205C2A8965D18347B4008E
:10B0D00093F7070E99C71305840197300100E780A5
:10B0E000E0A083574400231EF1008347840023011E
:10B0F000F1025C4003550900D98313F70708834721
:10B100001102231CA10093F7F707D98FA300F102C6
:10B1100083572900231DF1005C40F18313F71700CA
:10B120008347F102F99BD98FA307F10297A0000092
:10B13000E780609D2AD235D9834794006800139731
:10B1400057008347B400FD8BD98FA305F4001C483A
:10B1500003D647008C4397200000E78080ADA68788
:10B160001777010013070744740005464C10268525
:10B1700097000000E78060942A890DD98347B400C6
:10B18000A685FD8BA305F40097000000E78060DF33
:10B1900031BF1773FFFFE70283F4832485FE2A84FF
:10B1A0004111268597000000E78080D7834734FF50
:10B1B00093F7070E8DCB2AC6268597000000E780FF
:10B1C00060C809CD834734FFB245FD8BA309F4FE67
:10B1D00091C5228597300100E780008F41011773E8
:10B1E000FFFF670003F27DD98327C4FF268582977E
:10B1F00075F5834734FF93F7070E91C72285973083
:10B200000100E780A08E032584FE97000000E78000
:10B2100000E5E9B71773FFFFE70263E99C414111BD
:10B220002A8903C7070089472E84935667006380E5
:10B23000F6040D466388C6049307F0076304F7021B
:10B240002E8597200000E78040AFAA848149C16B1A
:10B25000130C490097B7FF1F938707B89C43984783
:10B2600063E4E90441011773FFFF670003E803D7B4
:10B2700045008547E3F8E7FE2E8597200000E7802C
:10B2800020B1E1B703D74500E3FEE7FC2E85972008
:10B290000000E78080AAAA84228597200000E7802A
:10B2A000E0ABC204C98C5DB7DC470355A900139A13
:10B2B00049003E9A93170501C187635DF0008357EB
:10B2C0000A006397A70263E774038327CA00034D4C
:10B2D0005A002DA0A1672167A98F1307F7EFE37428
:10B2E000F7FE6397090097000000E780209161FD59
:10B2F00085098DB783278A00034D4A00835DA90025
:10B3000003576900216A138BC7003AC6814A33CAC2
:10B310004D01631E5D0197B7FF1F938767AC9C4388
:10B32000E1DBA2866286814526858297D1B7A16737
:10B330009387F7EF930C4BFF63F24703B2455A85AF
:10B3400097F0FFFFE780A0710DC103278B00104726
:10B3500009CE10436382C4023107D5BFEE856685EE
:10B3600097000000E780008F71F993861A0093FA26
:10B37000F60F130B0B0271BF835644005C43E3E9E5
:10B38000F6F622853AC697200000E7800085A1677F
:10B390009387D7042A8A035D4400324763E8970005
:10B3A0008347D90093E707F8A306F9001C47668591
:10B3B0002286E2858297C1670844FD17337AFA0036
:10B3C000529508C02312A40125B797B7FF1F938792
:10B3D000A7A09843814715C31447814763FFD50051
:10B3E000939745004C47BE9519C903C7550081473F
:10B3F0006375E600DC451606B2973E85828003C77A
:10B4000045008147E37BE6FE16069C45F5B71773BA
:10B41000FFFFE70223CBAA892E8A814497BAFF1F38
:10B42000938A8A9B83A70A00984763E6E400177310
:10B43000FFFF670063CCDC471394440001493E944E
:10B4400013BB140083474400634BF900014913BB4D
:10B45000140083475400634FF9008504E1B70844A2
:10B46000931759005287DA860146A2853E95829944
:10B470000509C9BF4844931759005287DA86054623
:10B48000A2853E9582990509E9B71773FFFFE70288
:10B4900003C5814517F5FFFF1305054897B7FF1F43
:10B4A000239E079297000000E780A0F61773FFFF26
:10B4B000670023C597B7FF1F938707929C4395C3E7
:10B4C0001773FFFFE702A3C1814517F5FFFF1305BF
:10B4D000A54497000000E780C0F31773FFFF6700E3
:10B4E00043C282801773FFFFE702C3BD37E4040045
:10B4F0008327841241112315E100AE893289368AEF
:10B500003A8681460147ED45AA8482972AC621C919
:10B510000356A100D28597400100E780402C832785
:10B52000C413CE8526858297058905C98327440DD6
:10B530002314210101462C00268582972A8401C903
:10B54000B7E7040083A7C712ED452800829722853C
:10B5500041011773FFFF670023BA4944D5B765540B
:10B56000FDB75C41FD175CC182801773FFFFE702E6
:10B5700003B7B7E70400FC5F829795473305F502F0
:10B5800081450D811773FFFF6700A3B71773FFFF96
:10B59000E702E3B4B7E70400FC5F82979547330501
:10B5A000F5020D811773FFFF6700A3B51773FFFF47
:10B5B000E702E3B2B7E7040083A7870B0355050052
:10B5C00082971773FFFF6700C3B31773FFFFE7028C
:10B5D00003B1035505003287AE861786FF1F035659
:10B5E000C6ED97A5FF1F9385E57F97000000E780D4
:10B5F000A0EF1773FFFF6700C3B01773FFFFE702E9
:10B6000003AEB7E7040083A7C71782971773FFFF3E
:10B61000670023AF1773FFFFE70263ACB7E70400CF
:10B6200083A7871397A5FF1F9385C57B8297014545
:10B630001773FFFF6700E3AC1773FFFFE70223AA4E
:10B64000B7E7040083A7C71F81451785FF1F035570
:10B65000C5E282971773FFFF6700A3AA1773FFFF66
:10B66000E702E3A7B7E7040083A7871397A5FF1FA7
:10B6700093854578829701451773FFFF670063A89C
:10B680001773FFFFE702A3A5B7E7040083A7C71F4F
:10B6900081451785FF1F035545E482971773FFFF08
:10B6A000670023A61773FFFFE70263A32E85978029
:10B6B0000000E78060B797800000E78060F41773B0
:10B6C000FFFF670003A41773FFFFE70243A1978002
:10B6D0000000E78060FE1773FFFF670083A25C49EC
:10B6E000E1175CC95CC583572501A1072319F50043
:10B6F00083570501A1072318F5008280F147330520
:10B70000F50297A7FF1F9387E7709C433E958280C1
:10B710008D476315F60803D74600854763F0E708B1
:10B720001773FFFFE702A39B368536842E89971097
:10B730000000E780806029C9835744009314050105
:10B74000C18063E39704228597100000E780E05EE4
:10B75000FD14231294009307A0026300F5029307DF
:10B76000B0026307F50293079002631FF50022857C
:10B7700097000100E780408D01A80146CA85228517
:10B7800097A00000E780E0B71773FFFF670063979B
:10B79000228597100000E780400BFDB7828097A6B6
:10B7A000FF1F938666679C42014599CF9843D44218
:10B7B00017A6FF1F2322E6666396D70097A6FF1FF2
:10B7C00023AEE6641385C7FE82801773FFFFE7028E
:10B7D000039197000000E780A04B71443305850278
:10B7E000914597900000E780A0F011E5655517732B
:10B7F000FFFF6700039197A7FF1F23ABA760970088
:10B800000000E780E04833058502914597900000ED
:10B81000E78000EE61DD97A7FF1F23ADA75E9700CD
:10B820000000E780E04697A7FF1F239DA75C9700D5
:10B830000000E780E04597A7FF1F2396A75C977756
:10B840000100938767DB17A7FF1F2321F75C97078A
:10B850000000938707E917A7FF1F2327F75A014521
:10B8600079B71773FFFFE7028387AA8517A5FF1F24
:10B870001305455997100000E78040631773FFFFD9
:10B88000670023881773FFFFE702638597000000B6
:10B89000E78060FD97100000E780C06297A7FF1F58
:10B8A000938787579C4391CF1387C7FE19CB83D5C6
:10B8B000C7FF17A5FF1F1305A55697200100E780B6
:10B8C000A0201773FFFF6700C3831773FFFFE70212
:10B8D000038197000000E780C0EC09CD8347850015
:10B8E0002A8493F7070499EB0355E50097000000BD
:10B8F000E78080F91773FFFF6700A3808347C500C7
:10B900009304450117A9FF1F1309095185E38327F4
:10B9100009005CC997A7FF1F23A097508327490000
:10B92000F1FB97A7FF1F23AB974EE9B7FD1723063F
:10B93000F500610597800000E78040DE8307840002
:10B9400063CB07048347840093E707F82304F400DC
:10B95000B7E704009C5F82974205A9474181337590
:10B96000F5028347840093F707FCC98F2304F40092
:10B970008347D4003E951C402318A40089CF9843E8
:10B9800019CB8347C4005040814585073305F50234
:10B99000420541810297832709005CC897A7FF1FD2
:10B9A00023AC97468327490089E797A7FF1F23A762
:10B9B00097468347C4009DDF8355040117A5FF1FE9
:10B9C0001305054697200100E780001025B717638F
:10B9D000FFFFE702C37097A7FF1F9387A7699C47E4
:10B9E00001448583858B85E3AE84B2853A869710C2
:10B9F0000000E78000532A8419C597100000E780F3
:10BA00004049829408CC22851763FFFF6700636F6B
:10BA10001763FFFFE702036B41112E8932C6AA8923
:10BA200097000000E780C031324713060502CA863E
:10BA3000970500009385C5CC17A5FF1F1305853C0E
:10BA400097000000E780E0F82A8425C99304C50028
:10BA500097000000E780E0411946AA8526859710E7
:10BA60000000E780001D8545268597100000E780CF
:10BA7000E018177501001305E5B54E9583450500DF
:10BA8000268597100000E780A01D5C48314681455F
:10BA9000A1075CC85CC483572401E1172319F40093
:10BAA00083570401E1172318F4001C4C3E8597606E
:10BAB000FFFFE780C065A3042501228541011763CC
:10BAC000FFFF670063631763FFFFE70243614111F4
:10BAD000AA842EC632C497100000E780E03D004DD6
:10BAE000B2452246834784000CC050C093F7F70349
:10BAF00093E707042304F400231804002685971015
:10BB00000000E780003983479400A9462317A4006A
:10BB100013D7370005073307D7029D8B8507230608
:10BB2000F400A306E40083C70401D8488507230F67
:10BB3000F7FE17A7FF1F1307272E5843232A0400D9
:10BB40009307440129E317A7FF1F2329F72C17A701
:10BB5000FF1F2323F72C17A4FF1F1304642C228537
:10BB600097200100E78080E81C44858B5D8D19E5F6
:10BB70008145228597200100E78000F54101176388
:10BB8000FFFF670003581CC317A7FF1F2328F728D0
:10BB9000D9B71763FFFFE702835497050000938529
:10BBA00065B7014597000000E78000B001451763C5
:10BBB000FFFF670003551763FFFFE702435297003B
:10BBC0000000E78080B01763FFFF6700835383475F
:10BBD000C500A5E31763FFFFE70263502A840355FE
:10BBE000E50097000000E78000C821C1834784007A
:10BBF00093F7F7FB2304F4001C4091C7DC4381C793
:10BC00004C400145829797000000E78080B917A556
:10BC1000FF1F1305E52097200100E78020ED035565
:10BC2000E40097000000E78020C61763FFFF67006D
:10BC3000434D82801763FFFFE702634A97A7FF1F08
:10BC40009387871D97050000938565C817A5FF1F7B
:10BC50001305051D23A0070023A20700972001005C
:10BC6000E78060D61763FFFF6700A3491C4D91CFA3
:10BC7000DC4381CF1763FFFFE7026346834507007C
:10BC800082971763FFFF6700C347828097A7FF1F54
:10BC90009387471B9C4303C50700828097A7FF1F1C
:10BCA0009387471A9C4303C51700828097A7FF1FFD
:10BCB000938747199C4303C52700828097A7FF1FDE
:10BCC000938747189C4303C54700828097A7FF1FAF
:10BCD000938747179C4303C53700828097A7FF1FB0
:10BCE000938747169C4303C55700828097A7FF1F81
:10BCF000938747159C4303C56700828097A7FF1F62
:10BD0000938747149C4303C57700828097A7FF1F42
:10BD1000938747139C4303C58700828097A7FF1F23
:10BD2000938747129C4303C59700828097A7FF1F04
:10BD3000938747119C4303C5A700828097A7FF1FE5
:10BD4000938747109C4303C5B70011E11D458280CE
:10BD500097A7FF1F9387070F9C4303C5C7008280E7
:10BD600097A7FF1F9387070E9C4303C5D7008280C8
:10BD700097A7FF1F9387070D9C4303C5E7008280A9
:10BD800097A7FF1F9387070C9C4303D50701828069
:10BD900097A7FF1F9387070B9C4303C5270182804A
:10BDA00097A7FF1F9387070A9C4303D5470182800B
:10BDB00097A7FF1F938707099C4303D567018280DC
:10BDC00097A7FF1F938707089C4303D587018280AD
:10BDD00097A7FF1F938707079C4303C5A70182808E
:10BDE00097A7FF1F938707069C4303C5B70182806F
:10BDF00097A7FF1F938707059C4303C5C701828050
:10BE000097A7FF1F938707049C4303C5D701828030
:10BE100097A7FF1F938707039C438857828097A7A4
:10BE2000FF1F938727029C4303D5C702828097A7F1
:10BE3000FF1F938727019C4303D5E70219E11305F0
:10BE4000800C828097A7FF1F9387C7FF9C4303C581
:10BE50000703828097A7FF1F9387C7FE9C43C85B99
:10BE6000828097A7FF1F938767FD8843828097A7EB
:10BE7000FF1F9387E7FC8843828019E17D5582800C
:10BE8000F5DE984265DFFDD917A7FF1F1307871E50
:10BE90001847AA877155058B631D072403C5070042
:10BEA0001547E37DA7FC03C737001305F0057D1791
:10BEB0001377F70FE364E5FC03C35700E30003FCCB
:10BEC00083C86700E38C08FA03C7770049457917F0
:10BED0001377F70FE364E5FA03C7A70011481305CA
:10BEE000F7FF1375F50FE36BA8F803CE97000D4825
:10BEF0001305FEFF1375F50FE362A8F803C8B7003A
:10BF00006309080065181378F80F1305600DE367DF
:10BF100005F703C5C700794879151375F50FE36F69
:10BF2000A8F403C8D7000D457D181378F80FE36710
:10BF300005F503D80701930E40175118420813580E
:10BF40000801E3ED0EF303C8E7007D181378F80F3E
:10BF5000E36605F303C827017D181378F80FE36F34
:10BF600005F103C88700C54E75181378F80FE3E78D
:10BF70000EF103D86701856E938EBEE06D184208FE
:10BF800013580801E3EC0EEF03D847016D1842087F
:10BF900013580801E3E40EEF03D88701791842082B
:10BFA00013580801E36C05ED03C8A7017D18137849
:10BFB000F80FE36505ED03C5B7011D487D15137541
:10BFC000F50FE36DA8EA03C5D7017148791513751C
:10BFD000F50FE365A8EA03D5E7011308E00F7D1527
:10BFE00042054181E36CA8E803C507024948791579
:10BFF0001375F50FE364A8E8C85301C937C83400C6
:10C000005915130858BFE36BA8E603A8870237C584
:10C010003400130555BF5918E36205E717A5FF1F44
:10C020002320C5E203C6050117A5FF1F232CF5E059
:10C030000545E375C5E403D82501D04933760603E9
:10C04000E31E06E203C61501E30A06E217A6FF1F78
:10C050002326B6DE83C5270001466387A50003C6F5
:10C060001700F1453306B60283C707039305C002E4
:10C0700072971A071307C70516031A97960846976B
:10C08000B387B70241553E973297420741836362B7
:10C09000E8061763FFFFE7028304368597800000F8
:10C0A000E780207097000100E780A04F2A8497A0C6
:10C0B0000000E78000622A9497F00000E780E02DFE
:10C0C0002A9497900000E78020892A9497F0FFFF38
:10C0D000E780E06F2A9497400000E780E09A2A9476
:10C0E00097700000E78020A422951763FFFF670088
:10C0F000430182801763FFFFE70263FE4111A3073C
:10C10000A10097A00000E78020CD9305F10017055E
:10C1100000001305E5B597F0FFFFE780802F01458C
:10C1200041011763FFFF6700C3FD1763FFFFE702CD
:10C1300083F817A4FF1F1304E4F30328840079593C
:10C140009368180097A4FF1F23AA14F3137818000C
:10C1500063100802BA84BE89368B328A2E89AA8A75
:10C1600097F0FFFFE780E0A77D15269519E5315987
:10C170004A851763FFFF670083F797F0FFFFE780AB
:10C1800040A67D152695A167E353F5FE97A7FF1FEF
:10C190009387472598433E8C814B01CB014597F00F
:10C1A0000000E780A04B933B15004A85DA8656864F
:10C1B000D28597900000E78040552A8911CD1C4414
:10C1C000F99B17A7FF1F232BF7EA83270C00CDD37A
:10C1D000E3800BFA829769BF268597A7FF1F23ADDF
:10C1E00007E897F0FFFFE780809C4146CE8517A5C2
:10C1F000FF1F1305A5F197300100E780405E97D03F
:10C200000000E780C0A00325040B97D00000E78062
:10C2100080A4054597D00000E78080AB05459700D6
:10C220000000E78060EDA9B797A7FF1F938787E419
:10C230009C47858BEDC71763FFFFE70243EA17A50D
:10C24000FF1F1305E5EA97A7FF1F23A507E297A79E
:10C25000FF1F23A307E297A7FF1F23A107E2972051
:10C260000100E780A08897500000E78060FD9710EC
:10C270000100E780205497100100E780205A97A71B
:10C28000FF1F9387A7DD9C4391C70545978000005A
:10C29000E780C02797A7FF1F938707C69C4399C7CE
:10C2A00041657D1597700000E780C0A997F00000F8
:10C2B000E780604597D00000E780009797A7FF1FB1
:10C2C000938747F09C43139717016356070097F035
:10C2D0000000E78080B497A7FF1F23A907E297A774
:10C2E000FF1F23A707E297A7FF1F23A507E297A732
:10C2F000FF1F23A307E297000000E780008C970050
:10C300000000E780807997F0FFFFE780401897F002
:10C310000000E780C0DD1763FFFF670083DE8280D7
:10C3200097A7FF1F938707D58843828097A7FF1F92
:10C33000938747D4C8438280B7E7B00093870750FC
:10C3400063E1A70297A7FF1F9387C7D2D843FD5782
:10C350006367E50097A7FF1F23A0A7D281473E850B
:10C360008280B957EDBF1763FFFFE70243D797807D
:10C370000000E780407997800000E780A07B17638A
:10C38000FFFF670003D817A7FF1F1307A7CE83255A
:10C39000470B1DC51763FFFFE70263D497A7FF1F75
:10C3A000938747AA9C432A8403C61700B7E7040073
:10C3B000FC470E06829722851763FFFF670063D450
:10C3C0002E8582801763FFFFE702C3CF2A84930480
:10C3D000140201112E85B289A685214636C63A89F6
:10C3E00097300100E780403D0DE9B24638082686C7
:10C3F000CE851305940497500000E78060412146E4
:10C400002C084A8597300100E780003B1335150062
:10C4100005611763FFFF670023CE0145D5BF176392
:10C42000FFFFE702C3CB9305450617A5FF1F1305C2
:10C43000A5A197100100E78020691763FFFF67003F
:10C4400043CC1763FFFFE70283C941112EC697F063
:10C45000FFFFE780E013B24588C141011763FFFF8A
:10C46000670023CA1763FFFFE702C3C5AA842E84AF
:10C4700097800000E780006CAA8985452285970097
:10C480000000E780E07D83C7E4011389940899E305
:10C4900013890403CE85228597000000E780407C45
:10C4A000214693051902228597000000E7806078F5
:10C4B00097A7FF1F938707BC8C4322859710000026
:10C4C000E780C08221469385840222859700000080
:10C4D000E78020761763FFFF670003C21763FFFF43
:10C4E000E70263BD397197F00000E780E0B493057F
:10C4F000400661E997800000E78000606302051450
:10C5000097A7FF1F83C7079613B7170097A6FF1FAC
:10C51000238AE694014499CFC16417A9FF1F130928
:10C5200069B59309400EFD1497F0FFFFE780407F47
:10C530006342A40A97F0FFFFE78080054169B729AD
:10C540000900096AFD7A2A8B81447D199389F97B58
:10C55000130A0A71938A8AC797F0FFFFE780407C2D
:10C5600063D7A4041304400EB387840217A7FF1FE8
:10C57000130747B00324070B3E948357C40163821B
:10C58000270B18403307EB4063EAE9008347440078
:10C590008507B3874703D6976365F708014681454A
:10C5A000094597F0FFFFE780E046AA8B29E5974011
:10C5B0000000E780808385476317F50689659385CA
:10C5C000057117A5FF1F1305258897100100E78047
:10C5D000A04F95A0B30734030327090BBA9703D7DD
:10C5E000C7016308970003C75700A382070023828F
:10C5F000E700050415BF9305C500228597000000DC
:10C60000E78080E65E852286976501009385C5FDFB
:10C6100097F0FFFFE780604B5E8597100000E78092
:10C62000608A850415BF97A7FF1F9387A7A49C471F
:10C630008D83858BC1F721611763FFFF670023ABF3
:10C6400001468545094502D002D202D402D697F0B0
:10C65000FFFFE780203CAA8479DD97F00000E780A7
:10C66000E09C1389C4002A8481454A859700000014
:10C67000E780005F0C4041464A8597000000E78054
:10C68000405B832944006385090C4E8502D802DA99
:10C6900002DC02DE97300100E780E0382ACE141079
:10C6A00005462C0808184ECC97500000E780E00A99
:10C6B0001375F50F51ED8355840093E525004A85E8
:10C6C00097000000E780E05E11460C104A85970055
:10C6D0000000E7800056014697650100938545F10B
:10C6E000268597F0FFFFE780403E268597000000F3
:10C6F000E780407D5C40A1D3014685450D4597F01C
:10C70000FFFFE7802031AA841DD548401389C4006B
:10C7100097300100E78020312AC64A859700000043
:10C72000E780404C3246636FC5004C404A85970015
:10C730000000E780005001468145268597F0FFFF05
:10C74000E780A038268597000000E780A077E5B550
:10C7500083558400ADB71763FFFFE702439897A79F
:10C76000FF1F938727919C471DC193E7870017956B
:10C77000FF1F1305656D17A7FF1F2321F790971063
:10C780000100E78040321763FFFF67008397DD9B5E
:10C7900017A7FF1F2324F78E97300000E780E0647F
:10C7A0007DF11795FF1F1305256A97100100E7809B
:10C7B000E033D1BF1763FFFFE702E38F4169AA8926
:10C7C0002E8AB28A368BBA8B814417ACFF1F130CAA
:10C7D0006C8A930C400E7D1997F0FFFFE780405460
:10C7E00063C4A40001443DA03384940383270C0B4D
:10C7F0003E948357C401638627055A87D68652869E
:10C80000CE851305040397000000E780E0BB01C953
:10C8100023800B0022851763FFFF6700438D83474A
:10C82000F40185C35A87D6865286CE8513059408AF
:10C8300097000000E78040B909C585472380FB00C9
:10C84000D1BF850451BF835745006380071E17631E
:10C85000FFFFE702238701112A8497000000E78089
:10C86000C04D09C985476309F50605611763FFFFD8
:10C870006700838897E00000E780007C7DF58357A0
:10C8800044004947ED9BE392E7FEC14522859700AE
:10C890000000E7804033AA84228597000000E780EB
:10C8A000204F0357440002CE91472A89631AF700AC
:10C8B000228597000000E780A0513C082ACC3ECE9C
:10C8C00097E00000E78080765C55C5D374084A86FF
:10C8D000A6850545829751BF03574400D147E3F62B
:10C8E000E7F8032A0400C1690149979AFF1F938A58
:10C8F0006A78130B400EFD1997F0FFFFE780404266
:10C90000634FA90E2285032A040097000000E780E8
:10C91000C042A1452A89228597000000E780A02A0D
:10C92000AA84228597000000E780804A14402A8666
:10C93000AA8978082685CA8597000000E780C0E7A5
:10C94000AA8405D503C7F40189476315F700834717
:10C95000C10181DF5546D2851385640097300100FF
:10C96000E780E0E7014597800000E780C01901C536
:10C9700083D7C401A5E79797FF1F9387A76F9C47AD
:10C9800093551900858913D73700058B01CF89830B
:10C99000858B6399B70001452EC697000000E7809C
:10C9A000C0DBB2454E8597800000E780601F0346DC
:10C9B000C1012A8493751900268597900000E780AD
:10C9C000E03935C1268597800000E780E01826858C
:10C9D00011C0014597800000E780004C97300000AF
:10C9E000E780A0408547E312F5E883C754001307AA
:10C9F000F00FE38CE7E68507A382F400BDB5B3042E
:10CA0000690383A70A0BBE9483D7C401638B3701E4
:10CA10005546D2851385640097300100E780C0D960
:10CA200055DD0509D1BD5DD86DB782801753FFFF75
:10CA3000E702436997800000E780000C05C1C164EC
:10CA400001441799FF1F1309E9629309400EFD1471
:10CA500097F0FFFFE780C02C634EA4001795FF1FDF
:10CA60001305853E97100100E780E0031753FFFF91
:10CA700067008368330534038327090B3E9583578A
:10CA8000C501638897002312050097800000E780A6
:10CA9000A00C050475BF9797FF1F9387A75D9C4760
:10CAA0008D83858B8DE31753FFFFE7024363179553
:10CAB000FF1F1305653997100100E7802003175306
:10CAC000FFFF6700036482801753FFFFE7022361C3
:10CAD000970500009385C5A01795FF1F1305C53660
:10CAE00097100100E78020EE1753FFFF6700636196
:10CAF0001753FFFFE702A35E8841B7E70400BC5B62
:10CB0000050542054181829709C585472300F50047
:10CB100005051753FFFF6700C35E83C7F5FF2E852A
:10CB20008507A38FF5FE828083C7F5FFFD1793F776
:10CB3000F70FA38FF5FE99EF1753FFFFE702235A74
:10CB4000B7E70400BC571385F5FF82971753FFFF23
:10CB50006700235B82801C41035745008D8FBA9587
:10CB60001CC12312B5003E85828093D78500A205A3
:10CB70001441DD8D835745001387E6FF18C18907EF
:10CB80002312F50013D685004111238FB6FEA38F23
:10CB9000C6FE4101828018419307F7FF1CC18357ED
:10CBA000450085072312F500A30FB7FE8280835747
:10CBB00045008D8F2312F5001C41BE950CC12E85BA
:10CBC0008280AA8703D7470008410D8FAA95239238
:10CBD000E7008CC38280184108453305A740828056
:10CBE00083574500035765001D8F1C410845338559
:10CBF000A7403305A74082801753FFFFE702234E6B
:10CC000041112EC62A8497000000E780A0FDB2459E
:10CC10006373B50001A0835744000840BE952312FA
:10CC2000B4003E9541011753FFFF6700834D175332
:10CC3000FFFFE702C34A41112E84B28532C6970036
:10CC40000000E780A0FB3246A28597300100E78014
:10CC500000B941011753FFFF6700A34A1753FFFFB5
:10CC6000E702E3472E84854597000000E78000F93E
:10CC7000230085001753FFFF6700A3481753FFFFEA
:10CC8000E702E34541112317B100894597000000F1
:10CC9000E780C0F68347E1002300F5008347F100F9
:10CCA000A300F50041011753FFFF670083451753A9
:10CCB000FFFFE702C34293D78500A2054111DD8D36
:10CCC0002317B100894597000000E78020F38347D0
:10CCD000E1002300F5008347F100A300F5004101C6
:10CCE0001753FFFF6700E3411753FFFFE702233F9E
:10CCF0001397850193D78501C166938606F0D98F76
:10CD000013D78500758FD98FA2053707FF00F98DDE
:10CD10004111DD8D2EC6914597000000E78000EEA1
:10CD20006C00114697300100E78060AB410117535A
:10CD3000FFFF6700033D1753FFFFE702433A1C4123
:10CD4000854503C4070097000000E78080E6228540
:10CD50001753FFFF6700E33A1753FFFFE70223383B
:10CD60001C414111894503C7070083C717002307EA
:10CD7000E100A307F10097000000E78080E303557E
:10CD8000E10041011753FFFF6700A3371753FFFF6F
:10CD9000E702E3341C414111894503C7070083C7FB
:10CDA00017002307E100A307F10097000000E780C8
:10CDB00040E08357E100410113D58700A2075D8D54
:10CDC000420541811753FFFF6700A3331753FFFF4D
:10CDD000E702E3300C4141112A8411466800973084
:10CDE0000100E780C09F9145228597000000E78001
:10CDF00040DCB247C166938606F01397870113D5CE
:10CE00008701598D13D78700758F598DA207370772
:10CE1000FF00F98F5D8D41011753FFFF6700632EFF
:10CE20001C45BE950CC18280AE87944391E6584163
:10CE300001EF0CC15CC1828003C757001367170064
:10CE4000A382E700B687D5B70CC3EDB7AA87084120
:10CE500019CD1841D44398C36313D500D8C32A878A
:10CE6000034657009376160081E623200700828050
:10CE7000944381CA8C4203A847008CC36393060184
:10CE8000CCC3799A14C3A302C7003687D1BF1C450F
:10CE9000DC471D8DB777DBB6938777DB09853305D4
:10CEA000F502420541818280F147B385F50248458C
:10CEB0002E9582808347450085072302F5008280F6
:10CEC0001753FFFFE702A3212A8409E41753FFFF4A
:10CED0006700232383474400F5DBFD1793F7F70F23
:10CEE0002302F400E5F71C4403D72700050723912C
:10CEF000E700DC4399C3228582974C4889CD83475C
:10CF00005400898B99E71C4422859C479C439C478D
:10CF10008297232A04000040232004007DB7175382
:10CF2000FFFFE702C31B8357250041112EC681EB8B
:10CF30000144228541011753FFFF6700831C0357FB
:10CF400005008147F146E305F7FEB385D70240456A
:10CF500085072E948345440008C4F5F5B247AA849A
:10CF600081E7232A040009A81C456C0022859C4304
:10CF70009C43829748C84DDD85472312F400B24791
:10CF800023200400231804002319F4005C485CC427
:10CF900083D72400FD172391F40061BF1753FFFFCF
:10CFA000E702E3139797FF1F938707EC8843232635
:10CFB000050023240500410597100100E78000B318
:10CFC0001753FFFF6700E3131753FFFFE702231117
:10CFD0001794FF1F130444E91C40411199CF9C474B
:10CFE0002300B5002AC65CC197000000E78040FB23
:10CFF0001C40DC4399C33245829741011753FFFF20
:10D00000670023100347450029E3584DAA877D5543
:10D010001DCF1753FFFFE702830C1CC3DC47979615
:10D02000FF1F23A3E6E4F156130507012390D70061
:10D03000970500009385050297100100E780A098EE
:10D0400001451753FFFF6700C30B7D558280828027
:10D050001753FFFFE702A30801116146814528002D
:10D060009750FFFFE780A00A9797FF1F9387C7DFBE
:10D070009C4328009305F00FDC473EC69700000054
:10D08000E780C0F405611753FFFF67008307979798
:10D09000FF1F938767DD9C43D847A1679387C7022B
:10D0A000631EF70A397106DE22DC26DA80004AD8D0
:10D0B0004ED652D456D23285B28497000000E78013
:10D0C000C0C7AA89268597000000E78020C92318D9
:10D0D000A4FC268597000000E78040C82319A4FC23
:10D0E000268597000000E78060C783D744000A8A3E
:10D0F000231AA4FC858393F7F70F230EF4FC86070D
:10D10000BD0793F7073F3301F1408A8A01498347FE
:10D11000C4FD6367F902CE85130584FC232C54FDFE
:10D1200097000000E78080EA5281130104FCF2506E
:10D130006254D2544259B259225A925A2161828081
:10D14000268597000000E78060C193171900D697E5
:10D1500005092390A7001379F90F55BF828097978F
:10D16000FF1F938767D09C43D847A1679387A70287
:10D17000631AF70A397106DE22DC26DA80004AD803
:10D180004ED652D456D23285B28497000000E78042
:10D19000C0BAAA89268597000000E78020BCFD5709
:10D1A0002318A4FC26852319F4FC97000000E780CF
:10D1B000E0BA83D744000A8A231AA4FC858393F734
:10D1C000F70F230EF4FC8607BD0793F7073F3301E3
:10D1D000F1408A8A01498347C4FD6367F902CE851D
:10D1E000130584FC232C54FD97000000E78000DE2B
:10D1F0005281130104FCF2506254D2544259B25984
:10D20000225A925A21618280268597000000E78089
:10D21000E0B493171900D69705092390A700137956
:10D22000F90F55BF82809797FF1F9387E7C39C43F1
:10D23000D847A16789076310F70A397106DE22DC37
:10D2400026DA80004AD84ED652D456D23285328958
:10D2500097000000E78060AEAA894A859700000029
:10D26000E780C0AF835749000A8A2318A4FC85834E
:10D2700093F7F70F230CF4FC8607BD0793F7073FDE
:10D280003301F1408A8A8144834784FD63E7F402D5
:10D29000CE85130584FC232A54FD97000000E78007
:10D2A000E0D25281130104FCF2506254D25442592C
:10D2B000B259225A925A216182804A859700000011
:10D2C000E780C0A993971400D69785042390A70000
:10D2D00093F4F40F55BF82809797FF1F9387C7B8C9
:10D2E0009C43D847A1679387E704631EF70A397107
:10D2F00006DE22DC26DA80004AD84ED652D456D238
:10D300003285B28497000000E78020A3AA89268591
:10D3100097000000E78080A42318A4FC26859700CE
:10D320000000E780A0A3231AA4FC26859700000034
:10D33000E780C0A283D744000A8A2319A4FC85830E
:10D3400093F7F70F230EF4FC8607BD0793F7073F0B
:10D350003301F1408A8A01498347C4FD6367F902BA
:10D36000CE85130584FC232C54FD97000000E78034
:10D37000E0C55281130104FCF2506254D254425968
:10D38000B259225A925A2161828026859700000064
:10D39000E780C09C93171900D69705092390A70032
:10D3A0001379F90F55BF82809797FF1F9387C7ABFB
:10D3B0009C43D847A1679387C704631AF70A39715A
:10D3C00006DE22DC26DA80004AD84ED652D456D267
:10D3D0003285B28497000000E7802096AA892685CE
:10D3E00097000000E7808097FD572318A4FC26854E
:10D3F000231AF4FC97000000E780409683D744008E
:10D400000A8A2319A4FC858393F7F70F230EF4FCF3
:10D410008607BD0793F7073F3301F1408A8A014928
:10D420008347C4FD6367F902CE85130584FC232C72
:10D4300054FD97000000E78060B95281130104FC9D
:10D44000F2506254D2544259B259225A925A21612E
:10D450008280268597000000E7804090931719008E
:10D46000D69705092390A7001379F90F55BF82803D
:10D470009797FF1F9387479F9C43D847A167DD0776
:10D480006317F7041753FFFFE70263C5797132850D
:10D49000328497000000E780408A2AC622859700E0
:10D4A0000000E780A08B2311A102228597000000D5
:10D4B000E780A088B2452300A10228089700000059
:10D4C000E780C0B045611753FFFF670083C38280C8
:10D4D0009797FF1F938747999C43D847A1679387E6
:10D4E00087046317F7041753FFFFE70243BF7971FF
:10D4F0003285328497000000E78020842AC6228586
:10D5000097000000E78080852311A1022285970003
:10D510000000E7808082B2452300A102280897001E
:10D520000000E780A0AA45611753FFFF670063BDB5
:10D5300082809797FF1F938727939C43D847A167C3
:10D540009387A7046312F7021753FFFFE70223B97B
:10D5500001112800814597000000E78020A70561A0
:10D560001753FFFF6700E3B982809797FF1F9387E8
:10D57000A78F9C43D847A167938757026319F70287
:10D580001753FFFFE702A3B50111328597F0FFFFA4
:10D59000E780A07A2308A1008145280097000000B9
:10D5A000E780C0A205611753FFFF670083B5828043
:10D5B0009797FF1F9387478B9C43D847A167938713
:10D5C000E702631BF7041753FFFFE70243B10111A2
:10D5D0003285328497F0FFFFE7804078AA84228565
:10D5E00097F0FFFFE7808077854709E9228597F06C
:10D5F000FFFFE78080744205B337A0002800814513
:10D60000231891003ECA97000000E780209C056126
:10D610001753FFFF6700E3AE82809797FF1F938742
:10D62000A7849C43D84799476313F7081753FFFF14
:10D63000E702E3AA79713285328497F0FFFFE78031
:10D64000C06F2AC6228597F0FFFFE7802071231064
:10D65000A102228597F0FFFFE780206E2301A1023F
:10D66000228597F0FFFFE780406DA301A10222858C
:10D6700097F0FFFFE780606C2302A102228597F0FC
:10D68000FFFFE780806B2313A102228597F0FFFF45
:10D69000E780A06AB2452314A10228089700000081
:10D6A000E780C09245611753FFFF670083A5828022
:10D6B0009787FF1F9387477B9C43D847A167938732
:10D6C000C7036313F7081753FFFFE70243A17971FC
:10D6D0003285328497F0FFFFE78020662AC62285D4
:10D6E00097F0FFFFE78080672310A102228597F063
:10D6F000FFFFE780A0662311A102228597F0FFFFBC
:10D70000E780A0632302A102228597F0FFFFE78054
:10D71000C062A302A102228597F0FFFFE780E061CB
:10D720002303A102228597F0FFFFE7800061B24545
:10D73000A303A102280897000000E7802089456123
:10D740001753FFFF6700E39B82801753FFFFE70239
:10D75000039901112A8497F0FFFFE780005EAA84F5
:10D76000228597F0FFFFE780605F228597F0FFFF3B
:10D77000E780C05E035744008D4763F7E7002285CA
:10D7800097F0FFFFE780805D228597F0FFFFE7803D
:10D79000E05C2800A68597000000E78020830561F3
:10D7A0001753FFFF6700E3959787FF1F9387C76BAA
:10D7B0009C43D847A167FD07631FF7001753FFFF7E
:10D7C000E702E391328597000000E78040F81753A5
:10D7D000FFFF6700039382809787FF1F9387C768C7
:10D7E0009C43D847A167E5076315F7081753FFFF68
:10D7F000E702E38E79713285328497F0FFFFE7808C
:10D80000C0532AC6228597F0FFFFE7802055228566
:10D8100097F0FFFFE78080542310A102228597F044
:10D82000FFFFE780A053520551812311A1022285F9
:10D830002302010297F0FFFFE7802050A302A1021C
:10D84000228597F0FFFFE780404F2303A102228546
:10D8500097F0FFFFE780604EB245A303A1022808BE
:10D8600097F0FFFFE780807645611753FFFF670061
:10D87000438982809787FF1F9387075F9C43D84720
:10D88000A1679387E703631FF7001753FFFFE702C2
:10D890000385328597000000E78060EB1753FFFF98
:10D8A0006700238682809787FF1F9387E75B9C43EF
:10D8B000D847A16793874704631EF7021753FFFFFA
:10D8C000E702E38179713285328497F0FFFFE780C8
:10D8D000C0462AC6228597F0FFFFE7802048B24560
:10D8E000280897F0FFFFE780606E45611753FFFF40
:10D8F0006700238182809787FF1F9387E7569C43A9
:10D90000D847A167938787026310F7041743FFFF87
:10D91000E702E37C79713285328497F0FFFFE7807C
:10D92000C0412AC6228597F0FFFFE7800041B2453B
:10D930002300A102280897F0FFFFE78020694561D6
:10D940001743FFFF6700E37B82801743FFFFE70277
:10D950000379011197F0FFFFE780203EAA85280098
:10D9600097F0FFFFE780806605611743FFFF6700C0
:10D9700043799787FF1F9387274F9C43D847A16719
:10D98000D107631FF7001743FFFFE7024375328596
:10D9900097000000E780A0FB1743FFFF6700637656
:10D9A00082809787FF1F9387274C9C43D847A167A6
:10D9B000C507631FF7001743FFFFE7024372328575
:10D9C00097000000E780A0F81743FFFF670063732C
:10D9D00082809787FF1F938727499C43D847A16779
:10D9E000B907631FF7001743FFFFE702436F328554
:10D9F00097000000E780A0F51743FFFF6700637002
:10DA000082809787FF1F938727469C43D847A1674B
:10DA1000AD07631FF7001743FFFFE702436C328532
:10DA200097000000E780A0F21743FFFF6700636DD7
:10DA300082809787FF1F938727439C43D847894756
:10DA40006318F7021743FFFFE7026369011132858C
:10DA500032C897F0FFFFE780402EAA85280097F094
:10DA6000FFFFE780A05605611743FFFF670063696A
:10DA700082809787FF1F9387273F9C43D847A167E2
:10DA80008D076311F7041743FFFFE7024365011198
:10DA90003285328497F0FFFFE780202A1306610069
:10DAA000AA844C00228597300000E780C02328001C
:10DAB000A68597F0FFFFE780605105611743FFFFE0
:10DAC0006700236482809787FF1F9387273A9C43D0
:10DAD00081CFDC4391CB1743FFFFE702436082977E
:10DAE0001743FFFF6700E36182801743FFFFE702F0
:10DAF000035F79713C08AE843ED2A165B7070A0086
:10DB00002A843ED448103C08DD053ED636C432C6D1
:10DB10003AC297D0FFFFE780602812474810BA85C5
:10DB200097F0FFFFE780C01332464810B28597F0A8
:10DB3000FFFFE780E014A2464810B68597F0FFFF8C
:10DB4000E7800012501001478146A685228597D0B4
:10DB5000FFFFE780004A45611743FFFF6700635AF4
:10DB60001743FFFFE702A35701117C000329C501FA
:10DB7000AE843ECAA165B70707002A843ECC480898
:10DB80007C00C5053ECE97D0FFFFE780202183456E
:10DB9000D900480897F0FFFFE780800C5008014744
:10DBA0008146A685228597D0FFFFE78080440561E6
:10DBB0001743FFFF6700E3541743FFFFE7022352B9
:10DBC00083C7950093F7F707A384F500970000003B
:10DBD000E78040F91743FFFF6700A3521743FFFF99
:10DBE000E702E34F79713C08AE843ED2A165B707E6
:10DBF00009002A843ED448103C08938545043ED64B
:10DC000032C636C497D0FFFFE7804019A2464810BD
:10DC1000B68597F0FFFFE780A00432464810B28532
:10DC200097F0FFFFE780C005501001478146A685A9
:10DC3000228597D0FFFFE780C03B45611743FFFF78
:10DC40006700234C1743FFFFE702634983C7950032
:10DC500041112A8493F7F707A384F50032852EC675
:10DC600097F0FFFFE780800F85672AC46370F50295
:10DC700097700000E78020E92246B24509ED114780
:10DC80008146228597000000E78060E64101174346
:10DC9000FFFF6700034701478346F501DDB71743E0
:10DCA000FFFFE702234201113C003ECAB7070A000A
:10DCB0003ECC3C003ECE83C79500AA89328593F7BF
:10DCC000F707A384F5002E8497F0FFFFE780000993
:10DCD0008567637DF504A165AA849385850448085A
:10DCE00097D0FFFFE780800B268597700000E780C4
:10DCF00080E12A8929E19145480897F0FFFFE780F4
:10DD000020F6A685480897F0FFFFE78060F7CA85F0
:10DD1000480897F0FFFFE780A0F4014781465008CC
:10DD2000A2854E8597D0FFFFE780A02C05611743A1
:10DD3000FFFF6700633C8145480897F0FFFFE780DD
:10DD400020F20349090275BF1743FFFFE70283373B
:10DD500079711C103ECAB7070F003ECC404D1C1015
:10DD6000AA84AE894808994532C636893ECE97D0F6
:10DD7000FFFFE780A00232464808B28597F0FFFF18
:10DD8000E78000EE630C0902A545480897F0FFFF05
:10DD9000E780C0E62546CA8597200100E78020A4D9
:10DDA000500801478146CE85268597D0FFFFE78042
:10DDB000402445611743FFFF670003348355C402C5
:10DDC000480897F0FFFFE780A0EB0355E402814588
:10DDD00005C5854785456301F502C167FD179305B4
:10DDE000F00F630BF5007D1597700000E780208E23
:10DDF0009305150093F5F50F480897F0FFFFE780AE
:10DE000020E683450403480897F0FFFFE78040E5DC
:10DE100083451403480897F0FFFFE78060E48355CB
:10DE20002403480897F0FFFFE78080E5835544030B
:10DE3000480897F0FFFFE780A0E49DB71743FFFF76
:10DE4000E702E32983C795008146014693F7F70768
:10DE5000A384F50097000000E78040EF1743FFFF21
:10DE60006700232A1743FFFFE702632779713E8487
:10DE70001C103ECA2E89B7070F00A1653ECCFD05D8
:10DE80001C10AA84480842C03AC23ECE36C432C6EC
:10DE900097D0FFFFE78080F032464808B28597F0C0
:10DEA000FFFFE780E0DBA2464808B68597F0FFFF5A
:10DEB000E78000DD12474808BA8597F0FFFFE7804A
:10DEC00020DC0248630C08029145480897F0FFFFE8
:10DED000E780C0D21146A28597200100E7802090FC
:10DEE000500801478146CA85268597D0FFFFE78005
:10DEF000401045611743FFFF6700A320894548088C
:10DF000097F0FFFFE78080CF834704002300F500F0
:10DF100083471400A300F500E1B71743FFFFE702B2
:10DF2000631A83C7950001112A8A93F7F707A38420
:10DF3000F5003285AE8432C697F0FFFFE78000E23D
:10DF400032462A89328597F0FFFFE78000DF856738
:10DF50006373F902AA894A8597700000E780A0BA26
:10DF60002A8419ED114781464A86A6855285970075
:10DF70000000E780C0B705611743FFFF6700C317C4
:10DF80009387E9FF93F7F70F0547E366F7FE8347AB
:10DF9000F50195EB8947E380F9FE8346F40152854C
:10DFA00001474A86A68597000000E78040B4A16734
:10DFB000D90748083ECC230A010002CE9700000092
:10DFC000E780A0B04DBF639EE7008947639EF900DC
:10DFD00093071020231FF50097700000E780C0B75B
:10DFE0006DBF0947E39BE7FA8D47E398F9FA22856D
:10DFF00097700000E78080DF9787FF1F93870706F1
:10E000009C4399E79787FF1F938707EF9C4399C726
:10E0100003D5040097800000E780A0CE231F0400F2
:10E0200022855DBF1743FFFFE702630B01113C0030
:10E030003ECAB7070B003ECC3C003ECE83C79500DE
:10E040002A89328593F7F707A384F500AE8497F009
:10E05000FFFFE780A0D093170501C187635AF00640
:10E06000A1652A849385E502480897D0FFFFE780E1
:10E07000E0D2A285480897F0FFFFE78060C097874D
:10E08000FF1F938767E79C43A9EB01449375F40F47
:10E09000480897F0FFFFE780A0BC9355844093F5B4
:10E0A000F50F480897F0FFFFE78080BB93550441C8
:10E0B00093F5F50F480897F0FFFFE78060BA014736
:10E0C00081465008A6854A8597D0FFFFE78060F219
:10E0D00005611743FFFF6700C3024165854605469A
:10E0E000A2857D1597500000E78060BD59DD510580
:10E0F00097000100E780808F1304400633448502B7
:10E1000071B71743FFFFE70283FD0111B707060050
:10E110003EC683C7950021642A8993F7F707A38435
:10E12000F500AE8428009305A4040AC40AC897D059
:10E13000FFFFE780A0C6300001478146A6854A85DB
:10E1400097D0FFFFE780E0EA97E0FFFFE780000E4F
:10E1500013049404480822CC230A010002CE97003D
:10E160000000E780809605611743FFFF670063F9B1
:10E170001743FFFFE70203F5C1642A890144978929
:10E18000FF1F938929EF130A8002FD1497E0FFFF18
:10E19000E78000BA6347A40001451743FFFF67000B
:10E1A000A3F5B307440303A7C90ABA9703D7070027
:10E1B0006306970083D72700638427010504F9B716
:10E1C0000545E1BF1743FFFFE702C3EF2A8A2E8907
:10E1D00099C123A0050081498144978AFF1F938A32
:10E1E0002AC9614B97E0FFFFE780C0BA63C7A4006C
:10E1F0004E851743FFFF670023F03384640383A732
:10E200000A003E948357040099E763040900232021
:10E2100089008504C1BF4146D2851305440097108B
:10E220000100E780605975F5A289E5B71743FFFF44
:10E23000E70243E939717C083ED4B7070A003ED6AD
:10E240007C083ED883C795002A8A328593F7F70762
:10E25000A384F5002E8932C697F0FFFFE78000B057
:10E2600085676373F5083246AA84328597F0FFFF0D
:10E27000E780A0AC8547AA8963E8A706A1659385D6
:10E280008504281097D0FFFFE78040B1268597705E
:10E290000000E78040872A8429ED9145281097F0F7
:10E2A000FFFFE780E09BA685281097F0FFFFE7803F
:10E2B000209DCE85281097F0FFFFE780609A0147E8
:10E2C00081463010CA85528597D0FFFFE78060D223
:10E2D000A1679387770448183EDC230A010202DE17
:10E2E00097F0FFFFE780607E21611743FFFF670023
:10E2F000A3E08145281097F0FFFFE7806096A68590
:10E30000281097F0FFFFE780A0979787FF1F93875C
:10E31000270D9C4381CB22856389090097D000009B
:10E32000E78040248345040271B797D00000E7805E
:10E33000C022CDBF1743FFFFE702C3D883C79500B4
:10E340004111AA8993F7F707A384F5003285AE84BB
:10E35000328A97F0FFFFE78060A08567637FF50250
:10E360002A8997600000E780007A2A84914631C5A7
:10E370008347F50105476387E70291C70D47636649
:10E38000F704AD461DA89305050303250A00414681
:10E3900097100100E78040420DE941011743FFFF5C
:10E3A000670083D59305950803250A004146971019
:10E3B0000100E7806040814669F54A86A6854E8562
:10E3C00097000000E780C081C9BF83250A001305BC
:10E3D000940897700000E780A02919C1C146F1BFD9
:10E3E0009787FF1F938787C79C4399E79787FF1FEE
:10E3F000938787B09C4399C7228597800000E78068
:10E40000208A69FD8547A30FF400228597B000009C
:10E41000E7806084228597600000E780E0734E8586
:10E4200081464A86A68597F0FFFFE780607BA1675B
:10E430009387570448003EC42302010002C697F0A8
:10E44000FFFFE780806891BF1743FFFFE702A3C685
:10E4500083C795004111AA8993F7F707A384F500B4
:10E4600032852E89B28A97F0FFFFE780208F85677B
:10E470006374F50EAA8497600000E780C0682A8460
:10E480000DED416B014A978BFF1F938BABBE130CB5
:10E49000400E7D1B19A833048A0383A70B0B3E94FF
:10E4A0008357C40163836705050A97E0FFFFE78090
:10E4B0002087E342AAFE95460DA08357C5016396C7
:10E4C00097029305050303A50A0041469710010032
:10E4D000E780802E994611E181462686CA854E85C1
:10E4E00097F0FFFFE780C06F85A883A50A0013059A
:10E4F000040397700000E780A017C14679FD2285CC
:10E50000231E940097A00000E780E07422859760A6
:10E510000000E78060649787FF1F938767EC9C4348
:10E52000A9C323000402228597D00000E78040F0B1
:10E530004E8581462686CA8597F0FFFFE780406AB0
:10E54000A1679387070448003EC42302010002C666
:10E5500097F0FFFFE780605741011743FFFF670017
:10E5600003B989472300F402E1B7397106DE22DCE2
:10E570004AD8800052D456D25AD026DA4ED65ECE31
:10E580002E8A32892A8B97D0FFFFE78060760605B6
:10E59000710541998A8A3301A140232224FC231466
:10E5A00004FC97D0FFFFE780A07483479A0006051C
:10E5B000350593F7F7072315A4FCA304FA004A8551
:10E5C000232624FC97E0FFFFE7804079931705019D
:10E5D000C1876340F0025681130104FCF25062547B
:10E5E000D2544259B259225A925A025BF24B2161DB
:10E5F0008280AA844A8597E0FFFFE7802076AA8977
:10E600004A8597E0FFFFE7806075A1659385C502A5
:10E610002A89130544FC97C0FFFFE78020782685F0
:10E6200097C0FFFFE780606C854511C94A86CE859B
:10E6300097C0FFFFE780E065AA8B21E989451305B4
:10E6400044FC97E0FFFFE780A061A685130544FC2A
:10E6500097E0FFFFE780C062CE85130544FC97E09A
:10E66000FFFFE780E061CA85130544FC97E0FFFFE8
:10E67000E780006101478146130644FCD2855A8534
:10E6800097D0FFFFE780E096B9B78145130544FCBA
:10E6900097E0FFFFE780C05CA685130544FC97E088
:10E6A000FFFFE780E05DCE85130544FC97E0FFFFA8
:10E6B000E780005DCA85130544FC97E0FFFFE78013
:10E6C000205C814497D0FFFFE7808062E3D4A4FA06
:10E6D00083A70B0113971400BA9783D5070099C538
:10E6E000130544FC97E0FFFFE78080598504D9BFFC
:10E6F000797106D622D44AD000184ECE52CC56CAD2
:10E7000026D25AC8AE893289AA8A97D0FFFFE780FD
:10E71000205E0605690541990A8A3301A140232A32
:10E7200024FC231C04FC97D0FFFFE780605C83C7B8
:10E73000990006052D0593F7F707231DA4FCA38474
:10E74000F9004A85232E24FC97E0FFFFE780006153
:10E7500093170501C187634FF0005281130104FD37
:10E76000B250225492540259F249624AD24A424B60
:10E7700045618280AA844A8597E0FFFFE780005EBA
:10E78000A1659385A5022A89130544FD97C0FFFF63
:10E79000E780C060268597C0FFFFE780005585456C
:10E7A00009C9CA8597C0FFFFE780A0512A8B29E1DC
:10E7B0008945130544FD97E0FFFFE780604AA68581
:10E7C000130544FD97E0FFFFE780804BCA851305E2
:10E7D00044FD97E0FFFFE780A04A0147814613060A
:10E7E00044FDCE85568597D0FFFFE7808080B5B782
:10E7F0008145130544FD97E0FFFFE7806046A6854D
:10E80000130544FD97E0FFFFE7808047CA851305A5
:10E8100044FD97E0FFFFE780A046814497D0FFFFCB
:10E82000E780004DE3DBA4FA83270B011397140064
:10E83000BA9783D5070099C5130544FD97E0FFFFFC
:10E84000E78000448504D9BF1743FFFFE70223890F
:10E8500083474500404DD5EFFD575DC48346940086
:10E8600009476363D70A0346B400854663EEC608CA
:10E870008306E40063CA06085C45F9562390D70076
:10E880009777FF1F83C7075F99E3A304E400977797
:10E89000FF1F938767669C4381E78947A306F400BF
:10E8A0009787FF1F9387C7B39C4381E78947230658
:10E8B000F4009705000093854506AA84130504011A
:10E8C00097F00000E7802010FD57231AF4028147DB
:10E8D0001CDC01489777FF1F23AA87589777FF1FF3
:10E8E00093870759232E040304C0804397D0FFFF6A
:10E8F000E780404A61463306C5028145228597403C
:10E90000FFFFE780C08081473E851733FFFF670028
:10E91000437FFD57D5BF1733FFFFE702437C2A84AF
:10E920000355450297600000E780E01D19E5231EAE
:10E9300004001733FFFF6700C37C8357E401F5DB56
:10E94000930504FF174501001305450497E00000F7
:10E95000E780E014F9BF1733FFFFE70243782E8901
:10E96000A16541119385E5032A8436C432C6BE846D
:10E970003AC297C0FFFFE780604212472285BA85FE
:10E9800097E0FFFFE780C02D32462285B28597E0F1
:10E99000FFFFE780E02EA2462285B68597E0FFFFC5
:10E9A000E780002E630309029145228597E0FFFF6F
:10E9B000E780C0241146A68597100100E78020E279
:10E9C00041011733FFFF6700C3738945228597E034
:10E9D000FFFFE780A02283C704002300F50083C760
:10E9E0001400A300F500E9BF1733FFFFE702236F10
:10E9F00083C79500444D054793F7F707A384F500B7
:10EA00001C42411183C707006367F7062E842A89D9
:10EA1000B1C003C7D400630FF7021777FF1F1307B6
:10EA2000A74D184305C3A386F40097A00000E78014
:10EA3000404A83C7D40099E741657D15974000009F
:10EA4000E780403083D72403918B89C797E000008B
:10EA5000E780C0134A85A28597F0FFFFE78080100A
:10EA6000A167C10748003EC42302010002C697F017
:10EA7000FFFFE780800541011733FFFF67006368F0
:10EA80001733FFFFE702A36503D745008D47AA842C
:10EA900041112E8432892E8563E3E70297E0FFFF60
:10EAA000E780C02BAA8523000900268597C0FFFFB9
:10EAB000E780202141011733FFFF6700836497E05F
:10EAC000FFFFE780A0292AC6228597E0FFFFE780A5
:10EAD000E028B24585472A862300F900268597C09D
:10EAE000FFFFE780001BF9B7397106DE22DC26DA6A
:10EAF00080004ED652D456D24AD85AD05ECEAE8975
:10EB0000B284AA8A97D0FFFFE780801D060513050F
:10EB1000250241990A8A3301A140232224FC2314AF
:10EB200004FC97D0FFFFE780A01B83C79900060570
:10EB30004D0593F7F7072315A4FCA384F900268558
:10EB4000232624FC97E0FFFFE7804021931705016F
:10EB5000C1876340F0025281130104FCF2506254F9
:10EB6000D2544259B259225A925A025BF24B216155
:10EB70008280AA8B03AB040097C0FFFFE780E016FA
:10EB800051E583D7440001498544F11793B7170035
:10EB9000A301F4FC834734FCA165C9C79385E50450
:10EBA000130544FC97C0FFFFE780401FA6851305AF
:10EBB00044FC97E0FFFFE780A00ADE85130544FCD4
:10EBC00097E0FFFFE780C00B834734FC114691E3D9
:10EBD0000946DA85130544FC97E0FFFFE7806005EE
:10EBE0008144630A0900416B7D1B97D0FFFFE780DA
:10EBF000200F63CCA40201478146130644FCCE8556
:10EC0000568597C0FFFFE780C03EB1B7A6851306C3
:10EC100034FC97000000E780E0E6933415002A8971
:10EC200086048DBF9385C504A5BF8327C9001397AC
:10EC30001400BA9783D5070063886501130544FC67
:10EC400097E0FFFFE780C003850445B71733FFFF58
:10EC5000E702634679711C103EC4B7070F003EC639
:10EC60001C103EC883C79500AA8A328593F7F70720
:10EC7000A384F500AE89328497E0FFFFE780000EA1
:10EC800093170501C187635AF0062A8A228597E007
:10EC9000FFFFE780A00C2A895285032B040097C050
:10ECA000FFFFE780800439ED835744008144054429
:10ECB000F11793B71700A303F10083457100DA87BA
:10ECC0002287CA865286280097000000E780E0C8A5
:10ECD000014781463000CE85568597C0FFFFE7800B
:10ECE0004031A1679387D70348083ECC230A8100AF
:10ECF00026CE97F0FFFFE78040DD45611733FFFF29
:10ED00006700E33EA2851306710097000000E780CC
:10ED100060D7AA84094455D13544E30055FB4A85A0
:10ED200097F0FFFFE78000450D4441D9014497D09B
:10ED3000FFFFE780E0FA634DA400C16B0144FD1BB7
:10ED400097D0FFFFE780C0F9634EA4001544B5B724
:10ED5000DC4413171400BA9783D707006383270393
:10ED60000504F1B7D84493171400BA9703D70700E6
:10ED7000631B770123902701268597A00000E78079
:10ED800080DB01441DBF050465BF1733FFFFE702A9
:10ED9000633383C7950041112A8A93F7F707A38449
:10EDA000F50032852E89328497E0FFFFE78000FB73
:10EDB00093170501C1876353F006AA89228597E05E
:10EDC000FFFFE780A0F92311A1004E85832A0400EC
:10EDD00097C0FFFFE78060F139E583574400854421
:10EDE0000144F11793B71700A300F1000348110085
:10EDF00003572100D6875285CE862686CA8597F08E
:10EE0000FFFFE7806006A167F10748003EC42302C8
:10EE1000910022C697F0FFFFE78020CB4101173316
:10EE2000FFFF6700632DA285130611009700000005
:10EE3000E78040C52A84894455D98357210011674A
:10EE40008544BA97C2071167C1831307F7EFE36FD1
:10EE5000F7F89777FF1F938767209C4381CB854501
:10EE60001305210097500000E7802075835521008D
:10EE70002285814497C0FFFFE780C0DD25D923109C
:10EE80000500228597A00000E78040CD85B71733A5
:10EE9000FFFFE702432283C7950041112A8B93F7B6
:10EEA000F707A384F50032852E8A328497E0FFFFAE
:10EEB000E780C0EA93170501C1876351F006AA8A6B
:10EEC000228597E0FFFFE78060E92A895685832B3A
:10EED000040097C0FFFFE78040E131E5835744001D
:10EEE00081440544F11793B71700A301F1000348CB
:10EEF0003100DE875A854A87D6862286D28597F0EA
:10EF0000FFFFE78060F6A167ED0748003EC42302DB
:10EF1000810026C697F0FFFFE78020BB4101173331
:10EF2000FFFF6700C31CA285130631009700000095
:10EF3000E78040B5AA8409445DD99167CA97C207A2
:10EF40001167C1831307F7EF0544E362F7FACA8537
:10EF500097C0FFFFE78000D0014451F9814997D065
:10EF6000FFFFE780E0D863DBA9009848939719007A
:10EF7000BA9703D7070005EF2390270197D0FFFF2B
:10EF8000E78000D71544E384A9F6268597A0000002
:10EF9000E780C0BC9777FF1F9387470C9C430144D1
:10EFA000B9D74A8597500000E780C05889B78509CE
:10EFB0007DB71733FFFFE702E31079713E847C08C9
:10EFC0003EC82E8AB7071400A1653ECAE5057C0835
:10EFD000AA89080836C4428932C6BA8AC6843ECC99
:10EFE00097C0FFFFE78080DBCA85080897E0FFFF36
:10EFF000E78000C732460808B28597E0FFFFE78048
:10F0000020C8A246630A09049D45080897E0FFFF4F
:10F01000E780C0BE1D4681459730FFFFE780200F87
:10F0200063890A089145080897E0FFFFE78000BD63
:10F030001146A68597000100E780607A1008014715
:10F040008146D2854E8597C0FFFFE78080FA4561F3
:10F050001733FFFF6700430AB685080897E0FFFFF4
:10F06000E78000C21C400808D8439355C701858932
:10F0700012075183B205D98D97E0FFFFE78040C0AA
:10F080001C40080883C5870097E0FFFFE78040BD6C
:10F090001C40080883C5A70097E0FFFFE78040BC3D
:10F0A0001C40080883C5970097E0FFFFE78040BB3E
:10F0B00085BF8945080897E0FFFFE78020B483C734
:10F0C00004002300F50083C71400A300F500BDB7BA
:10F0D0001733FFFFE70203FF83C795004111AA8999
:10F0E00093F7F707A384F5003285AE84328497E066
:10F0F000FFFFE780A0C693170501C187635DF00499
:10F100002A89032A040097C0FFFFE78000BE19E99F
:10F11000835744000548F11793B71700A307F10080
:10F12000814631A81306F100A28597000000E78010
:10F1300060951DC51C459DC783D647000148034700
:10F14000F10093078500D2884A86A6854E859700F0
:10F150000000E78040E641011733FFFF6700C3F975
:10F1600009487DBF1D486DBF1733FFFFE70283F5D8
:10F1700065715C083EC4B7077B013EC65C083EC8AB
:10F1800083C795002A8A328593F7F707A384F50091
:10F19000AE8997E0FFFFE78040BA8357E100E1C7FF
:10F1A0008945280097C0FFFFE78040BF81452800C0
:10F1B00097E0FFFFE780C0AA97C0FFFFE78020C568
:10F1C0009777FF1F9387C7219C431774FF1F034442
:10F1D00064CAAA843334800099C3136424009777E7
:10F1E000FF1F938767D19C4399C3136444009777AB
:10F1F000FF1F9387A7E69C4399C31364840083D5BC
:10F2000004002800014997E0FFFFE78060A783D54D
:10F210002400280097E0FFFFE78080A683D5440004
:10F22000280097E0FFFFE780A0A597D0FFFFE780C9
:10F2300020A793150501C181280097E0FFFFE78013
:10F2400020A4A285280097E0FFFFE78060A39C44EC
:10F250006360F902014781463000CE85528597C030
:10F26000FFFFE78000D959611733FFFF6700C3E84C
:10F27000DC441314490028003E9497E0FFFFE78028
:10F280006096834744000347540089070607BA97EE
:10F290008607E36AF5FC835524002800814A97E03D
:10F2A000FFFFE780E09D83454400280097E0FFFFD3
:10F2B000E780009B83455400280097E0FFFFE7802C
:10F2C000209A8347440063C9FA00814A8347540067
:10F2D00063C1FA020509A5BF1C4413975A00280010
:10F2E000BA9783D50700850A97E0FFFFE78040992A
:10F2F000C9BF032BC40093975A0028003E9B835537
:10F300002B00850A97E0FFFFE780809783550B006D
:10F31000280097E0FFFFE780A0964DBF1733FFFF5F
:10F32000E702E3DB5C4993E717005CC997A00000A4
:10F33000E78020B61733FFFF6700A3DC1733FFFF1A
:10F34000E702E3D92E84814597F0FFFFE780C0E70D
:10F3500005C583570500FD172310F50009C4835721
:10F3600025002310F40097000000E78060FB0145B2
:10F370001733FFFF6700E3D831457DD82310040021
:10F38000C5BF1733FFFFE702E3D383C795004111E1
:10F390002A8A93F7F707A384F50032852E893284F1
:10F3A00097E0FFFFE780809B93170501C1876356B5
:10F3B000F006AA89C145228597E0FFFFE780A0807B
:10F3C0002A8B4E85832A040097C0FFFFE780E091D7
:10F3D00031E983574400231101000544F11793B725
:10F3E0001700A300F10081440348110003572100D6
:10F3F000D6875285CE862286CA8597F0FFFFE780A2
:10F40000A0A6A1679387170248003EC4230281008B
:10F4100026C697E0FFFFE780406B41011733FFFFEF
:10F42000670083CD13061100A28597F0FFFFE780E8
:10F430006065AA8409E523110100094475B79305A5
:10F4400021005A8597000000E78080EF8357210054
:10F450002A84D9DB9777FF1F938747C09C4381CBD2
:10F4600085451305210097500000E780001583555E
:10F4700021002685314497B0FFFFE780A07D2DD580
:10F4800023100500268597900000E780206D014439
:10F49000A1BF1733FFFFE70283C441112E896C001F
:10F4A000AA8402C697F0FFFFE78000D20DC1035780
:10F4B000050005072310E50097000000E78040E6FF
:10F4C00081473E8541011733FFFF670083C3324701
:10F4D000954765DBCA85268597300000E780400D9B
:10F4E000C147E34005FE3244854741462310F400FE
:10F4F00083570900A685130544002311F4009700E3
:10F500000100E780C02D228545BF1733FFFFE702CA
:10F5100063BB83C795004111AA8A93F7F707A384B9
:10F52000F5003285AE89328497E0FFFFE7800083E3
:10F5300093170501C1876356F0062A8AC1452285C3
:10F5400097D0FFFFE7802068AA845285032B040030
:10F5500097B0FFFFE780607931E9835744002311BA
:10F5600001008544F11793B71700A300F10001448F
:10F570000348110003572100DA875685D286268674
:10F58000CE8597F0FFFFE780208EA1679387070263
:10F5900048003EC42302910022C697E0FFFFE780A7
:10F5A000C05241011733FFFF670003B5A285130660
:10F5B000110097F0FFFFE780E04C2A8409E5231152
:10F5C0000100894475B72685930521009700000046
:10F5D000E78060ECAA8449FD83552100228597B01D
:10F5E000FFFFE780206749F5014997C0FFFFE780EB
:10F5F0002070635DA900184893171900BA9703D7C4
:10F6000007000DEF035721002390E70097C0FFFF8D
:10F61000E780006E630625039777FF1F938707A493
:10F620009C4399C70355210097500000E78080F064
:10F63000228597900000E78060521DBF050975B7CD
:10F6400095443DB705C19307F00F630FF500C5471B
:10F65000630CF5009307F5FF05453315F5004205EA
:10F66000418182800145828041657D158280B9E9B2
:10F670001733FFFFE702A3A6034506033284970072
:10F680000000E78060FC9305803EB305B502C2052B
:10F69000C18181CD0357E402854763F8E700130574
:10F6A000040197E00000E78020428357E4024167AD
:10F6B0007D176385E700FD172317F4021733FFFF5B
:10F6C000670023A482801733FFFFE702C39E004236
:10F6D00083C79500444D0349140093F7F707A384AB
:10F6E000F50083470400220911673369F900A16717
:10F6F000B347F90041112A8BAE8A63ECE70E8347CA
:10F7000024001307C00EB91793F7F70F6373F710B0
:10F7100003473400C14763EEE70E834744001307F5
:10F72000E00793C707086371F70C83498400834798
:10F730007400A209B3E9F900856763F7F90A034A7F
:10F740006400834754004E85220A336AFA009750BA
:10F750000000E780403B61C123962403834B3400C3
:10F76000137AFA00239A34032388740323994403F9
:10F7700093890401631C090023A604022398040250
:10F780004E8597E00000E78060363DA003492400E5
:10F790004A8597000000E78020EB2397A402834767
:10F7A00044004E85A388F402E38D0BFCE30B09FCB7
:10F7B00097E00000E780202F97900000E78000731B
:10F7C00081460146D6855A8597E0FFFFE7800058BD
:10F7D000A167938797033EC423020100480002C635
:10F7E00097E0FFFFE780602E41011733FFFF6700BE
:10F7F00003908544A2862686D6855A8597E0FFFF2A
:10F80000E780C054A167938797033EC42302910009
:10F81000F1B7BD44C5B79144F1BF1733FFFFE7020D
:10F82000638A01111C08404D3EC2B7070F003EC459
:10F830001C083EC62A89AE8997C0FFFFE78020D307
:10F84000585C1C5C6346B70E6394E50063E2A70E48
:10F850003385A740B3B7A700B305B7401306803E72
:10F8600081469D8D97000100E78080B793140501C4
:10F87000C180A1659385C503480097B0FFFFE7806D
:10F88000E0518145480097D0FFFFE780603D8355F8
:10F890000404480097D0FFFFE780803E835524048E
:10F8A000480097D0FFFFE780A03D814589CCC16724
:10F8B000FD179305F00F6388F4002685975000002C
:10F8C000E780E0E0AA85480097D0FFFFE780403955
:10F8D00003554404814501CDC167FD179305F00F21
:10F8E0006307F50097500000E78060DEAA854800B6
:10F8F00097D0FFFFE780C03683456404480097D067
:10F90000FFFFE780E03583457404480097D0FFFF90
:10F91000E7800035500001478146CE854A8597B083
:10F92000FFFFE780006D05611723FFFF6700C37CC1
:10F93000814481B71723FFFFE702637A83C79500ED
:10F9400093F7F707A384F50097000000E78020ED08
:10F950001723FFFF6700E37A1723FFFFE702837691
:10F9600083C795004111404D93F7F707A384F50035
:10F970002A8A3285B284AE8997D0FFFFE780003EA5
:10F980002A8B268597D0FFFFE780403D2A89268570
:10F9900097D0FFFFE780603A93170B0163CA070215
:10F9A000E177CA97C207C183116763E3E702930750
:10F9B0000910C207C1831307B00F637BF7009317C9
:10F9C0000901C187AA8A634AF000C54763FE57014F
:10F9D00041011723FFFF6700237297B0FFFFE78005
:10F9E0004021E31725FFD5B763080B026306090220
:10F9F000814463890A02B7077F002310640523113D
:10FA000024057CC0568597000000E780E0C393047E
:10FA1000803EB304950239A0B7077F002320040479
:10FA20007CC081440355240497E00000E780A0A334
:10FA3000A1C497C0FFFFE78080B3269593D7F44118
:10FA400033379500AE97BA9708DC5CDCCE855285DB
:10FA500097000000E780A0DC99E023220404A1675E
:10FA60009387B70348003EC42302010002C697E013
:10FA7000FFFFE7808005A9BF814701481CDC232EDA
:10FA80000403E9B71723FFFFE702636597C0FFFF91
:10FA9000E7804030E1473305F5029145975000007B
:10FAA000E78000C5E55711C59767FF1F23A2A73C54
:10FAB00081473E851723FFFF6700A36485471767CB
:10FAC000FF1F2309F73A82801723FFFFE702236114
:10FAD0009767FF1F9387873980433DC0835704048E
:10FAE0006390A70683572404639CB7043689B284C5
:10FAF00097C0FFFFE780A0A75C5C63C3B704639572
:10FB0000B7001C5C63EEA7028347640463F3F40050
:10FB1000A6872303F4048347740463F39700A6873E
:10FB2000A303F4048357440441677D176385E7000A
:10FB300085072312F4043C4481C7CA852685829731
:10FB40001723FFFF6700E35B9767FF1F9387073269
:10FB50009C43014599C303C5870082801723FFFF9B
:10FB6000E702E3570111B70707003EC683C79500B8
:10FB7000584D0AC493F7F7070AC8A384F5002A89E9
:10FB8000AE8411CB1C4283C707002304F700979073
:10FB90000000E7800034216493055402280097B0E8
:10FBA000FFFFE780A01F97000000E78020FAAA85EA
:10FBB000280097D0FFFFE780A00A30000147814668
:10FBC000A6854A8597B0FFFFE780A0421304440250
:10FBD000480822CC230A010002CE97E0FFFFE7800D
:10FBE000C0EE05611723FFFF6700A3511723FFFF36
:10FBF000E702E34E01117C003ECAB70707003ECC86
:10FC00007C003ECE83C795002E84AA8493F7F70725
:10FC1000A384F500A16593855502480897B0FFFFBE
:10FC2000E780C01797000000E78040F2AA854808E7
:10FC300097D0FFFFE780C002500801478146A285A8
:10FC4000268597B0FFFFE780C03A05611723FFFFC5
:10FC50006700234B9767FF1F938747219C43094504
:10FC600099C303C5970082809767FF1F938707207A
:10FC70009C43094599C303C5D70082809767FF1F3E
:10FC80009387C71E9C43014599C303C5A700828083
:10FC90001723FFFFE70203430111B70708003EC621
:10FCA00083C79500404D0AC493F7F7070AC8A38499
:10FCB000F5002A89AE8429C41442854703C706008B
:10FCC00063E0E70A83479400094681496380C702DD
:10FCD000B307F740A304E400B339F00083C716006C
:10FCE0002305F40097900000E780A01E035724032B
:10FCF000058B19C76386090097D00000E78000E9EB
:10FD0000216493058402280097B0FFFFE780000973
:10FD100097000000E78040F4AA85280097D0FFFFF5
:10FD2000E78000F497000000E78080F5AA852800AE
:10FD300097D0FFFFE780C0F2014781463000A685DB
:10FD40004A8597B0FFFFE780C02A13047402480871
:10FD500022CC230A010002CE97E0FFFFE780E0D625
:10FD600005611723FFFF670023391723FFFFE70211
:10FD7000033701117C003ECAB70708003ECC7C0067
:10FD80003ECE83C795002E84AA8493F7F707A384F9
:10FD9000F500A16593858502480897B0FFFFE780CD
:10FDA000E0FF97000000E78020EBAA85480897D085
:10FDB000FFFFE780E0EA97000000E78060ECAA859B
:10FDC000480897D0FFFFE780A0E950080147814627
:10FDD000A285268597B0FFFFE780A0210561172344
:10FDE000FFFF670003329767FF1F938727089C4335
:10FDF000014599C303C5B70082801723FFFFE702BF
:10FE0000032E0111B70707003EC683C79500404D7A
:10FE10000AC493F7F7070AC8A384F5002A89AE84B9
:10FE200005C81C42054783C707006368F7060347F8
:10FE3000B400630FF700A305F40097900000E7807B
:10FE400040098347B400B9CF97D0FFFFE78040BE99
:10FE500021649305B400280097B0FFFFE78000F409
:10FE600097000000E78060F8AA85280097D0FFFF80
:10FE7000E78000DF014781463000A6854A8597B0BC
:10FE8000FFFFE78000172904480822CC230A01005D
:10FE900002CE97E0FFFFE78040C305611723FFFF15
:10FEA0006700232697D0FFFFE78020BF55B71723B1
:10FEB000FFFFE702C32201117C003ECAB70707001B
:10FEC0003ECC7C003ECE83C795002E84AA8493F757
:10FED000F707A384F500A165AD05480897B0FFFFBB
:10FEE000E780C0EB97000000E78020F0AA85480873
:10FEF00097D0FFFFE780C0D6500801478146A28512
:10FF0000268597B0FFFFE780C00E05611723FFFF2E
:10FF10006700231F9767FF1F938747F59C43094599
:10FF200099C303C5C70082801723FFFFE702231B85
:10FF300001117C00AE843ECAA165B70707002A8480
:10FF40003ECCD1057C0048083ECE97B0FFFFE7804D
:10FF5000E0E497000000E78020FCAA85480897D0DD
:10FF6000FFFFE780E0CF500801478146A685228544
:10FF700097B0FFFFE780E00705611723FFFF6700E9
:10FF800043181723FFFFE702831583C7950093F7F4
:10FF9000F707A384F50097000000E78020F91723F6
:10FFA000FFFF670003161723FFFFE702A31183C7B4
:10FFB00095000329C501411193F7F707A384F500C4
:10FFC0001C4283C90700854763E637079767FF1F11
:10FFD000938707419C432E84AA8485CF9700000015
:10FFE000E78080F389476306F502630409028347CB
:10FFF000C900638037032306390197900000E7802A
:020000040001F9
:1000000040ED83572903898B89C797D00000E7808B
:10001000E0B72685A28597000000E78020F1A16760
:10002000CD0748003EC42302010002C697E0FFFF4F
:10003000E780A0A941011723FFFF6700E30B976743
:10004000FF1F9387A7E29C431D4599C303C5E700A3
:1000500082801723FFFFE70283080111B70707001B
:100060003EC683C79500584D0AC493F7F7070AC8E0
:10007000A384F5002A89AE8415C71C4283C70700F4
:1000800093968701E18663C4060685466381D70699
:100090008346E7006388F6002307F7009790000087
:1000A000E78020E321649305E400280097B0FFFF78
:1000B000E780C0CE97000000E780A0F8AA8528005E
:1000C00097D0FFFFE780C0B9014781463000A68581
:1000D0004A8597B0FFFFE780C0F13504480822CC7D
:1000E000230A010002CE97E0FFFFE780009E056132
:1000F0001723FFFF6700E3001723FFFFE70223FE3C
:1001000001117C003ECAB70707003ECC7C003ECE02
:1001100083C795002E84AA8493F7F707A384F5007C
:10012000A165B905480897B0FFFFE78020C7970091
:100130000000E78000F1AA85480897D0FFFFE7801C
:1001400020B2500801478146A285268597B0FFFF5F
:10015000E78020EA05611723FFFF670083FA172372
:10016000FFFFE70223F6AA8401441769FF1F130962
:1001700029D0E14997C0FFFFE780C0C16344A400D4
:10018000014519A833053403832709003E95835799
:1001900025006397970011051723FFFF6700C3F53C
:1001A0000504C9BF032E8500630A0E121763FF1FE3
:1001B0001303C3EA03230300631503002943639079
:1001C000061203234E01631503001D4363990710B4
:1001D0001723FFFFE70223EEC689428A3E89BA8AC7
:1001E000B684328BAE8B2A84B5E103554E0019E5F7
:1001F00001431A851723FFFF670063EFA167A98FEB
:10020000116763FBE70097000000E78080F58145F8
:1002100097F0FFFFE780C0120844B70700E058419D
:10022000F98F18455CC1B707001FF98F1CC55C49E1
:1002300091C7610597E00000E780408BE38A09FAE7
:10024000228597900000E78060C65DB7328597C031
:100250000000E78040430D4349DD1C44116703D58E
:100260004700A167A98F63FBE70097000000E780C4
:1002700040EF814597F0FFFFE780800C0323840067
:1002800093164B01D1828347B300035663008588E0
:10029000FD8BA305F300FD777D8E558EFD76FD1653
:1002A000B204F18E83274301C58E231273012313F9
:1002B000D3002304530123052301A3044301BDDF1D
:1002C000228597B0FFFFE780A0C5AA850844B5D175
:1002D000610597D00000E780207F8DB71D431A8508
:1002E00082801723FFFFE702E3DD0569AA84AE8958
:1002F000328A0144FD5A7D1997C0FFFFE780409E76
:100300006347A40001451723FFFF6700E3DED844DD
:1003100093171400BA9703D70700631F370323907E
:10032000570163070A00268597900000E780A080A8
:100330009C449DC383D76700B3F72701639E3701B1
:10034000D28801488147014781460146814526857B
:1003500097000000E78040E5050479BF1723FFFF01
:10036000E70243D679711C103EC4B7070F003EC6A2
:100370001C103EC883C79500AA8A328593F7F707F9
:10038000A384F5002E89328497D0FFFFE780009D7B
:1003900093170501C187635AF006AA89228597D071
:1003A000FFFFE780A09B2A8A4E85032B040097B0AD
:1003B000FFFFE780809339ED835744008144054473
:1003C000F11793B71700A303F10083457100DA8793
:1003D0002287D2864E86280097E0FFFFE780E0570D
:1003E000014781463000CA85568597B0FFFFE780F8
:1003F00040C0A1679387F70348083ECC230A8100D9
:1004000026CE97D0FFFFE780406C45611723FFFFA2
:10041000670083CEA2851306710097E0FFFFE78097
:100420006066AA84094455D1528597E0FFFFE780B2
:1004300060D40D4459D90546D28526859700000021
:10044000E78060EA2A8451B71723FFFFE70223C938
:10045000835507000346270041112A842E8532C6A2
:100460002EC497E0FFFFE780E0D001C93246A245E5
:10047000228597000000E78000E741011723FFFF76
:10048000670023C81723FFFFE702E3C283C7950075
:100490004111AA8A93F7F707A384F5003285AE8944
:1004A000328497D0FFFFE780608B93170501C187E7
:1004B0006357F00AC1452A8A228597C0FFFFE7806B
:1004C00080702A8D228597D0FFFFE78020892A89B6
:1004D000228597D0FFFFE7804086930705F893F7C2
:1004E000F70F1307E007AA8B637BF706228597D0E7
:1004F000FFFFE78080842A8C228597D0FFFFE7806A
:10050000C083AA8C5285032B040097A0FFFFE780CD
:10051000C07D39E983574400231101008144F1175C
:1005200093B71700A300F100054403471100835659
:100530002100938784005685DA8822885286CE85EA
:1005400097F0FFFFE78020A7A167E90748003EC4B6
:100550002302810026C697D0FFFFE78000574101A4
:100560001723FFFF6700A3B813061100A28597E0C9
:10057000FFFFE7802051AA8409E523110100094407
:100580006DB7930521006A8597F0FFFFE780A0F023
:100590002A8441FD835521009356C9001316490151
:1005A00085486688E2875E87858A5182268597001E
:1005B0000000E78060BF2A848DBF1723FFFFE7029A
:1005C00083AF83C7950041112A8B93F7F707A38464
:1005D000F5003285AE89328497C0FFFFE78000784E
:1005E00093170501C1876352F00A2A8A228597C0B2
:1005F000FFFFE780A076AA8A228597C0FFFFE780E9
:10060000E0752A89228597C0FFFFE7800073930772
:1006100005F893F7F70F1307E0072A8C6377F706BF
:10062000228597C0FFFFE7804071AA8C228597C082
:10063000FFFFE78080702A8D5285832B040097A0EE
:10064000FFFFE780806A39E5835744008544014411
:10065000F11793B71700A301F10003473100930787
:1006600084005A85DE882688D6865286CE8597F005
:10067000FFFFE78040948D4748003EC4230291006D
:1006800022C697D0FFFFE780404441011723FFFFB8
:100690006700E3A5A2851306310097E0FFFFE7801E
:1006A000603E2A84894455D99356C90013164901DE
:1006B00085486A88E6876287858A5182D685970051
:1006C0000000E78060AEAA8449BF1723FFFFE7025E
:1006D000639F2A8981440144617A916A176BFF1FE5
:1006E000130BCB9797B0FFFFE780806063C7A40030
:1006F00022851723FFFF670023A083270900939912
:100700001400CE9703D50700330745014207418304
:100710006364570305C103270B0019C785453E8550
:1007200097400000E78060E9832709000504CE9721
:100730002390070085047DB797000000E78060A242
:10074000832709000504CE972390070065D58145CE
:1007500097F0FFFFE780C0BEF1BF1723FFFFE7025E
:10076000639683C7950041112A8A93F7F707A384FC
:10077000F50032852E89328497C0FFFFE780005E46
:1007800093170501C187635AF004AA89832A0400DC
:1007900097A0FFFFE780605531E58357440085440B
:1007A0000144F11793B71700A301F100034831008A
:1007B000D68752850147CE862686CA8597D0FFFF09
:1007C000E780806AA167F50748003EC423029100D4
:1007D00022C697D0FFFFE780402F41011723FFFF7C
:1007E00067008391A2851306310097E0FFFFE78041
:1007F00060292A8489445DD99767FF1F93870786FC
:100800009C4381CF044997B0FFFFE780604EAA85E3
:10081000268597400000E78040DA13050401970021
:100820000000E780C0EA228597800000E78000335F
:100830008144ADBF1723FFFFE702E38783C795001D
:100840004111AA8A93F7F707A384F5003285AE8990
:1008500032842311010097C0FFFFE78020509317D7
:100860000501C1876354F0062A8AC145228597C0D5
:10087000FFFFE7804035AA8B5285032B040097A029
:10088000FFFFE780804621E9835744008544014407
:10089000F11793B71700A300F100034811000357A5
:1008A0002100DA875685D2862686CE8597D0FFFF2F
:1008B000E780805BA1679387270248003EC423023C
:1008C000910022C697D0FFFFE78020204101172327
:1008D000FFFF6700C381A2851306110097E0FFFFA9
:1008E000E780401A2A8489444DD99757FF1F938780
:1008F000E77698433E8901CF044997B0FFFFE78030
:10090000203FAA85268597400000E78000CB13058D
:10091000040197000000E78080DB97B0FFFFE780CD
:10092000203D95443DD9930521005E8597F0FFFF5A
:10093000E78060B6AA8435F11C4803572100228560
:100940002390E70097800000E7804021832709007B
:10095000A9D70355210097400000E780A0BD35BF0F
:100960001713FFFFE702237583C795004111AA8A79
:1009700093F7F707A384F5003285AE89328497C0D8
:10098000FFFFE780A03D93170501C1876351F00683
:100990002A8A228597C0FFFFE780403C2A8952853A
:1009A000032B040097A0FFFFE780203431E5835735
:1009B000440085440144F11793B71700A301F100E7
:1009C00003483100DA8756854A87D2862686CE8547
:1009D00097D0FFFFE7804049A167F90748003EC470
:1009E0002302910022C697D0FFFFE780000E41014D
:1009F0001713FFFF6700A36FA2851306310097E06E
:100A0000FFFFE78020082A8489445DD99167CA974F
:100A1000C2071167C1831307F7EF8544E362F7FA52
:100A20009757FF1F938787639843BE8B01CF044975
:100A300097B0FFFFE780C02BAA852685974000006E
:100A4000E780A0B71305040197000000E78020C8E5
:100A500097B0FFFFE780C02995443DD11C4822850F
:100A600081442390270197800000E780200F83A70F
:100A70000B00B9D74A8597400000E780A0AB89B743
:100A80001713FFFFE702A3652A844105B28497008C
:100A90000000E780C0C311C5228597800000E78071
:100AA000E00B81460146A685228597800000E780FD
:100AB000C04E1C4C89C7DC4799C322858297171307
:100AC000FFFF670003649757FF1F9387273A9C43F4
:100AD000014599C31385070182809757FF1F9387AC
:100AE000E738884382801713FFFFE702435F9317BD
:100AF000C600DD8DC2054111C1812A8432C697C06E
:100B0000FFFFE780E0173246228511829375F60FCA
:100B100097C0FFFFE780C01441011713FFFF670074
:100B2000435E1713FFFFE702E35979713C083ED299
:100B3000B7070C003ED43C083ED683C79500AE8470
:100B40002A8993F7F707A384F500A16593853504F7
:100B5000481097A0FFFFE7806024C165FD150144A0
:100B6000175AFF1F130A0A51930A400EAE892E8BA3
:100B70002EC697B0FFFFE780A01A42059317040125
:100B80004181C183B24563E9A702C167FD1763874D
:100B9000F500481097C0FFFFE780800E5010014716
:100BA0008146A6854A8597A0FFFFE780804445617E
:100BB0001713FFFF670043543307540383270A0BBF
:100BC000BA9703D6C701630A3601638A3501481014
:100BD00097000000E78060F1DA85050451BFB28517
:100BE000EDBF1713FFFFE702034D79717C083EC884
:100BF000B70711003ECA7C083ECC83C79500AA897E
:100C0000328593F7F707A384F5002E8997C0FFFF7D
:100C1000E780C01485676378F504A165AA84890517
:100C2000080897A0FFFFE78060172685974000001F
:100C3000E78060ED133415000A04A285080897C008
:100C4000FFFFE780E001A685080897C0FFFFE78067
:100C5000200325CC014781461008CA854E8597A000
:100C6000FFFFE780003945611713FFFF6700234846
:100C7000B30754030327CA0ABA9703D70700631CB4
:100C8000970003D6270063806505080897000000D9
:100C9000E780A0E5DE8505042EC697B0FFFFE7805C
:100CA00020094205931704014181C183B245E3E164
:100CB000A7FCC167FD17E38FF5F8080897C0FFFF91
:100CC000E78000FC41BFB285F9B7C165FD1501445D
:100CD000175AFF1F130A0A3A930A80022E8BAE8B13
:100CE00065BF1713FFFFE702833F184183471700D3
:100CF00083460700A207D58FD207D1832390F50042
:100D000083472700034717008D45A207D98F91839A
:100D10002310F60097C0FFFFE780A0E91713FFFF3D
:100D20006700233E1713FFFFE702C339C164014484
:100D30001759FF1F1309093493098002FD1497B056
:100D4000FFFFE780E0FE6347A40001451713FFFFA4
:100D50006700833A330534038327C90A3E958357D6
:100D60000500E38597FE0504D9BF1713FFFFE702CF
:100D700063352A8AAE89B284B68A97400000E7803C
:100D800080D819E591473E851713FFFF6700C336EA
:100D90002A894E8597C00000E780E08E2A84638E02
:100DA0000A048D476DD103570500C547E31D47FD74
:100DB0000347F9018546AD47E317D7FC8347450054
:100DC00081CF4146A6855D0597F00000E780C09E73
:100DD000814755D9AD4745BF130965012302E50099
:100DE000CA85268597100000E780606231C1A5475B
:100DF000E38B0AF82302040079B705C18357050085
:100E0000E39247F94146A685190597F00000E7806F
:100E1000A09A81472DD99947BDB74E85970000000C
:100E2000E78080F02A84954739DD130955004DBFCE
:100E30004146A685231044012311340113051900EE
:100E400097F00000E780A099228597800000E78056
:100E5000A0EA81470DBF1713FFFFE702432879710E
:100E60007C003ECCB7070A003ECE7C003ED083C754
:100E70009500B2842E8493F7F707A384F500130638
:100E8000A1002A892C00268597000000E780A0E5B4
:100E9000A16528088D0597A0FFFFE78020F090400E
:100EA0008355A10003558100854697000000E78027
:100EB00000ECAA84AA85280897C0FFFFE78040DAE3
:100EC0000356A10083558100280897000000E780A1
:100ED000C0C1300801478146A2854A8597A0FFFF1F
:100EE000E7802011854748103ED42302910202D6A4
:100EF00097D0FFFFE78060BD45611713FFFF6700D4
:100F000043201713FFFFE702831D79717C003ECC5D
:100F1000B7070A003ECE7C003ED083C79500B2845E
:100F20002E8493F7F707A384F5001306A1002A89FE
:100F30002C00268597000000E780E0DAA1652808EC
:100F40008D0597A0FFFFE78060E590408355A100E5
:100F500003558100814697000000E78040E1AA84A4
:100F6000AA85280897C0FFFFE78080CF0356A1001D
:100F700083558100280897000000E78000B73008FB
:100F800001478146A2854A8597A0FFFFE78060065A
:100F900048102302910202D402D697D0FFFFE780C7
:100FA000C0B245611713FFFF6700A3151713FFFFBA
:100FB000E702E31297000000E78060DB1713FFFFF2
:100FC000670023149757FF1F938787EA884382801F
:100FD0001713FFFFE702A310835725004111AE84CA
:100FE0002A842307B10017F5FFFF130525466C007F
:100FF0002316F10097A0FFFFE780A04191C422854E
:1010000097800000E780E0D6FD572310F400130618
:1010100020028145130554009710FFFFE780200F41
:1010200041011713FFFF6700C30D1713FFFFE7020E
:10103000630979717C003ECCB7070A003ECE7C0084
:101040003ED083C79500AA89AE8493F7F70732850F
:10105000A384F5001306A1002C0097000000E78090
:1010600080C803558100114497400000E780A0A983
:1010700015C50355A100014497B00000E780A060AA
:1010800011CD035705008357810045446318F700CD
:10109000854597000000E780E0F30144216993054E
:1010A0003900280897A0FFFFE78040CFA2852808D5
:1010B00097C0FFFFE780C0BA0356A10083558100A7
:1010C000280897000000E78040A2300801478146C9
:1010D000A6854E8597A0FFFFE780A0F148104AD46F
:1010E0002302810202D697D0FFFFE780009E456170
:1010F0001713FFFF670043001713FFFFE70283FC8E
:101100009757FF1F938787D62A8488432E8915C552
:10111000035745038357C4016311F70223260502D1
:1011200023180502410597D00000E780209C630644
:10113000090097800000E78060DB81449759FF1F1A
:10114000938949F3130A800297B0FFFFE78040BEFE
:1011500063C4A4049757FF1F938707DA9C4399C77A
:101160000355C40197200000E780C0BD6307090054
:10117000228597800000E780C0A01306400E8145BD
:1011800022859710FFFFE78080F8FD57231EF400AB
:101190001713FFFF670043F63385440383A7C90A8B
:1011A0003E95035705008357C4016317F700CA85AE
:1011B00097000000E78000E2850479B71713FFFF6E
:1011C000E70243F083C795004111AA8993F7F70717
:1011D000A384F5003285AE8497C0FFFFE78000B896
:1011E00085676378F5042A8997400000E780A0911D
:1011F000014401CD83D7040031446388270185452C
:1012000097000000E78080EF01444E85A2864A8661
:10121000A68597D0FFFFE780A09CA167938717045E
:1012200048003EC42302810002C697D0FFFFE7803A
:10123000C08941011713FFFF670003EC1713FFFF7D
:10124000E70243E89757FF1F938747C2804329C4AB
:10125000014597C00000E780002181470148C16433
:101260001CDC232E0403232004041759FF1F130939
:1012700069E001449309400EFD1497B0FFFFE78039
:1012800020AA634FA400814517F5FFFF1305857F52
:1012900097A0FFFFE780E0171713FFFF6700C3E584
:1012A000330534038327090B3E958357C5016387B4
:1012B0009700854597000000E78040E4050475BF6E
:1012C0009357050113D78700A380F50093170501F5
:1012D000C183A1832380E5002381F500A381A500BC
:1012E00082801713FFFFE70283DF2300050083C717
:1012F0001500A300F50083C725002301F50083C76F
:101300003500A301F50083C745002302F50083C71C
:101310005500A302F50083C7650093059500A3035C
:1013200005002303F5002304050032859700000023
:10133000E78040F91713FFFF6700A3DC1713FFFFD7
:10134000E70243D84111E9540DCD85CD93F9C5FF8E
:101350002E842A89AA84338AA900B7EA0400631874
:101360009A020D88854411CCB7E704009C5F8297F0
:101370002AC622866C003305390197E00000E78019
:101380000046268541011713FFFF6700E3D683A7B8
:101390008A039104829793170501C183A183A38EC9
:1013A000F4FE93570501238FF4FEA183238EA4FE40
:1013B000A38FF4FE6DB763E6D5021713FFFFE702B4
:1013C00003D2B28741113686BE8536C697E000004B
:1013D000E780E040B246410136851713FFFF670002
:1013E00043D2814636858280838705001387F500C6
:1013F0003D05FD8793F77708834607007D15860630
:10140000B58FA300F5006307B7007D17834717006A
:101410009D83DDB782801713FFFFE70243CCB7E758
:10142000040083A7070932872A863A8582971335F5
:1014300015001713FFFF6700C3CC15C181478DC18D
:101440001713FFFFE702A3C9414697E00000E780BA
:10145000003985473E851713FFFF670083CA814720
:101460003E8582801DCD1713FFFFE70243C741462B
:1014700081452A849710FFFFE78060C94146814576
:10148000130504039710FFFFE78060C80147C16799
:101490002322040438C87CC805451713FFFF6700E2
:1014A00043C60145828081473DCDB5CD1713FFFF6F
:1014B000E702E3C2B2842E891306800581452A849F
:1014C0009710FFFFE780A0C4CA8524C42685970033
:1014D0000000E780C0F64146814522859710FFFF56
:1014E000E780E0C23044A285228597000000E780B3
:1014F000C0F293040401A285268597000000E780CE
:10150000E0EEA6851305040297000000E78000EED8
:10151000228597000000E78020F585473E85171358
:10152000FFFF670003BE3E8582801713FFFFE702BF
:1015300063B94111E9540DCD85CD93F9C5FF2E84D2
:101540002A89AA84338AA900B7EA0400639844036D
:101550000D88814411CCB7E704009C5F82972AC6AE
:1015600022866C003305390197E00000E7802027D0
:10157000268541011713FFFF670003B883A78A037D
:101580009104829793170501C183A183A38EF4FE72
:1015900093570501238FF4FEA183238EA4FEA38F0E
:1015A000F4FE6DB765CD1713FFFFE702A3B1B28458
:1015B00011E605451713FFFF670003B42A842E893F
:1015C0000145EDD93C487848B3E6E700E5D6938677
:1015D000F7FFB3B7F6007D17032A4404BA9734C85F
:1015E0007CC863050A06C14913050A03B38949414A
:1015F0002295637D3601B2862E86A685970000006F
:10160000E780A0DB7C40BE9464C065B7CE862E86A2
:10161000CE8597000000E78040DAC114D2944E993D
:1016200023220404A2879306040103C7070003C60C
:1016300007038507318FA38FE7FEE398F6FE30445A
:10164000A285228597000000E78020DD2699C14908
:101650003306994063EC9900A9DCA686A68513059C
:10166000040397000000E78040D579BF8147B306A7
:10167000F4003307F6000347070083C5060085071B
:101680002D8F2380E600E39437FF3044A285228526
:1016900097000000E78060D8C1145DBF01458280DB
:1016A0000DC11713FFFFE70283A3130680058145D1
:1016B0009710FFFFE780A0A505451713FFFF670000
:1016C00043A401458280814749C5C1C51713FFFF67
:1016D000E702E3A0FC4141462E84AA846399C70433
:1016E00013860501A2878146C14503C7070003C5CC
:1016F00007038507298F3305D600034505008506B6
:10170000298FA38FE7FEE392B6FE3044A28526859B
:1017100097000000E78060D0228597000000E780F6
:1017200060F885473E851713FFFF6700839D13858B
:1017300007031D8E814522959710FFFFE780209DAE
:101740007C40130700F813060402A2972388E702DF
:1017500051BF3E8582801713FFFFE70243986D71EA
:101760002E84B284AA859010280036899700000044
:10177000E780A0D309EDD55725A050400C402800A4
:1017800097000000E78040E27DD5FD142104F5F4C8
:101790002C004A8597000000E78020F3814761DD37
:1017A0003E8551611713FFFF6700A3951713FFFFD5
:1017B000E702E39241112EC432C62C000546970081
:1017C0000000E78080F941011713FFFF6700639372
:1017D0001713FFFFE702A39001112A842EC602C847
:1017E00002CA02CC02CE97E00000E780C023B246D6
:1017F0002A86A285080897000000E78060FB137521
:10180000F50F05611713FFFF6700A38F1713FFFF85
:10181000E702E38C7971B2872A8421462308B1005C
:1018200013051101BE853AC436C697E00000E78073
:1018300000FBB24693059101368597000000E780D2
:1018400060A82285141035460C0897000000E78038
:1018500020F62A84224701E921460C103A8597E0B8
:101860000000E780C0F7228545611713FFFF67007E
:1018700043891713FFFFE70283867171AE84AA853F
:101880000A85328497000000E78060BB11C90A8690
:10189000A685228597000000E78020B8814711E1E6
:1018A000C5473E854D611713FFFF6700838517030A
:1018B000FFFFE702C37F1D712A8AB289BE843546C5
:1018C0008547130511012E8CB68A3A8BC28C468D42
:1018D0002308F10097E00000E78060F010100C088A
:1018E0005285231F010097000000E780C0F82A847A
:1018F0003DEDA1476313FD089307900591E0E5478F
:101900003546E2851305110113990A012308F100F8
:101910001359090197E00000E78060EC1357890034
:1019200093978A00D98F90080C085285231FF100E5
:1019300097000000E78020F42A8415E9A1E493874A
:10194000FA0091831379F9003EC6631309004149F7
:10195000668B8144C14B854DB247639F970C6A8665
:101960008C0033855C0197E00000E78040E722852A
:1019700025611703FFFF6700437793079004C9F0C1
:10198000A547BDBF834701050947C14B2308F100A7
:1019900083471105A58FA308F10093872400814494
:1019A00063E1FB04014714083386E6008C08B38624
:1019B000E400BA95DA9683C6060083C505000507DC
:1019C000AD8E2300D600E390E7FE4147639CE70419
:1019D00090080C08528597000000E780C0E925D1E7
:1019E00081A0B3069B00BA871008B305F6009008E3
:1019F0003E9603C506000346060085078506298E28
:101A00002380C500E39277FF998F90080C085285D8
:101A1000BE9497000000E78000E68947014749D15E
:101A20002A84B1B790083E96034606001408BE9675
:101A30002380C600850759BFB24785046387971482
:101A400081471808B306F70098083E973386F900D7
:101A500003470700034606008507318F2380E60011
:101A6000E39177FF90080C08528597000000E7800B
:101A700080E05DF53546E285130511012308B101CB
:101A800097E00000E780A0D5139704014183939766
:101A900084002183D98F10180C085285231FF10070
:101AA00097000000E78020DD25FD8147101833876F
:101AB000F9003E960347070003460600B306FB0005
:101AC0008507318F2380E600E39277FF65A8180829
:101AD000B306F70098083E973386F90003470700DE
:101AE000034606008507318F2380E600E3E127FFE8
:101AF000CA87639E770990080C08528597000000FA
:101B0000E78060D711FD81479800B306F700900881
:101B100018103E973E9603470700034606008507C8
:101B2000318F2380E600E39177FF3546E285130588
:101B300011012308B10197E00000E78040CA139724
:101B400004014183939784002183D98F10180C08D6
:101B50005285231FF10097000000E780C0D1E311F8
:101B600005EC814710183387F9003E9603470700BC
:101B700003460600B306FB008507318F2380E6008D
:101B8000E3E227FFC109410BC1BB814785B7940838
:101B9000BE9683C6060018083E972300D700850727
:101BA00089BF638006321703FFFFE7024350597174
:101BB0002A84BE89B28B85473546130511022E8BC8
:101BC000468C4289BA8A368A2300F10297E00000E7
:101BD000E780E0C010180C1022852317010297003F
:101BE0000000E78040C963180512A147631FFC0687
:101BF0009307900563930900E5473546DA85130599
:101C0000110293140A012300F102C18097E0000041
:101C1000E780E0BC93178A0013D78400D98F90081F
:101C20000C1022852317F10297000000E780A0C462
:101C30007DE1639209049307FA00BD88918391E0E6
:101C4000C144C207C183DE8C814A3EC6414DB247C2
:101C500063E2FA0E6286B3854B01881097E00000BC
:101C6000E78080B54DC93D557DA093079004E3966C
:101C700009F8A54759B7834701050947C14C230017
:101C8000F10283471105B3C7F900A300F10293875E
:101C90002900814963E1FC04814618103306D7000E
:101CA0008C083387D900B69556970347070083C53C
:101CB000050085062D8F2300E600E390D7FE4147FF
:101CC0006390E70690080C10228597000000E780DB
:101CD00080BA35D189A0B3863A01BA871010B3050E
:101CE000F60090083E9603C50600034606008507E9
:101CF0008506298E2380C500E39297FF3387EC4049
:101D000090080C102285BA9997000000E780A0B6D1
:101D10008947014741D165611703FFFF6700E33C35
:101D200090083E96034606001410BE962380C60017
:101D3000850779B7B247850A93990A01939D8A006E
:101D400093D909016391570F85473546DA85130505
:101D500011022300F10293D9890097E00000E78087
:101D600000A8B3ED3D0190000C1022852317B103AC
:101D700097000000E78020B059FD8147A68963EAFB
:101D8000970626860C084A8597E00000E78020A584
:101D900081471810B306F700100898083E973E9642
:101DA00003470700034606008507318F2380E600BE
:101DB000E3E197FE639FA90590080C102285970028
:101DC0000000E78040AB21F981479810B306F70087
:101DD000900818183E973E960347070003460600F2
:101DE0008507318F2380E600E391A7FF4109C10CED
:101DF000B9BD18089000B306F7003E963387FC0083
:101E000003470700034606008507318F2380E6005D
:101E1000B5B798084E97034707001C10CE9723804C
:101E2000E700850941BF85473546DA85130511026C
:101E30002300F10293D9890097E00000E780209AFF
:101E4000B3ED3D0190000C1022852317B1039700DC
:101E50000000E78040A2E31005EC814718089000DD
:101E6000B306F7003E963387FC000347070003469E
:101E700006008507318F2380E600E391A7FF4146E6
:101E80000C084A8597E00000E780609581471810AC
:101E9000B306F700100898083E973E9603470700E0
:101EA000034606008507318F2380E600E391A7FFF4
:101EB00090080C10228597000000E780C09B1DD57C
:101EC00099BD7D5582801703FFFFE7024321011171
:101ED0002A842E8593055100328902C002C202C4B1
:101EE00002C69304740097F0FFFFE780A03D1D46F3
:101EF000A6851305910097E00000E780408E10084A
:101F00008A854A8597000000E780E09619ED9307DF
:101F10001400180883C60700034607008507050755
:101F2000B18EA38FD7FEE397F4FE05611703FFFF81
:101F30006700231D1703FFFFE702C3182E848C419F
:101F40004111AA89838715003289914463D3070020
:101F5000A1449747FF1F9387A7489C43A1C7C1CAC5
:101F60008D472310F10083C725004A852301F10026
:101F700083C73500A301F10083C745002302F100A8
:101F800083C75500A302F10083C765009305910044
:101F9000A30301002303F1002304010097F0FFFFD6
:101FA000E78040320C404A860A8597F0FFFFE780C1
:101FB00080330328040083564400A6881D08814707
:101FC0000147E51642868A854E8597000000E78026
:101FD000408E2A8919E5A685228597B0FFFFE78004
:101FE000E0C14A8541011703FFFF6700E3104A86FD
:101FF0000A8597F0FFFFE780002F6DB71703FFFFFB
:10200000E702430C2E848C414111AA898387150075
:102010003289914463D30700A1449747FF1F9387F8
:10202000273C9C43A1C7C1C68D472310F10083C73D
:1020300025004A852301F10083C73500A301F10083
:1020400083C745002302F10083C75500A302F100B6
:1020500083C7650093059100A30301002303F100EA
:102060002304010097F0FFFFE780C0250C404A865B
:102070000A8597F0FFFFE780002783564400032876
:1020800004008A85858EC2061D08C1822312D400F1
:10209000A68881470147E51642864E8597000000D5
:1020A000E78060B041011703FFFF6700E3044A8641
:1020B0000A8597F0FFFFE78000234DBF1703FFFF5E
:1020C000E702E301B335B000011185052A89131534
:1020D000F601336515012308B1009305110136841B
:1020E0003AC632C03EC442C297F0FFFFE780801D6F
:1020F000A2471248425593D68700230BF10093055F
:10210000910193578800A30AD100A30BF100230C7F
:10211000010197F0FFFFE780E01A324702460328EB
:102120000400B337E000835644009207914411C283
:10213000A1444A85A68842860C0897F0FFFFE780F5
:1021400040772A8919E5A685228597B0FFFFE780A9
:10215000E0AA4A8505611703FFFF670083FA1703AA
:10216000FFFFE70223F601113EC68647B335B000F4
:102170008505AA891315F6015D8D2308B100930525
:10218000110136843A89B28442C446C297F0FFFFF7
:10219000E780401322489248164593578800A30AC7
:1021A000F1009305910193D78800230B0101A30B44
:1021B000F100230C110197F0FFFFE780A0103247D8
:1021C000104083564400B337E0009207032809000B
:1021D000914891C0A1480C084E8597000000E78007
:1021E000809CAA8401E9835544004A8597B0FFFF8B
:1021F000E780C0A0268505611703FFFF6700C3EFD6
:10220000AA959307F00F170701001307A77B631721
:10221000B50013C5F7FF1375F50F828005058346DA
:10222000F5FFB58FBA9783C70700D5B703574500A9
:1022300014419307F00F170601001306A67836978E
:1022400042074183139506014181631BE500AD8F71
:10225000B29703C50700130515F3133515008280E7
:10226000850603C5F6FFA98FB29783C70700D9BFBC
:102270001703FFFFE702A3E6B28736842E86BA86ED
:10228000AA853E85BA8497F0FFFFE7806052634FCE
:102290000500228597D00000E780E0782A86A68690
:1022A000A285268597F0FFFFE78080501703FFFF88
:1022B000670023E51703FFFFE702C3E05D712A8B88
:1022C000AE8A170501001305656D2C00B284368AAD
:1022D000BA893E8997F0FFFFE780C04F2A845DE10D
:1022E00034104146DA85280097F0FFFFE780404C24
:1022F0002A8449E98547A303F100A6C29307710028
:102300002408BEC4A68685470D462C18281002DC7A
:1023100002DED6C0BEC697F0FFFFE78000442A84E5
:1023200035E183477102A6860D4693F7F707230030
:10233000FA00C1473EDE2C188947281026DCA3038B
:10234000F10097F0FFFFE78040412A8405ED414608
:10235000A6854E8597D00000E78060488D47A68609
:102360000D462C182810A303F10097F0FFFFE7801B
:10237000C03E2A8401E94146A6854A8597D00000DF
:10238000E780E045228561611703FFFF6700C3D640
:102390001703FFFFE702A3D497F700009387C7A1B5
:1023A000984383C7470079712A89AE8417050100D5
:1023B0001305455F0C083AC42306F10097F0FFFFB0
:1023C000E78040412A8405ED14104146CA8508087B
:1023D00097F0FFFFE780C03D2A8415E114081546F9
:1023E0002C00081097F0FFFFE780803C2A8401E969
:1023F00021462C08268597D00000E780403E2285A4
:1024000045611703FFFF6700C3CF1703FFFFE70214
:1024100003CD97F700009387279A9C477971AA8488
:102420002E8417050100130565580C083EC697F069
:10243000FFFFE780203A0DE914104146A685080801
:1024400097F0FFFFE780C03605E1140811466C00E5
:10245000081097F0FFFFE780A03519E58347F101E9
:1024600093F7F7032300F40045611703FFFF6700AC
:1024700043C91703FFFFE70283C63688A148814797
:102480000147E54697F0FFFFE780A0421703FFFFF3
:10249000670023C71703FFFFE70263C43688A1481C
:1024A00081470147E54697F0FFFFE780C06F1703BC
:1024B000FFFF670003C51703FFFFE70243C20111D7
:1024C0002A842E850C0832C697F0FFFFE780803003
:1024D00009ED3247970601009386C64B1008C145A7
:1024E000228597000000E780E0D805611703FFFF11
:1024F000670023C11703FFFFE70263BE4111C14715
:102500002EC032C48A8509463EC23EC697F0FFFF00
:10251000E780A02441011703FFFF670083BE170374
:10252000FFFFE702C3BB4111AE8613061009AA855F
:102530000A8502C002C202C402C697F0FFFFE7800C
:10254000202741011703FFFF6700A3BB1703FFFF0D
:10255000E702E3B83287970601009386A6452E86E8
:102560009305000297000000E780C0D01703FFFF2B
:10257000670023B91703FFFFE70263B67971C1470C
:102580002ACC2ED032D42C080D4628003ECE3ED286
:102590003ED602C402C602C802CA97F0FFFFE78017
:1025A000C01B45611703FFFF6700A3B51703FFFFBB
:1025B000E702E3B20111AA842E8417050100130576
:1025C000E53F8A8597F0FFFFE780C02015E51408F6
:1025D0004146A6850A8597F0FFFFE780601D09ED5B
:1025E0008347E1010347F101A207D98FCA07C983D5
:1025F0006177D98F2310F40005611703FFFF67008F
:1026000043B015CD1703FFFFE70263AD9747FF1FE8
:102610009387878A90439745FF1F9385258A17459F
:10262000FF1F1305658597D00000E78000C517459B
:10263000FF1F130565841703FFFF670083AC174571
:10264000FF1F1305658382808DCD1703FFFFE7020F
:1026500003A99747FF1F93872786944301112E8470
:102660000A869745FF1F9385658597D00000E78010
:1026700040C60A850294014505611703FFFF670004
:1026800043A87D5582801703FFFFE70243A597D03B
:102690000000E78080D19747FF1F23AFA78017F581
:1026A000FFFF1305E5C997B00000E780C07417036A
:1026B000FFFF670003A51747FF1F13072782931724
:1026C000150008433E95FD572310F500828017033F
:1026D000FFFFE702C3A02A84084009E51703FFFFB4
:1026E000670023A21C4158401CC06313E5005CC076
:1026F0008347550023200500F99BA302F50097A00E
:10270000FFFFE780207CC9BF1703FFFFE702839B21
:102710009737FF1F9387877E98432A8411CB83477F
:10272000350093F7070289C70355050089450297CD
:102730001305440197B00000E780403B8355040037
:102740000355E40097300000E780A00C485819C5F5
:1027500097A0FFFFE7800077232A04021305840374
:1027600097000000E780E0F68144B1499790FFFFB1
:10277000E780406663CBA40283473400232004042F
:1027800093F727FCA301F40000489790FFFFE78030
:10279000606513161500814522859700FFFFE780CD
:1027A00000971703FFFF67002395B38734030329BE
:1027B000040385043E994A8597000000E78060F194
:1027C0002304090065B78347350093F7070299E3AF
:1027D000014582808357E500E39CB7FEC167FD1782
:1027E0006316F60005458280054599A81703FFFF8B
:1027F000E702E38E93170601C187B2842A84014958
:102800006359F002835705009DCB01456367F600CD
:10281000034584003E953325A6001375F50F0DA0E2
:102820001C4813171900BA9783D70700E38E97FA4D
:1028300005099790FFFFE780E05AE343A9FE0145B1
:102840001703FFFF6700E38B1703FFFFE702838790
:10285000AE89AA849790FFFFE780804E2A8497D0A4
:10286000FFFFE780A02EAA86014713068401970583
:102870000000938585E41735FF1F13056566979063
:10288000FFFFE78000152A8925C98C441304C50081
:1028900022859E0593F5050897A0FFFFE780403C41
:1028A000CC4083877400E18163DD070493E505086C
:1028B000228597A0FFFFE780A03A0D46938544004C
:1028C000228597A0FFFFE780C03683D504002285CC
:1028D00097A0FFFFE780E03D83D52400228597A0E5
:1028E000FFFFE780003D03D6490083A5090022854C
:1028F00097A0FFFFE780E0334A8517F3FEFF6700EC
:10290000A37F93F5F5076DB717F3FEFFE702237D6D
:1029100001112A84328532C697A0FFFFE780E027A5
:102920009780FFFFE780E02C835704001737FF1FD5
:10293000130747743246231BF100930700F8A30DD9
:10294000F1001C471843231AA1008983858BB30724
:10295000F740B28548083ECE231C0100230D01003C
:1029600097000000E78080EE056117F3FEFF670027
:10297000437917F3FEFFE702E374004101453DC4CC
:102980009304C40026853289AE8997A0FFFFE780B3
:10299000C02495452A8A2685035B040197A0FFFF82
:1029A000E7802021268597A0FFFFE780603E8D45C8
:1029B000AA8A268597A0FFFFE780A01F268597A0FB
:1029C000FFFFE780E03C5C48420A135A0A01D297B5
:1029D0005CC423186401814763983A0146054D8120
:1029E000330625419337160013F5F70F17F3FEFF53
:1029F0006700837017F3FEFFE702E36B89692A8B98
:102A0000AE8B328AB68A81440144314CFD199790CD
:102A1000FFFFE780203C63CDA4009790FFFFE78095
:102A2000603E018D33B5AA0017F3FEFF6700236CEB
:102A30003389840383270B003E9963170A00834779
:102A4000890085043E94E1B703560A00DE854A8575
:102A500033F6C90097000000E780E0F16DD105452D
:102A6000E1B717F3FEFFE702836701112A847C00B8
:102A70000355E5003ECAB70707003ECC7C003ECEBA
:102A800097200000E78020082A898545480897A0FC
:102A9000FFFFE78020399945480897A0FFFFE780AE
:102AA000E015AA844A8597200000E780A0082380CB
:102AB000A4009737FF1F9387E75B9C43416613068B
:102AC00006F09396870113D78701558F93D6870019
:102AD000F18E558FA207B706FF00F58FD98F1146EB
:102AE0002C00138514003EC497D00000E78020CF4F
:102AF0005008A38204008945228597000000E780E2
:102B0000E0E019C9AA851305840397A0FFFFE780B9
:102B1000E0313C4085073CC0056117F3FEFF6700CC
:102B2000435E17F3FEFFE702835B9790FFFFE780AA
:102B3000602D2A8405049790FFFFE780A02B3305C2
:102B4000A402F14791453305F50297200000E78084
:102B500020BA11E5655517F3FEFF6700835A9737D2
:102B6000FF1F23A5A7389790FFFFE780A0292A849D
:102B700005049790FFFFE780E0273305A40289450D
:102B8000060597200000E780A0B669D59737FF1F9C
:102B900023A6A7349790FFFFE780C0262A84050468
:102BA0009790FFFFE78000253304A4029737FF1FAB
:102BB000239887329790FFFFE780C0242A8497905C
:102BC000FFFFE7802023930714003385A702973780
:102BD000FF1F2398A730970701009387E7A11737B6
:102BE000FF1F2323F7300145BDB717F3FEFFE702B0
:102BF000634DAA842E8901449739FF1F9389894721
